:020000040800F2
:1000000000A000201938010831EA00084D28010835
:100010002FEA00082DEA00082BEA00080000000083
:1000200000000000000000000000000029EA0008B5
:1000300027EA00080000000025EA00085F12010816
:1000400081380108813801088138010881380108A8
:100050008138010881380108813801088138010898
:100060008138010881380108813801088138010888
:1000700081380108A54D0008BBD900088138010866
:100080008138010881380108813801088138010868
:1000900091EA000881380108813801086D120108D1
:1000A0005FD6000889D600088138010899D6000873
:1000B0007DD600086DD60008813801088138010816
:1000C0008138010881380108813801088138010828
:1000D0008138010849D800083DD8000831D8000807
:1000E000711201088138010815EA000881380108F9
:1000F00081380108813801088138010881380108F8
:10010000000000000000000000000000813801082D
:1001100081380108813801088138010881380108D7
:1001200081380108813801088138010881380108C7
:10013000813801088138010800000000000000003B
:100140008138010881380108813801080000000069
:10015000000000000000000000000000000000009F
:10016000000000000000000081380108813801080B
:1001700081380108000000000000000000000000BD
:080180000000000081380108B5
:100188002DE9F04F2DED068B7D4E7E4B3360AFB0E1
:10019800002373600FF0B4FF18B90FF0D5FF0BF010
:1001A800BDF90BF079FA784A137843F0010313701C
:1001B800764B4FF47001C3F88810002309930A9313
:1001C80003F1804303F504339B46196841F48031F9
:1001D80019600492DBF8003003F400330A93099B9A
:1001E800013309930A9B1BB9099BB3F5A04FF1D1C1
:1001F800DBF8003013F4003318BF01230A930A9B7D
:10020800012B00F08680614D614BEB60DBF82430F8
:10021800B360DBF82430DFF8ACA1DFF8AC8143F041
:100228008073CBF82430DBF8143043F4FC032EAC95
:10023800CBF8143003238DF86A3041F6FF7324F8A5
:10024800503D4FF09040214604F09EFE4FF6FF735C
:100258005048ADF86830214604F096FE50462146D5
:1002680004F092FE4C48214604F08EFE4B4821468D
:1002780004F08AFE21464A4804F086FE20460AF029
:10028800D9FA1A9B474AB3FBF2F3474ADFF83CE135
:100298001360464B464A4FF00009C3F80090C3F874
:1002A8000490444B5A60F02285F823200722C3F8B3
:1002B8000890414D1A60D8F80830CEF800300FCDBC
:1002C80027460FC7DBF8143095E8030043F40023F2
:1002D80087E80300CBF81430DBF8143043F400232C
:1002E800CBF81430DBF8143043F40023CBF8143087
:1002F8004FF40043CAF818304FF48043CAF8183056
:100308004FF40053CAF81830A5F11003774602934A
:100318005EE02A4B12221A60DBF80430CBF8043076
:10032800DBF80430CBF80430DBF8043043F48063A6
:10033800CBF80430DBF8043023F47C13CBF804301A
:10034800DBF8043043F4E813CBF80430DBF8003072
:1003580043F08073CBF80030DBF80020184B920193
:10036800FAD55A6822F003025A605A6842F002022B
:100378005A60DBF8043003F00C03082BF9D142E78C
:100388007801002023AE0008782F002000ED00E05F
:100398000005FA0500040048000C00480010004859
:1003A8000014004840420F00042B0020FC2A0020C3
:1003B8003F19010010E000E06071010800200240D0
:1003C800001002400008004870120020741A002033
:1003D80009F1040154F80900214409F1080904F05D
:1003E800D3FDB9F1180FF3D1642010F025FFA02236
:1003F800B848002115F011FADBF81C30B64A43F072
:100408000303CBF81C30DBF8183043F48433CBF803
:100418001830DBF8143043F42023CBF8143002F101
:10042800B00C937B506892F80FE003F00701DB08EB
:1004380000EB83038900186A4FF00F090EFA01FEDA
:1004480009FA01F120EA01011962196A10324EEA2B
:10045800010162451962E4D10023DFF8B09209F185
:100468000C020021995401330B2BF6D1FF2389F894
:10047800173089F8183089F8193089F81A30974BED
:10048800974DDFF88CA21D60964B04221A705046D7
:10049800302215F0C2F914238AF800300223012211
:1004A8008AF82430904B8AF8182098F805A083F829
:1004B80000A08E493F68A5F5F173C9F81C30A5F571
:1004C80091730B608A4B03EBCA035B78C9F8203041
:1004D800BB0648BFC9F820200023864A40F2DC51F9
:1004E80022F813100133082BF7D113A800211C227E
:1004F80015F093F9BAF10E0F03D00AF0EF03082BA9
:1005080002D101238DF85E30022008F05FFD18B19A
:100518004088003018BF0120C7F340038DF85230DF
:10052800C7F380138DF85530C7F340338DF84C303E
:10053800C7F3C03300F001008DF84F3017F40063A3
:100548008DF8510007D098F8843103F1FF3EDEF1B1
:10055800000343EB0E038DF85030C7F300438DF8CA
:100568005630336AB8F844E1ADF862E0003318BF9A
:1005780001238DF85730C7F300538DF85830B8F879
:100588004631ADF85C30B8F85231ADF85A30C7F39F
:1005980080438DF8533098F85431181C18BF012047
:1005A800FD0407F00101C7F3C00248BF524F8DF8A0
:1005B8005400B8F8500144BFB7F84C71ADF86270F8
:1005C800B0F5FA7F8DF84D108DF84E20ADF860002B
:1005D80002D90BB9ADF8623098F8D431474886F89B
:1005E8002430002386F8253043709DF85E30002BB8
:1005F8000CBF0023022301B902B10133029A02EBB6
:1006080083054FF00009AB699A1E143302920593D3
:10061800029A32F8023F02924FF6FF72934200F0BC
:10062800A2819DF85100190ADAB2CBB278B12A4DED
:10063800334F05EB02156868B84208D12889B0F530
:10064800806F00F08B81B0F5006F00F087819DF816
:10065800560078B11001204F3D183F58294887426D
:1006680000F07C816868B0F1904F03D1A87B062820
:1006780000F074819DF8520050B1174D224F05EBE0
:1006880002156868B84203D12889012800F06681FC
:100698009DF84F0050B1104D1B4F05EB02156868CF
:1006A800B84203D12889042800F058819DF85000E9
:1006B80050B1094D144F05EB02156868B84203D1D3
:1006C8002889022800F04A81022923D19DF84C107C
:1006D80024E000BF4C2B002038920108842A002017
:1006E80062140020411200206C090020682C0020B0
:1006F8008C970108A8110020701200209D0100208D
:100708000004004800440140000800487801002027
:10071800882A0020012904D19DF84D10002900F0F5
:100728001D819DF85710C54D170151B19DF85E10F8
:1007380039B9511F032904D8E959B1F1804F08BFCD
:1007480004239DF858103D4431B19DF85E1019B945
:10075800043A032A40F2EA80012B4AD1DFF8E88202
:10076800FF2388F86C3088F86D30B44BC8F87C509B
:10077800DA194FF0000A02F1080C517B506812890F
:10078800ADF868208DF86A1002221AA988F870A0BE
:100798000693CDF80CC08DF86B2088F828A0C8F80F
:1007A8002CA0C8F830A0C8F834A0C8F868A088F809
:1007B8006EA088F86FA004F0E7FB069BDDF80CC07C
:1007C800D8599CF80210524604F032FA284611F023
:1007D80053FA9B4BC8F880309A4BC8F88430C8F855
:1007E80088A0284608F1800108F184020CF0C2FFB5
:1007F800B4E0022B48D15FFA89F21C2101FB02FC0C
:10080800914ACDF81CC002EB0C088C4A06920121D3
:1008180088F87010D11901F108024FF0000A4868F1
:10082800098992F805E088F87190ADF8681088F8A1
:1008380072A01AA988F87AA0C8F87C508DF86AE0E6
:1008480003928DF86B3004F09FFB039B069A99780E
:10085800D059524604F0ECF9284611F00DFA7A4BBB
:10086800DDF81CC0794AC8F880209C44784AC8F84A
:1008780084200CF18001C8F888A028460A1D0CF0D5
:1008880079FF09F1010969E0032B4DD19DF8533037
:100898006D4FDFF8F08103B39DF8543097F826C008
:1008A800DFF8BCA1CDF80CC053B16A4BBDF860208D
:1008B800B3FBF2F22846082192B2BDF8623003E099
:1008C800284608214FF6FF7204F087FBDDF80CC0BC
:1008D80048F82C00C0F80CA020E0BDF8602097F87C
:1008E80026A0BDF86230B2F5FA7F0BD95949B1FBA1
:1008F800F2F22846082192B204F06FFB564B48F8F2
:100908002A000AE05549B1FBF2F22846012192B2C9
:1009180004F063FB524B48F82A00C36097F826306E
:10092800013387F8263019E0042B17D1464FBDF85C
:100938005A2097F82580494B93FBF2F22846BDF8D8
:100948005C30012192B204F048FB97F8253007EBA0
:1009580088080133C8F8500187F82530029B059AAA
:1009680093427FF455AE96F8252086F870213D4ACB
:100978003D4B1778A7F117020025022A1D709E46E5
:100988001AD8F3692B44D3ED007AF5EE407AF1EEEC
:1009980010FA02D1336A63BB26E0344A05EB020C35
:1009A8000FCB8CE80F009EF8003010350133C02DB6
:1009B8008EF80030E5D1EDE72D4B13F837808EF82F
:1009C800008003EBC703D3F80490B9F1000FE1D01E
:1009D8004545DFDA254A2B0103EB020C4B440FCBCC
:1009E80001358CE80F00F3E7224D2B68DA044DD46B
:1009F8001DE0214B214A13F83700107003EBC703A1
:100A08005D68002DF0D000238342EDDAC3EBC3010B
:100A18006A18DFF874C0D2F8008041F80C8001EB46
:100A28000C069188B1809279B2710133ECE707F036
:100A3800EF03082B124B49D14AE000BF3892010856
:100A4800CD490008AD4A000878010020354D00085E
:100A5800A549000800127A00CD4A000840420F005C
:100A6800BD4A00086C090020482B0020A808002077
:100A78008C970108741A0020C07E0108F42B00200E
:100A8800901A0020182B0020F52B00209EF800203B
:100A9800012ACCD9AC4B03EB02121032103393422B
:100AA800C5D053ED047AB6EE007A67EE877A43ED47
:100AB800047A53ED057A67EE877A43ED057A53EDAC
:100AC800037A67EE877A43ED037AE7E70E2F08D1BA
:100AD8001A7842F010021A70182F08D110F030FE60
:100AE80005E01A7822F010021A70192FF5E710F0B5
:100AF8000BFE2B68954D5B035EBF954B01221A7068
:100B0800049B049A1B7843F0040313704FF40053BA
:100B1800ADF86830DBF814304FF0020A012743F4CF
:100B2800802321468DF86BA028468DF86A70CBF893
:100B3800143004F029FA874B874A1A60002010F015
:100B480095FBDBF8183043F48053CBF81830DBF80A
:100B58000C3043F48053CBF80C30DBF8143043F4FA
:100B68008023CBF814302B6A23F470432B622B6A52
:100B780043F4A0432B622B6A23F470232B622B6A65
:100B880043F4A0232B622B6A23F470032B622B6A95
:100B980043F4A00300262B624FF0030838232846AD
:100BA80021461A938DF86CA08DF86D808DF86E60D3
:100BB8008DF86F6009F0ACFFDBF80C20674D42F44C
:100BC8008052CBF80C20DBF80C2022F48052CBF8B2
:100BD8000C20634A918821F480510904090C918002
:100BE800918889B241F480519180118801F4415172
:100BF80041F4457141EA08011180918821F470613E
:100C08000904090C41F4E0619180918B21F40061A1
:100C180009040723090C91831382118889B241F0D2
:100C2800400111804F4A1560DBF8142042F400326D
:100C3800CBF81420DBF81C2042F48002CBF81C20EF
:100C4800DBF8302022F02002CBF83020DBF830200F
:100C580042F080524FF0904942F02002CBF8302009
:100C6800D9F8242022F0F002C9F82420D9F8242049
:100C780042F04002C9F82420D9F8242022F47062F6
:100C8800C9F82420D9F8242042F48062C9F8242025
:100C980048464FF4007221468DF86CA01A928DF8E0
:100CA8006E608DF86F608DF86D8009F031FF4FF43C
:100CB8008062484621461A9209F02AFF2A682A4B80
:100CC80022F001022A602968284A0A402A60284A34
:100CD8002A612A683A432A60AE60EE60AE60AA686C
:100CE80042F40042AA602A682A606A6822F07842C0
:100CF80022F400426A602A683A432A601C681D4D43
:100D08000393284604F4004331461022029314F05A
:100D180084FD039B8DF83DA004F4006914EA0A04DD
:100D28008DF83E608DF83F608DF83C809A4625D05E
:100D380011480E970EA909F0EBFE06232B70072326
:100D48006E70EB70AF701AE0B00800200004004825
:100D5800D80D00208C2F00205911010800580040A0
:100D68000030014074110020741A0020FFE0CF0009
:100D7800300E5000DC1E0020000800482746029B69
:100D880073B1042382480E930EA909F0C1FE08230B
:100D98002B710723EB7101236F711F44AB71FFB2F5
:100DA800B9F1000F0DD0022379480E930EA909F06E
:100DB800AFFE07232B73EB7301236F731F44AB73D1
:100DC800FFB20EA9082372480E9309F0A1FE092369
:100DD8002B7207236F72EB720123AB721F44DBF88F
:100DE8002C306C486B4C23F4F873CBF82C30DBF8C0
:100DF8002C3043F4D873CBF82C30DBF8143043F0A4
:100E0800805343F00103CBF8143009F048FC1AA8CA
:100E180009F01AFC604B1A93FFB2604B1B93012F29
:100E28004FF000030CBF1A4680221F924FF48072C5
:100E380020924FF4806221922022204622921AA901
:100E48004FF400521C931E9323922493ADF87470B0
:100E580009F007FC236843F0010323604FF0A04426
:100E68000A20A36823F04053A360A36843F080538B
:100E7800A36010F0E1F9A36823F08043A360A3689E
:100E8800A360A36843F00043A3604FF0A0429368B7
:100E9800002BFADB9368424923F040539360936830
:100EA80043F00053936088683E4B034043F4683333
:100EB8008B60D1683C4B0B4043F40053D360136BF9
:100EC800013F23F00F031F431763002401232A194E
:100ED800917800297AD05E1C042B2F5DD078F6B269
:100EE8004FF0A04E0ED803EB43035A00DEF8301043
:100EF8001F23934021EA030107FA02F30B43CEF8BC
:100F0800303031E0092B0ED8053B06225A43DEF873
:100F180034101F23934021EA030107FA02F30B431D
:100F2800CEF8343020E00E2B4FF006010ED8A3F196
:100F38000A024A43DEF838C01F2393402CEA030113
:100F480007FA02F30B43CEF838300DE00F3B01FBF4
:100F580003F2DEF83CC01F2393402CEA030107FA92
:100F680002F30B43CEF83C30092F4FF0A0421DD9B5
:100F78009369A7F10A0303EB430397690721994093
:100F880027EA0101916191699840084390611CE04A
:100F9800000800480800024040000050EC1E0020F5
:100FA80000030050E010FCFF07C0FFFD53697B1EE3
:100FB80003EB430357693821994027EA010151613E
:100FC8005169033398400843506133460434102C68
:100FD8007FF47DAF4FF0A042936843F00103936024
:100FE8004FF0A0431A68D707FAD5DA68A04D22F067
:100FF8000202DA60DA6842F00202DA60DA6842F085
:101008000102DA609A6842F004029A60B5F8583131
:10101800002B40F0C087B5F95A21002A40F0BB8761
:10102800B5F95C21002A40F0B68795F8693102933A
:10103800904B914C1B689148B3F8623003930021A0
:101048000C224FF0000895F85FB195F86A7114F01A
:10105800E4FB002114228A4814F0DFFB41460C22ED
:1010680084F8718184F8728104F5BA7014F0D5FBA4
:10107800844BC4F88031232010F0DEF8752001215C
:101088000BAA0CF02FF9B0B17F4BC4F878317F4B25
:10109800C4F87C314046432301210CAA84F87431FA
:1010A8000CF020F99DF8303003F07E038DF83030D5
:1010B800002849D151E094F884317BBB74494A69CE
:1010C80042F400324A61102603224FF001084FF023
:1010D80090401AA98DF86D208DF86E308DF86F301C
:1010E8001A968DF86C8009F013FD4FF09043694A09
:1010F8009E61138823F04003B340F34013801388A4
:1011080023F03803B340F34043F0080313801388F7
:101118009BB243F04003138084F884817520012139
:101128001AAA0CF030F99DF86830702B5AD10523B3
:1011380084F87131432384F87431574BC4F87831FB
:10114800564BC4F87C314DE0682B06D1012384F856
:1011580071311D2384F8743144E09DF82C3003F07C
:101168007E03682B8DF82C3037D10223062084F8B3
:1011780071310146D4F878311AAA98479DF86D1054
:1011880001F001029DF86B1001F001014B0043EAE8
:1011980082019DF8692002F001030B430AD05BB27B
:1011A800012B01D1002302E0022B0FD1012384F887
:1011B800723117E0304B0C20D3F8783101210EAA98
:1011C80098479DF8383013F00F0303D1032010F02F
:1011D800AFF807E0042BE9D1E4E7702B04BF042340
:1011E80084F871312E4B94F8710100221A70021F95
:1011F800012A994615D8224B2A4A1A602A4A5A6067
:101208002A4ADA602A4A1A612A492B4A042389F8A9
:10121800003007230B70136843F0010313608846FE
:1012280003E0012010F084F871E159460A2928BF2B
:10123800002101238B4040F202261E40002E45D19A
:1012480040F2FD161E40002E40D004283CD10B4B26
:101258001A4919601A4959601A4B04211970082350
:1012680088F80130136843F00203136035E000BFCB
:1012780070120020B811002078010020D82A002020
:101288007027002088710108EDD2000805D20008F7
:1012980000100240003001408FD3000873D30008CB
:1012A8008427002011D500082DD1000811D100088D
:1012B80090C1793D040100208C1A0020C9D500088E
:1012C80075D10008A82F00200528C0D001294FF0AB
:1012D800000BAAD8684B83F800B0042F71D80126F8
:1012E80006FA07F313F0160B72D113F0090F66D044
:1012F8000A200FF0A1FF7720A02132460EAB03F0A1
:1013080059FF002864D01E213246772003F0CEFF13
:101318000FF076FF07460FF073FFC01BB0F52F6F75
:10132800F9D3ABF160010027C9B202221AAB7720CA
:101338008DF868708DF8697003F03CFF9DF869308E
:101348009DF8682043EA02224C4B03F5C3712BF841
:1013580001200BF1020BBBF1100FE2D1B3F894217D
:1013680002F47F4EA3F894E102F00F0101203B46FE
:1013780027F001022244B2F88621002A18BF002073
:10138800FE0703D5D2B25340082202E083EA1223B3
:10139800FAE71E0448BF83F4C053013A4FEA4303F7
:1013A800F7D10137102FE3D14EEA0102A4F89421B6
:1013B80070B9C3F30333994200F0D08508E0012FD8
:1013C80006D02F4A88F80270136843F004031360AC
:1013D8002B4F3B68990702D52A4B1B689847002377
:1013E80084F89631284B4FF47A721A60274BBC2048
:1013F8001B689847029E264A0023022E13709346C4
:1014080004D0032E19D0002E40F0BA8500238DF8A1
:101418006830C4F898311E200A2101221AAB03F063
:10142800C9FE50B19DF86830482B06D1194B1A4AAD
:101438001A601A4A5A60022336E04FF0000C0C205A
:10144800614601221AAB8DF868C0CDF808C003F0D8
:10145800B1FE68B19DF86830DDF808C0482B40F04F
:1014680009860C4B0E4A1A600E4A5A6003231BE089
:10147800844600F0FFBD00BFA82F0020780100209F
:101488008C1A0020D82A0020E011002070270020A4
:10149800A42F0020AC060020996F0008016F0008F7
:1014A80003D3000811D2000888F803303B6843F0E2
:1014B80008033B6095F855310BB189F8003095F871
:1014C80056310BB1C04A137095F857310BB18BF8F0
:1014D80000303B681A0740F15985BDF90C10DFED63
:1014E800BB6A642291FBF2F302FB131212B207EEFD
:1014F800902AB8EEE77A07EE903AF8EEE77AE7EE48
:10150800267AB2EE047A67EE877AC4ED677AB04A33
:10151800137843F002031370AE4B4FF480421A85E0
:101528004FF400429A610A26AA4FBB8A9BB283F401
:101538008043BB82BB8A9BB283F40043BB821920E1
:101548000FF07AFE01200FF091FE19200FF074FEC3
:10155800013E00200FF08AFE16F0FF06E4D14FF49A
:1015680000434FF480489C4EBB61C7F8188033682D
:101578001B0709D5994BA7F828801B689847984BF3
:10158800C7F8188001221A70964B9FED978A1F683A
:10159800DFED968A3B7B00EE103AB8EEC00A4FF0BA
:1015A800000820EE080A09F05FFF914B83ED000A5E
:1015B800904B1B8807EE903AF8EEE77AB7EE007A80
:1015C800C7EE277A8C4BB0EE680AC3ED007A8B4BD6
:1015D800D3ED047A8A4B67EE887AC3ED007A3B78BC
:1015E800884F07EE903AF8EEE77A874BC7EE277AEE
:1015F800C3ED007A77EE677A844BC3ED007A844BAB
:1016080083ED027AC3ED008AC3ED018A814B83ED35
:10161800027AC3ED008AC3ED018A09F025FFB0EE16
:10162800408AB0EE680A09F0BFFE20EE006A68EE54
:10163800086A66EE007A784BE6EE887A3846FF212B
:1016480020EE087AC3ED007A67EE007A1B22F0EEEE
:10165800675AD7EE085AE7EE087A28EE468AC3EDAD
:10166800015AA6EE808AC3ED027A83ED038A6B4B9A
:1016780083F8008014F0D1F83268694B87F800804D
:10168800012112F0020F19701FBF79700321197020
:10169800022118BFB9703846570741BF19784E1C48
:1016A8001E70032648BF465412F00A0F0CD01A7851
:1016B80004218154511CC9B205264654D11C02325A
:1016C800D2B2197006218154DAF800108E0641BF93
:1016D8001A78561C1E70072648BF86540A0608D575
:1016E8001A7809268654961C0132D2B21E700A2630
:1016F80086546E79082E01D00E2E04D11A78571C04
:101708001F700B2787541A7811F4803F4FF00C0E86
:1017180000F802E002F101071CBFDFF804E1023221
:10172800FFB21F701FBF8EF80020364A4FF00E0E12
:1017380002F807E04A0741BF1A78571C1F701027A4
:1017480048BF87541A78571CFFB24FF0120E11F495
:10175800806F1F7000F802E00ED095F814E2BEF119
:10176800000F09D0DFF8B8E002328EF80020254AD1
:101778004FF0130E02F807E08F0541BF1A78571C87
:101788001F70152748BF8754182E0DD11A781627B1
:101798008754571CFFB24FF0170E00F807E0D71C0C
:1017A8000232D2B21F7086540E0348BF1A781D4FFA
:1017B80041BF561C1E7019268654CA0542BF1A78A6
:1017C800511C197030E000BFA82F00208988883C80
:1017D800782F0020000800488C1A0020AC06002052
:1017E800C40600206828002035FA8E3C000000005E
:1017F80064280020040000201C28002070270020F6
:1018080020280020811100207C2800206C2800203E
:10181800802800207028002054280020DA27002083
:1018280080110020B811002044BF1A2181541A7871
:10183800511C19701423835400219822B94813F0BD
:10184800ECFF0EF016FBB84BB849B9481960B94B14
:10185800B5F84E210160B8491A800023B74AD7F875
:1018680000E00B70B5F89611138093701FFA81F998
:101878000EF18502DFF82883B148D8F80060DFF858
:1018880024C320F8139006F596764CF823600133AC
:10189800122BEFD1AB4ED6F800C01CF4805F08BF06
:1018A800B5F89C91A0F806900EF1D50E1378F3B90F
:1018B80092F80290D378994519D2B9F1000F08D05F
:1018C80009F1FF3909EB890909EB890909F5617300
:1018D80006E0013303EB830303EB830303F5617332
:1018E80092F8019009F104099BB220F819300432EA
:1018F8007245DBD11CF0080F00F0C18095F89031DB
:10190800062B00F2B680DFE803F004070E35506FAF
:101918006F0045F2F05201E042F6F8228A4B1A8035
:101928000EF055FBA4E0884B42F6F8221A80090114
:101938000A2391FBF3F10023A1F5B061834A42F831
:1019480023100133122BF9D1814A82491160824A4E
:101958004020137007F016FC002800F08A8001234D
:101968004FF0070A90F900007C4A8DE808044021EE
:101978007B4B78E0744B42F6F8221A80744B794A14
:101988001A60754B102240201A7007F0FBFB0028E4
:101998006FD001234FF0000990F90000724A8DE8DA
:1019A800080240214FF4E1335DE0674B42F6F8222C
:1019B8001A80674B6D4A1A60674B082240201A70DC
:1019C80007F0E0FB002854D001234FF0000C90F9F9
:1019D8000000674A8DE8081040214FF4E13307F012
:1019E800F5F9C4F8A00140E0574ADFF8BC91DFF8E8
:1019F800BCC1DFF8BCE15F4D5F4842F6F8211180B9
:101A080055490C22062B0A700FD0002389F80030A4
:101A18008CF800308EF800301B232B70574B027067
:101A280005221A704FF4E1350CE0002189F8001006
:101A38008CF800108EF80010027021214F4A29708E
:101A48004F4D1370424B4F4A1A60402007F09AFBE3
:101A580078B101234FF0000E4B4A90F90000402165
:101A68008DE808402B4607F0B1F9003018BF012077
:101A780028B9082009F020FD354B444A1A6033681C
:101A8800354A13F4804F1FBF122111703049404866
:101A980018BF086042F20101194003F0010003F485
:101AA800005581B1284944F6206EA1F800E025B11F
:101AB800082111702649374D0D6020B10C21117095
:101AC800234935480860117804395170190640F1E6
:101AD800AC800025DFF8DCA0DFF8DC902F48DFF8C9
:101AE800DCB0C4F8A491294615228AF80150CAF836
:101AF8000450CAF8085013F090FEA9F105032846CF
:101B0800CBF8003005F00EFED8F80030CAF80C30DB
:101B1800022007F037FB002852D1802009F0CCFCC6
:101B28007CE000BFE0290020500F0020F8130020BF
:101B38001C2F0020540F00208B0E00204C2F00205B
:101B4800202F0020741A002056080020482E00205C
:101B5800F4000020ED2501087C2A00200127010857
:101B6800A086010081A200085526010869A2000884
:101B7800B5A30008721E0020F31D0020731E00206C
:101B880090D0030085A1000895A2000851260108FD
:101B980021260108412601083126010820030020DA
:101BA80048120020D40E0020F41D0020711E0020D1
:101BB800701E002004080020621400202408002061
:101BC80045799AF80130C3490C2202FB0312527876
:101BD800AA4204D00133DBB2042BF4D900238AF8DB
:101BE8000130DBF800309AF801201B7890F90000EA
:101BF800002B4FF00C0303FB021314BF0325012530
:101C080000225B7800950192022107F0DFF8B24BC1
:101C18001860002881D0012005F084FD3868AF4B9A
:101C280000F5CB721A6005F02BFEAD4AAD4B136080
:101C3800AD4AAE4F8033136033680025DA033D7038
:101C480040F1A980DFF80CB3DFF80C9340F22A3A90
:101C58004FF001080DF020FB29465246584687F8F8
:101C6800008013F0DAFDD9F81430A14F4FF09040FE
:101C780043F40033C9F81430036A23F07063036235
:101C8800036A43F080730362402302220C930CA979
:101C980003238DF8342002928DF835308DF83650B4
:101CA8008DF8378008F034FFD9F81830029A43F4D9
:101CB8000033C9F818303B8823F440731B041B0C0D
:101CC8003B801D23FB620EA93A8560233D8638467A
:101CD800C7F814800E93ADF83E501095ADF84450F7
:101CE800ADF84650ADF84850ADF84A50ADF83C80D4
:101CF80008F062FDBB6943F00803BB617B6C43F4E9
:101D080000437B64D9F8143043EA0803C9F8143057
:101D1800A9F57D69484608F0C2FC1AA808F094FCA9
:101D2800744B1A9310231C9380231F934FF48073D2
:101D38001AA9209348464FF400532393CDF86CB06A
:101D4800ADF874A01E9521952295249508F089FC7C
:101D5800FB6843F40073FB60D9F8003043F00203DA
:101D6800C9F800300BA80D238DF82C308DF82D8084
:101D78008DF82E508DF82F800FF060FF29465E4BAE
:101D88001A685E4B43F8212001312029F7D103F06E
:101D98001DF803F01BF833685B0553D5584BD4F88E
:101DA800E8741F60042007F0EDF90421C4F8EC047E
:101DB80007F0C2F9534B84F8F00408201F6007F0BD
:101DC800E1F9514B514D1860082107F0B5F9002190
:101DD80084F8F1042C22284613F01FFD8E236B7023
:101DE8004FF07C09E0234FF07D08EB7085F80090F8
:101DF80085F82B80464D2C220021284613F00DFD36
:101E08008A236B701020A023EB7085F8009085F86A
:101E18002B80C4F8F47407F0B5F91021C4F8F8045D
:101E280007F08AF984F8FC042020C4F8007507F04C
:101E3800A9F92021C4F8040507F07EF984F80805FB
:101E480010F0CCF83368334A13F4002318BF012389
:101E580013700FF0D5F9304B1860304B5A79052ABA
:101E6800194602BF2E4B4FF4C8721A802D4B4FF4FF
:101E78007A721A802C4BC8221A802C4A137843F0A5
:101E8800080313702A4A137823F002031370326888
:101E980040F6020313406BB1264B274A1A60274BC2
:101EA80003221A70264B01221A70264A0023138037
:101EB800254A13808B683360244B01221A70244A08
:101EC800137863F07F0313702FB0BDEC068BBDE869
:101ED800F08F00BFD8710108741D0020A40F0020E6
:101EE800B01D002094140020AC1D0020D90D002046
:101EF8000044014034440140A0710108DA0D00207B
:101F0800801A0020D81A0020241B0020A81A0020BC
:101F1800DD1A00206C2C00202808002070120020F8
:101F2800EE270020A22F00209C2F0020901A0020CE
:101F3800A62F0020781A0020EA130020DC1A0020BF
:101F4800FC000020481000204A100020D80D002076
:101F5800782F00203503002000100240494B42F240
:101F680010721A805A80484A5A60484A9A60484A09
:101F7800DA60484A1A61484A5A610327FFF721BACA
:101F8800012E7FF697AA1E46FFF735BA0023C4F83C
:101F98009C31FFF7BCBA1BB208EE103AB5F95A31BA
:101FA800DFED3E7A3E4A09EE103AB5F95C31B8EEFB
:101FB800C88A08EE903A28EE278AB8EEC99AF8EE51
:101FC800E88A0021B0EE480A29EE279A68EEA78A27
:101FD800117009F049FAF0EE40AAB0EE480A09F08B
:101FE800E3F9B0EE408AB0EE490A09F03DFAF0EEA6
:101FF800409AB0EE490A09F0D7F9B0EE40AAB0EE1F
:10200800680A09F031FAB0EE409AB0EE680A09F0B1
:10201800CBF960EE2A6A68EE097AF0EE665AE7EEC6
:102028008A5A204B29EE2A6A28EE007AC3ED035A11
:10203800F0EE465A29EEC00AE7EE4A5AE6EE8A7AE8
:10204800A6EE4A7A29EE299A83ED010A28EE698AD2
:1020580029EEAA0A83ED009A83ED02AAC3ED045A79
:1020680083ED058A83ED067AC3ED077A83ED080AC6
:10207800FEF7DBBF012E7FF61DAA00268BF800C0F5
:10208800FFF7C4B9D0060020FBD10008DDD2000854
:10209800F1D10008CDD2000851CF000835FA8E3CA6
:1020A80068000020B81E00202DE9F04FA249A34C7B
:1020B8000A6802F59C432DED028B20332360A04B68
:1020C80087B01E780091C6B19E4909688A4240F2DD
:1020D8000581013E1E7001E1D9F800309A48072DAC
:1020E80098BF595D994B88BF29461B689847032DAF
:1020F8000CD904EB45050136A880934BDFF87092A4
:102108001A78F5B2AA421946E6D820E0D9F8002094
:1021180005F10E0302EB83039988DA880028E8D0DA
:102128004FF47A73401A5843531A90FBF3F040F671
:10213800C90300F57A70984205DC40F2EE23984214
:10214800B8BF184601E040F6CA0080B2D1E7804B1C
:102158001B6842F2010803EA08087E4BB8FA88F8BF
:102168004FEA58181B68B8F1000F06D194F82920D7
:1021780084F82820784A5078107094F828701FB195
:10218800754A177887F0010794F82BB091F800A0EA
:102198000F220326BBFBF6F606EB460684F82A2038
:1021A800C6EB0B06D9F80020DFF8CC91F6B2002573
:1021B800554559DA4FEA450C1FB1684931F8150001
:1021C80000E03846918ADFF8B4E1814202D8D18A2A
:1021D80081421ED25EF825005849834203D26049E5
:1021E80031F80C0019E0E8B202920193039110F063
:1021F800ABFA032D019B029A0FDC03994FF0010CF7
:1022080091F82AE00CFA05FC2EEA0C0E81F82AE077
:1022180003E003F596714EF82510B8F1000F1CD1B4
:1022280094F8BC1029F8160031B9BBF1020F14D983
:102238004249012081F8BC00B9F80210B9F8000041
:102248000844B9F804100844464980B221F815003A
:1022580000B2032190FBF1F080B2414909F106096F
:1022680021F815000135A3E794F82A2039493E4B97
:10227800A2F10F0EDEF1000242EB0E0284F8D62026
:102288006AB13A4A1268570109D40A68D9689A604B
:10229800521AC82A1DD9012283F8212019E02E4A92
:1022A8000120507010700A689968DA605B68521AE9
:1022B8009A4282BF2C4B002283F8212000255545E5
:1022C80007DAE8B210F040FA254B23F8150001357B
:1022D800F5E794F82B30013384F82B301C4B1A683F
:1022E80012F4805F984605D0204B1B68DE0701D4A6
:1022F8000FF048FC009B19681D4B1868837A002B67
:102308003ED0013B164D027B35F813301AB1C3F5A8
:102318003B6308339BB21BB2A3F57A73B3F57A7F9C
:10232800A8BF4FF47A7323EAE37307EE903A9FED60
:10233800117AF8EEE77A5CE0842F0020600E002026
:10234800482F0020442F00207C2A0020F400002081
:10235800741A00204812002001000020640E00209A
:10236800202F00201E0F00204C2F00207C11002061
:102378001C2F002000007A448C0E0020D40E002070
:10238800D8F80020150440D5D4F8D820934E8A1ADE
:10239800002A3ADB01F59C422032C6F8D820904A40
:1023A800C07A55798F4A32F8152096F8DC500135F5
:1023B80092B292FBF0F205F00F0086F8DC00304490
:1023C80080F8DD201A468848185C01330244102B37
:1023D80092B2F8D112B292FBF3F31BB2642BA8BFEE
:1023E800642323EAE37307EE903A9FED807AF8EED0
:1023F800E77AC7EE877A7E4A9FED7E7A67EE877A1C
:10240800FCEEE77A17EE903A1380D8F800307A4F4E
:1024180013F4807F00F00981784BDFF8E49199424A
:1024280005D999F8022012B9012289F8022099F8F1
:102438000220002A00F0F980714A3E7892F8215073
:102448006A1E554255416F4A1168002DC1F38063D9
:10245800C6F380060093924614BF4FF0000B4FF06E
:10246800030B99F82020052A00F2D980DFE802F052
:10247800034D527584A1002E3AD0D4F8F000B4F878
:10248800F4100EF079FE012809D15F495F4A096806
:102498001268C988642000FB0122C9F81020009B3B
:1024A8006BB1594A126812794AB110F07DF80322CB
:1024B80089F820204FF47A72C9F81C20D1E7002D42
:1024C80040F0AD80514AD9F8101010684C4A884243
:1024D8000AD9019210F068F8019A032182F82010B5
:1024E80040F6B831D161BCE7012182F82010B8E785
:1024F800009B4FF4806013B108F0CEFF01E008F0B4
:10250800BBFF0022C9F8102089E0002D46D110F049
:102518004BF8A6E725B1052289F82020012000E024
:10252800284666B1D4F8F020D189394A1180518003
:102538009180354909684988D1804FF0020B334AA8
:102548001168D9F81420914201D8002E64D147F2BD
:102558003052C9F81C20032221E03A7842F00202E6
:102568003A700FF00FFB294AD9F81C1012680A4478
:10257800C9F81820042212E0244A9DB11168D9F83C
:10258800182091424BD9234A92781AB9DAF80020D8
:10259800D30744D43A7822F002023A70052289F827
:1025A80020205EE71268D9F81C100A44C9F81820E0
:1025B80035E01549154A09681268C988642000FB86
:1025C8000122C9F810204FF48060002289F82020E9
:1025D80089F8032008F050FF43E700BF600E002091
:1025E800DC1E0020EC1E00203D0F00200000C84229
:1025F800DC11002000C07F44A62F0020404B4C0077
:102608004C2F00207C110020442E0020481200206E
:10261800202F00200100002000287FF422AFBBF10A
:10262800000F02D058460EF03BFE8D4D05F5C470E4
:10263800B5F84E110EF0A0FD834668B90FF0A6FF5D
:10264800884BC3F800B0C3F804B0C3F808B0864B91
:1026580000221A605A609A603B785E0736D5D8F82F
:102668000030D80632D5814B1B78D9062ED4804B42
:102678009B7893B195F8E031BBF1000F15D17BB190
:102688007C4B1A68D4F8F8309B1A002B08DA0FF044
:1026980079FA794B83F8FCB018E0BBF1000F0DD143
:1026A80010200EF0FDFD01230EE03BB1714A1268C7
:1026B8004FF47A7101FB0323C4F8F83094F8FC3026
:1026C80023B10EF0D9FD002384F8FC30002295F8E0
:1026D800DEA195F8DF11B5F898E1B5F89AC113466F
:1026E8006648009030F912609B087645C4BF63F0D5
:1026F8007F03DBB201326645B8BF43F04003042ACA
:10270800EED194F8FD205C489A4205D190F8FE205D
:10271800F92A04D8013200E0002280F8FE2084F86B
:10272800FD30534B564E9A789946E2B93368DA072A
:1027380008D5BBF1000F16D13B78DB0713D50FF096
:102748008DF810E03B7858070DD54B4B93F828309F
:102758004BB14C4BDB7833B911B10FF013FA02E0EF
:10276800BBF1000FF9D094F8FE30434ADFF830B1DE
:10277800142B40F0B08099F802301AF1000A18BF03
:102788004FF0010A6BB392F8FD305F2B11D13B7803
:1027980003F0040303F0FF0113B10FF0F3F908E0AD
:1027A8000B20029101920EF07BFD019A029982F8AA
:1027B800FE10BAF1000F14D094F8FD307D2B10D123
:1027C8003B7803F0040303F0FF0213B10FF0DAF9CA
:1027D80007E00B2001920EF063FD274B019A83F866
:1027E800FE203B7803F0040303F0FF01002B72D1B5
:1027F80094F8FD30204A572B16D1234B4FF47A72A8
:102808001A80D8F80030190601D505F09BF81F4B3F
:102818001B685A0742BF1E4A0A21118013F0080399
:1028280059D11C4A138056E0D8F80000400739D522
:102838005A2B37D1184B187820B11970174B012231
:102848001A7048E092F8FF3083F0010382F8FF30F5
:102858000BB10C2000E00D200EF022FD3BE000BF84
:102868007012002014270020B81F0020901A0020A2
:102878000100002048120020600E0020202F0020B8
:102888007C1100204C2F0020A22F00208C1A002041
:102898009C2F002060120020192800201A280020F0
:1028A800B81100205D2B00F036855B2B00F03585D4
:1028B8005E2B00F03485562B01D109F099F899F870
:1028C8000230002B00F0FB8494F8FD306F2B40F0B1
:1028D800F0840EF0C3FFD8F80030580732D594F8CA
:1028E800FF30A3B13B78590711D5009BB3F90620F7
:1028F800B5F898319A420ADD336813F0010301BF35
:10290800AE4A32211180AE4A08BF82F8FF303368E0
:10291800DA030AD5AB4B1A782AB9AB4A127812B93E
:10292800A64A3221118001220BE0A74A13784BB145
:102938003B7803F0040303F0FF011BB9A34B1170AC
:1029480001221A70DBF800A0002333600AF187091E
:102958000AF1D70B99F8002099F8013019F8010C01
:102968009A420BD2494606F079FC38B119F8022C84
:10297800012303FA02F233681343336009F10409AF
:10298800D945E7D1924B1B7853B1924B924E1A68B6
:10299800DFF85CA212F0020F994640F0418338E359
:1029A8000AF1D6060AF58F793278737816F8010C91
:1029B8009A4225D2314606F051FC08B3B37896F80E
:1029C80004C0864A96F803A07D480C21013B01FB10
:1029D8000C4103EB43031344D1F804219A420FD06E
:1029E800C1F80431002390F83021C1F808310123DF
:1029F80003FA0CF322EA030381F800A180F83031CE
:102A080006364E45D0D1764B1E68764B1B6802932E
:102A180094F828300393744B019300230093019B8F
:102A28001B68002B00F0EA8293F800A0BAF1000FAF
:102A380000F0E482019A029952688A1A002A0CDB93
:102A480001F5FA7201994A60009901228A4094F8C6
:102A5800301121EA020284F83021039A002A00F09A
:102A6800CD82019A597812F8042C0432D2B2002986
:102A780040F083825D4931F91210B5F8962102F1D0
:102A8800C800814202DD93F802B015E0C83A9142CD
:102A980003DA9978C1F1000B0EE0009A0123934004
:102AA80094F8302122EA030384F83031029B019A1A
:102AB80003F5FA735360A1E294F83031009A134198
:102AC800DB0700F19B82BBF1000FCCBF0220012085
:102AD8000EF016FC0AF1FF33DFF8E490132B00F236
:102AE8008582DFE813F01400250037004B006400EE
:102AF8008D00F0005301BA01E801180283024B006F
:102B08005A008D00F0005301C20025018A0196F891
:102B18000090D944B9F1FA0FA8BF4FF0FA0929EA91
:102B2800E979304686F8009006F07EFB01200FE038
:102B380096F80190D944B9F1640FA8BF4FF0640921
:102B480029EAE979304686F8019006F06DFB022003
:102B58004946DDE196F803A0DA44BAF1640FA8BF4C
:102B68004FF0640A2AEAEA7A86F803A03046D9F8D0
:102B7800341106F00FFB03205146C9E1717959441D
:102B88006429A8BF642121EAE17171710D200EF05A
:102B980023FBBAF10D0F00F02982317959446429D9
:102BA800A8BF642121EAE17131710E20B0E1B17949
:102BB800594481F30801B1710520A9E100280020DA
:102BC800600E002018280020192800201A2800204C
:102BD800A72F00207C1100208C1A0020D475010832
:102BE800E411002048120020640F0020202F00204C
:102BF800541B002000007A440000C8420000000076
:102C0800D9F838311A78022A20D107EE90BAB8EEEE
:102C1800E70A5FED077A93ED097A80EE270A30EE2E
:102C2800070AB5EEC00AF1EE10FA07D4B4EE670A47
:102C3800F1EE10FAC8BFB0EE670A01E01FED110A05
:102C480083ED090A0F200EF0B1FA0AE09978594489
:102C5800C829A8BFC82121EAE17199700F200EF098
:102C6800BBFABAF10F0F00F0C181D9F838311A78E0
:102C7800022A1ED107EE90BAB8EEE78A5FED227AF3
:102C880093ED080A88EE278A38EE000AB5EEC00AE6
:102C9800F1EE10FA07D4B4EE670AF1EE10FAC8BFE5
:102CA800B0EE670A01E01FED2B0A83ED080A122037
:102CB80056E159785944C829A8BFC82121EAE171C9
:102CC8005970122024E1D9F838311A78022A20D113
:102CD80007EE90BAB8EEE70A5FED397A93ED0C7A11
:102CE80080EE270A30EE070AB5EEC00AF1EE10FAB8
:102CF80007D4B4EE670AF1EE10FAC8BFB0EE670A5F
:102D080001E01FED420A83ED0C0A10200EF04EFA86
:102D18000AE0197B5944C829A8BFC82121EAE171F2
:102D2800197310200EF058FABAF1100F00F05E81F6
:102D3800D9F838311A78022A1ED107EE90BAB8EEBF
:102D4800E78A5FED537A93ED0B0A88EE278A38EE0F
:102D5800000AB5EEC00AF1EE10FA07D4B4EE670A1D
:102D6800F1EE10FAC8BFB0EE670A01E01FED5D0A88
:102D780083ED0B0A1320F3E0D97A5944C829A8BF78
:102D8800C82121EAE171D9721320C1E0D9F838319C
:102D98001A78022A22D107EE90BA1FED6A0AF8EED5
:102DA800E77A87EE800AD3ED0F7A30EE270AB5EE80
:102DB800C00AF1EE10FA09D45FED717AB4EE670A31
:102DC800F1EE10FAC8BFB0EE670A01E01FED750A10
:102DD80083ED0F0A11200EF0E9F90AE0997D5944B4
:102DE800C829A8BFC82121EAE171997511200EF000
:102DF800F3F9BAF1110F00F0F980D9F838311A78DF
:102E0800022A20D107EE90BA1FED860AB8EEE78AAB
:102E180088EE008A93ED0E0A38EE000AB5EEC00A75
:102E2800F1EE10FA09D45FED8C7AB4EE670AF1EE90
:102E380010FAC8BFB0EE670A01E01FED900A83EDF3
:102E48000E0A14208CE0597D5944C829A8BFC8210E
:102E580021EAE171597514205AE0D9F838311A7805
:102E6800022A1ED107EE90BAB8EEE78A5FED9E7A85
:102E780093ED0A0A88EE278A38EE000AB5EEC00AF2
:102E8800F1EE10FA07D4B4EE670AF1EE10FAC8BFF3
:102E9800B0EE670A01E01FEDA70A83ED0A0A0920D0
:102EA8005EE0D9785944C829A8BFC82121EAE17150
:102EB800D97009202CE0D9F838311A78022A1ED1A5
:102EC80007EE90BAB8EEE78A5FEDB57A93ED0D0A92
:102ED80088EE278A38EE000AB5EEC00AF1EE10FA3D
:102EE80007D4B4EE670AF1EE10FAC8BFB0EE670A6D
:102EF80001E01FEDBE0A83ED0D0A0A2030E0597B80
:102F08005944C829A8BFC82121EAE17159730A2088
:102F18000EF062F96AE0D9F838311A78022A22D11B
:102F280007EE90BA1FEDCD0AB8EEE78A88EE008A60
:102F380093ED100A38EE000AB5EEC00AF1EE10FA69
:102F480009D45FEDD37AB4EE670AF1EE10FAC8BF80
:102F5800B0EE670A01E01FEDD70A83ED100A0B20D7
:102F68000EF024F942E0D97D5944C829A8BFC821E8
:102F780021EAE171D9750B20CAE7012936D1987881
:102F8800B84B33F91230B3F5617F05DB40F63302F5
:102F98009342A8BF134601E04FF46173BAF10C0FD6
:102FA80024D14FF4966292FBF0F0AF4AA3F5617317
:102FB80093FBF0F35FFA83F913784B4516D0B9F118
:102FC800040F34BF4B4602231370A84A0AFB03536D
:102FD80003F2D273136008F03BFB504649460EF0EB
:102FE800FBF809F10100C0B20EF08AF9009A01233A
:102FF800934094F83021134384F83031009B013317
:103008000093019B0C330193009B042B7FF407ADC5
:10301800BBE4D8F80030D80510D5954BDB786BB1F8
:10302800336899070AD5BAF8003013F0010B0AD1B2
:103038000FF0ACFA012008F02FFA04E0012008F0A4
:103048001BFA012300E00023D9F8002052070DD510
:1030580063B1012008F010FABAF800309B0708D4D1
:103068000FF094FA022008F017FA02E0022008F0A4
:1030780003FABAF800307F4A13F0030F4FF4804187
:103088000CBF91611185326812F00A0F27D0D9F868
:103098000020D00609D559070AD4042008F0FCF905
:1030A800754B1B88A4F83C3102E0042008F0E4F9D1
:1030B800D9F800309A0607D5BAF800305B0606D46E
:1030C800402008F0E9F902E0402008F0D5F9D9F8E5
:1030D8000030580642BF684B1B88A4F83E3133685D
:1030E800990609D4D9F800301A0540F191804FF4B7
:1030F800807008F0D1F98FE0604B1B789B0753D59F
:103108005F4B1B78042B4FD9D9F8003013F4007BA0
:103118000FD0BAF80030DE063AD4102008F0BCF917
:10312800202008F0A9F95748011D04F05FFB02238D
:103138002AE0BAF8006006F01006B6B22EB11020E8
:1031480008F09AF9012684F840B1D9F800305805FA
:1031580012D5D4F844314C495A89B1F90030002BC2
:10316800B8BF5B42934207DAB1F90230002BB8BF0F
:103178005B429342C0F2FA80BAF80030990608D54B
:10318800202008F079F9002384F84031012600E076
:10319800002694F84831BBB90E200EF081F83B4B5D
:1031A800012283F848210FE0BAF8003003F0300319
:1031B800002B97D0102008F05FF9202008F05CF968
:1031C800002384F8403101E0002E8BD0304B0020E2
:1031D80003F1280603F150042E4A002122F81010AA
:1031E8002D4A596022F810100432716022F810102C
:1031F80000221A609A603260B26022606160A26048
:1032080014331436143400287FF46CAF0120E3E73C
:103218004FF4807008F030F96B79082B01D00E2B31
:1032280002D1402008F028F9D8F800305A0540F1BA
:10323800B38095F814321BB93B7813F0040F03E000
:10324800D9F8003013F4002F2AD0144B00221A703A
:103258003C200CF005FF002800F09E800DF062FC79
:10326800F6E700BF202F0020B82A0020E411002034
:103278004C2F00200008004860120020901A0020FF
:10328800961A0020EC11002068120020600E002021
:10329800AC0F00209E2F002024100020812A00203F
:1032A8000EF09CFE07B0BDEC028BBDE8F04F0CF0B1
:1032B800E0BDBAF1000F02D07E2B3FF40AAB94F8C0
:1032C800FD30972B05D1374B4FF4C8721A80FFF7A2
:1032D80002BBA72B06D1344A137843F004031370BA
:1032E800FFF7F9BA0022BB2B059201D1022303E0B4
:1032F800B72B04D14FF6FE73ADF816301FE0BE2B86
:1033080001D1022304E0BD2B7FF4E5AA4FF6FE733A
:10331800ADF8143013E0012002E0022000E00320A1
:103328005FFA80F909F1FF3385F8D03708F0F6F82D
:1033380008F0B2F948460DF0E3FFFFF7CCBADBF826
:103348000030BDF81410B3F864200A44A3F86420D0
:10335800BDF81610B3F866200A44A3F8662008F0F2
:1033680047FB002384F8FE30FFF7B5BABAF80030FF
:103378009B063FF50EAF202008F08EF80B480C4B4B
:10338800011D1A685B684360026004F02FFA094B5C
:10339800012683F84061FCE607B0BDEC028BBDE86E
:1033A800F08F00BFEE270020901A0020F4110020B3
:1033B800981A0020600E00202DE9F04FC14BB3F998
:1033C8000610C14B2DED028B1F687A898FB0914290
:1033D80001930EDBB1F5FA6FFC79BDBF8B1A63431D
:1033E800A2F5FA64C4F16404BCBF93FBF4F464343A
:1033F80000E06424B54BB64AB3F896B193F95E3150
:10340800126802929BB2154603930022AD4B33F922
:1034180012E0CBEB0E0303F2F31640F2E6308642DD
:103428004FEA420C03D8002BB8BF5B4201E04FF4CF
:10343800FA73022A2ED0029E96F81D611EB1B3427D
:10344800CCBF9B1B0023A34E6FF0630A642093FB41
:10345800F0F836F818900AFB083A08F1010836F92E
:1034680018600FFA89F8C8EB060606FB0AF696FB01
:10347800F0F699484E4420F80C60BE18642036795E
:103488007343964E93FBF6F364339BB2634393FB0B
:10349800F0F02DE0029890F81E611EB1B342CCBF47
:1034A8009B1B0023DFF860926FF06308642093FB96
:1034B800F0F008FB003A39F910600130002B39F9B7
:1034C8001000A0EB060000FB0AFABDF80C009AFBFE
:1034D800F8FAC6EB0A0A1AFB00FA7F48A0F804A01B
:1034E800B879B8BF5B4243437C4893FBF0F0643043
:1034F8006B787B4E4FF06408434393FBF8F3B35467
:10350800784EEB7A434393FBF8F3B3546B7D724EDA
:103518005843754B90FBF8F0022A9854734B0ED120
:10352800DE4583F802800DDB684CB4F8982191429F
:1035380014DBB1F5FA6FA8BF4FF4FA610FE0DE456E
:103548009C5404DA36F80C305B4226F80C30013211
:10355800032A05F101057FF459AFE5E71146DFF8C5
:10356800BCE15D4D891A4FF47A736FF063075943D4
:10357800C2F5FA626423B1FBF2F191FBF3F23EF873
:10358800120007FB0211013207B23EF91220D21BCA
:10359800514391FBF3F30344F380554B1B885806C2
:1035A80035D5544B544A1B881288DFED547A9B1A40
:1035B8001BB208EE103AB8EEC88A28EE278AB0EE99
:1035C800480A07F051FFF0EE408AB0EE480A07F0CB
:1035D800EBFEB5F9023006EE903AB5F90030F8EE98
:1035E800E66A07EE903A20EE667AF8EEE77AA7EEFA
:1035F800A87A67EE807ABDEEC77AE6EEA87A17EE6B
:10360800103AFDEEE77A2B8017EE903A6B803C4D2E
:103618002B68990740F1A1803A4B3B4F1A687B69A8
:1036280045F20721D31A8B4240F397807A6107F05D
:103638005DFB364BDFF8E8901A78032A9846B9F80C
:10364800003022D10A2B2AD90023282088F80030FC
:103658000DF0F2FD07F04AFB2D4B188807F030FB00
:103668002C4B1A68D37890FBF3F0013008282A4BCA
:10367800A8BF08201870537980B213FB00F33B836E
:10368800137913FB00F0788309E00A2B07D803238A
:10369800214A88F80030002313703B837B8398F815
:1036A80000301A4A012B3DD002D3022B4CD054E0F3
:1036B8003A8BB9F800309A424FDD012388F8003080
:1036C80040E000BF202F0020E411002070120020ED
:1036D800B8110020661D0020681200200CFEFFFFB4
:1036E800CC1F00203E100020E01F002004270020EF
:1036F800541B0020601200209E0F002035FA8E3CDB
:10370800741A0020842F002030100020DC1A0020BA
:10371800F41E0020781A0020FC0000204E1D002016
:103728007C1A0020B9F800107B8B8B4202DD022343
:1037380013700FE0A04B1B8B0133994202DD00236D
:1037480013700AE0082006E07B8BB9F800200133EB
:103758009A42B2DC07200DF0A3FD2D682A0573D527
:10376800964B954F1B68FA69C2EB030845F207228E
:10377800904569DDFB61B6F90630B4F84E11904EFC
:10378800A3F57A7B8F4BD3F8009099F80A30012B78
:1037980003D042D3022B20D041E08B4B396A5A7BAD
:1037A8008A4B33F81220082092B291FBF0F3C91A21
:1037B8008B18BA843B6240F6E44293FBF0F39BB269
:1037C8005343B9F80820C2EB13334FF47A725343CA
:1037D800B9F9062093FBF2F320E07D4BB9F808A075
:1037E8001B78C6F800A05B0719D57A480DF0C4FC11
:1037F80020B915F0100F18BF4FF0000BB9F90620CB
:103808000BFB0BF1322391FBF3F35B445A434FF468
:103818007A7392FBF3F3534400E000233360D7E953
:103828000A0133686C4A03FB08F84FF47A7398FB73
:10383800F3F810EB080041EBE8710023C7E90A012F
:103848000FF022FA654B1860654E3368DF0427D500
:10385800280622D5634B1B7899071ED5624B18782A
:1038680004281AD90022614BD7180521951C4FF05E
:103878000A0E122AD154E9B287F801E004D0B0EB5D
:10388800510F2A46EFD800E014215A18322002F8C6
:10389800010CFF225A540F2000E00A200DF000FD11
:1038A800534D2A68002A55D0524B534F186839682F
:1038B800814298464ED8514BDFF84C9118785168A0
:1038C80008BB01201870B9F80030CB5C5BB31378E3
:1038D800013B00FA03F2D4F8FC371A4201D10DF08B
:1038E800C5FC474B01221A700EF084FFB9F800306E
:1038F800CBB92B681B78053B012B14D80DF080FC45
:10390800404B18600FE04FF0000A83F800A0B9F8A8
:103918000030CB5C3BB150460DF0A8FC384B83F827
:1039280000A00EF067FF2A68B9F8003052683648E0
:10393800D25CFE2A01D100230BE0FF2A02D10DF050
:103948009BFC07E0D8F800500A2111FB02523A60AC
:10395800013303801E4D2B785A0704D52B4B4FF4A7
:1039680000421A856AE03268D7075CBF43F001035A
:103978002B701C4B224A1B781E075EBF2B7823F046
:1039880001032B70224B1B6813F0040F02D021494E
:10399800098851B92049098809B1980705D41F4BEE
:1039A8001B88003318BF0123D3B3022313702B786D
:1039B80023F001032B7038E030100020842F002002
:1039C800841A0020781A0020DC1E0020EC1E00203B
:1039D800A62F0020F8130020407E0500881A00203A
:1039E8007C110020901A0020961A0020E42A00205A
:1039F800142B0020481200200C2B0020082B00203C
:103A0800702F00200C2E0020102B002000080048EA
:103A18008C1A00209C2F0020EE270020A22F0020C7
:103A28002978C90758BF022313700DF0E9FBB34B7F
:103A38001B68C01A002801DB0EF0DCFE0EF0CEFA7F
:103A4800AF4B1E789846002E00F0AA80AD4E336822
:103A5800002B00F0EC8630680DF0C5FC002800F063
:103A6800E686A84BA84C18680DF0BAFC092801D0C6
:103A78003F2850D14FF0000AD4F80090A34D574684
:103A8800B9F1000F05D0A24829684A4611F012FF83
:103A980010B9AA4607B92F469E4B10359D42EFD361
:103AA800C7B1D7F800E0DAF800C023681EF8035061
:103AB8001CF80300A8420DD15A1C954938B92D2B82
:103AC80005D8914D2A602025CD54885402E0CD5464
:103AD8002260EAE723680BB1574511D08E480DF0F4
:103AE80015F9574507D857F8100B0DF00FF90920AD
:103AF8000DF004F9F5E789480DF008F94FF00009D1
:103B080023689945A7D2824B13F809000DF0F6F8FF
:103B180009F10109F4E72368002B40F06C860428BA
:103B280040F0AE867A4805F015FD00F080BED9F861
:103B38000000DFF8F8A10DF056FC38B3DAF8000001
:103B48000DF04EFCDBF8003093F8481002460029CF
:103B580034D124286BD1012283F84820DBF80030C7
:103B6800DFF8C4A193F84820062AE0D193F8490069
:103B780001F00AFC8346002800F083803B689879AE
:103B88000DF00DF83B68002283F84820644B93F849
:103B98003530002B40F01D864C36982E00F04786B5
:103BA800604BF21892F84A100129F5D15E4FF3588C
:103BB8003A605E4ABB4613609146B8E7012904D1D2
:103BC8004D2814BF00220222C6E7022904D13C284E
:103BD80014BF00220322BFE703290CD140284FF06D
:103BE800000102D983F84810B8E758711971D971E2
:103BF80098710422B0E7042906D1997983F849001D
:103C08004A409A710522A7E70529A7D15879197959
:103C18008842987906D950409871481C18710B440D
:103C28001A729BE790420CBF0622002294E72B7879
:103C38003F49580792D4232ADAF8003014D10120DA
:103C480088F800002F480391036035480292036307
:103C580038480DF05BF831480DF058F80399029A8E
:103C68000B7843F002030B70334B1B681B789342AD
:103C780001BF324B324A1A60324B04BF324ADA6013
:103C88006CE7DAF8002092F849304C2B00F0A88451
:103C980000F28480332B00F0DE8421D8292B00F039
:103CA8006B8409D8252B00F02584272B00F0298464
:103CB800232B40F0E1854CE22D2B00F06E8407D8D1
:103CC8002B2B40F0D9850CF04DFF607100F07CBDC6
:103CD8002F2B00F02C85312B00F03E8500F0CCBD59
:103CE8003E2B00F02C8146D8372B00F0E8842DD8E5
:103CF800352B00F0818200F0BFBD00BF742F00207B
:103D0800A72F0020D42A0020A81D0020B87C010875
:103D1800781D0020687E0108DF950108E4950108F8
:103D280030100020E0290020341B0020381B002020
:103D3800A62F002014960108842A0020FC9F00204A
:103D4800EFBEADDE00ED00E00400FA05392B00F00F
:103D5800E5833C2B40F09085DFF86494D9F800A007
:103D68000CF000FF8AF80000D9F8003018780AF043
:103D780009FE00F029BD432B00F07E8406D8412BB4
:103D880040F07A854FF0000900F06ABC442B00F03F
:103D980017854A2B00F0188500F06EBDD02B00F077
:103DA800228355D8CA2B00F0D48009D8C82B00F03C
:103DB800858000F239834E2B00F01F8400F05CBD33
:103DC800CD2B00F01B8304D8CC2B00F03D8200F0F3
:103DD80053BDCE2B00F01B83CF2B40F04D850CF04C
:103DE800CBFE6FF4AF6283189BB2C62B98BFA4F8C2
:103DF80096010CF0C1FEA4F840010CF0BDFEA4F839
:103E080042010CF0B9FEA4F844010CF0B5FEA4F888
:103E1800D8010CF0A7FE84F8ED010CF0A3FE0CF01D
:103E2800A1FE84F8EE010CF09DFE84F885010CF0EB
:103E380099FE84F892010CF095FEE14BD3F80090BE
:103E48000CF09AFE00EB80004000A9F8620065E3E0
:103E5800D62B00F04C820AD8D22B19D0C0F00B8395
:103E6800D32B25D0D42B00F04E8200F005BDEF2BCC
:103E780055D005D8D82B40F0FF844FF0000AFAE05F
:103E8800F22B00F08882FA2B00F0CA8200F0F4BC12
:103E98002B78590700F198840CF064FE022884F806
:103EA800D00740F2A682C74B002283F8D027A0E2B1
:103EB8000CF062FEC44B188000F086BC92F80590A6
:103EC8004FEA5909B9F1120F03D90CF0C5F800F0FF
:103ED8007BBC4FF0000ACA4507D20CF04DFE05AB7B
:103EE80023F81A000AF1010AF5E74A4600234B4570
:103EF80007DA05A931F81300B44921F81300013392
:103F0800F5E7122A05D0B14B002123F8121001322F
:103F1800F7E7AF4B012283F8342000F055BCDFF8F7
:103F2800A092D9F800A00CF027FEAAF86600D9F8EC
:103F380000900CF021FEA9F8640000F045BC0CF0DC
:103F480011FE84F8E0010CF00DFE84F8DF0100F0AA
:103F58003BBC9B4B1A681278022A824699466FD15D
:103F6800D9F800B00CF0FEFD07EE900AF8EE677A7B
:103F7800B2EE048AC7EE887A0BEB8A0BCBED087A8F
:103F8800D9F800B00CF0EEFD07EE900A9FED917A9B
:103F9800F8EE677A0BEB8A0BC7EE877ACBED0B7AD4
:103FA800D9F800B00CF0DEFD07EE900A9FED8A7A92
:103FB800F8EE677A0BEB8A0BC7EE877A0AF1010AEB
:103FC800BAF1030FCBED0E7ACAD1BAF1070FD9F8BF
:103FD80000B01CD10CF0C6FD07EE900AF8EE677A27
:103FE800C7EE887ACBED117AD9F800B00CF0BAFD9B
:103FF80007EE900AF8EE677AC7EE887ACBED127A68
:10400800D9F800B00CF0AEFD8BF84C0012E00CF0C3
:10401800A9FDD3448BF80100D9F800B00CF0A2FD3B
:10402800D3448BF80B00D9F800B00CF09BFDD344B7
:104038008BF815000AF1010ABAF10A0FC5D1C3E3DA
:10404800D9F800B00CF08EFDD3448BF80100D9F8F4
:1040580000B00CF087FDD3448BF80B00D9F800B002
:104068000CF080FDD3440AF1010ABAF10A0F8BF86B
:104078001500E5D1A8E3DFF848919FED578AD9F8F4
:1040880000B00CF079FD07EE900AF8EE677A0BEBBA
:104098008A0BC7EE887ACBED087AD9F800B00CF015
:1040A8006BFD07EE900AF8EE677A0BEB8A0BC7EE0A
:1040B800887ACBED0B7AD9F800B00CF05DFD07EEED
:1040C800900AF8EE677A0BEB8A0BC7EE887A0AF14A
:1040D800010ABAF1030FCBED0E7ACCD1BAF1070F72
:1040E800D9F800B01CD10CF047FD07EE900AF8EEA5
:1040F800677AC7EE887ACBED117AD9F800B00CF060
:104108003BFD07EE900AF8EE677AC7EE887ACBEDAA
:10411800127AD9F800B00CF02FFD8BF84C0012E0A1
:104128000CF02AFDD3448BF80100D9F800B00CF04C
:1041380023FDD3448BF80B00D9F800B00CF01CFD1C
:10414800D3448BF815000AF1010ABAF10A0FC5D158
:104158003AE30CF007FD132883463FF6B6AEDFF8C6
:1041680060A0DAF800900CF0FDFC00231B4A0C213B
:1041780001FB0322117A81423AD10FFA8BFB09EB3A
:104188008B09137889F885300CF0ECFC89F88600E7
:104198000CF0E8FC89F887000CF0E4FC104B114A9D
:1041A8001A6089F88800104BDAF8000018600021BE
:1041B800853005F079F80D4B80F00100187003E3A5
:1041C800B8110020701200209C0F0020902E0020B3
:1041D800301000200000C84200007A4440760108F0
:1041E800940F0020B0130020980F00200300002037
:1041F80001331C2BBAD168E60CF0B4FC0B288246BC
:104208003FF663AECE4BD3F800900CF0ABFC03281E
:104218003FF65BAE062303FB0A9989F8DA000CF037
:10422800A1FC89F8D5000CF09DFC89F8D6000CF0AB
:1042380099FC89F8D7000CF095FC89F8D8000CF0A7
:1042480091FC89F8D900BFE25379092B7FF63DAE7E
:10425800019BD3F800900CF085FC019B89F80000C5
:10426800D3F800900CF07EFC89F801000CF07AFC81
:10427800019B64281B68A8BF642018710CF072FCAD
:10428800019B64281B68A8BF642058710CF06AFC65
:10429800019BFF281B68A8BFFF2098710CF062FCE7
:1042A800019B6428D3F8009028BF642089F8070090
:1042B8000CF058FC019B89F80200D3F800900CF030
:1042C80051FC019B89F80300D3F800900CF054FCD2
:1042D8003B68A9F80A005B790A2B40F27582994B72
:1042E800D3F800900CF03EFC89F808006CE2824696
:1042F8000CF042FC944B23F81A000AF1010ABAF1B7
:10430800080FF5D160E253790F2B7FF4DEAD0CF086
:1043180029FC072881463FF6D8ADDFF824A2DAF851
:1043280000B00CF029FC0E2303FB09F9CB44ABF8D1
:104338002501DAF800B00CF01FFCCB44ABF82701DC
:10434800DAF800B00CF018FCCB44ABF82901DAF825
:1043580000B00CF007FCCB448BF82B01DAF800B066
:104368000CF000FCCB448BF82C01DAF800B00CF010
:10437800F9FBCB448BF82D01DAF800B00CF0F2FB16
:10438800CB44DAF800A08BF82E010CF0FFFBD144E7
:10439800C9F82F0118E20CF0E5FB0F2881463FF61B
:1043A80094AD0CF0DFFBC9EBC909A14489F8D00032
:1043B8000CF0D8FB89F8D1000CF0D4FB89F8D200B6
:1043C8000CF0D0FB89F8D3000CF0CCFB89F8D400B2
:1043D8000CF0C8FB89F8D5000CF0C4FB89F8D600AE
:1043E8000DF0AEF9F0E12B785B0700F1ED810BF0F1
:1043F800ABFE07F093F807F04FF9E5E12B78580783
:1044080000F1E281514B4FF4C8721A80DCE12B783D
:10441800590700F1D9814E4A137843F0040328E084
:104428002B785A07E5D527E20CF09CFB484B1A7805
:1044380010B142F0020201E022F002021A700CF000
:1044480091FB444BDFF82C9118700CF09FFBC9F8D6
:1044580000000CF09BFBC9F804000CF08DFB3E4BF0
:1044680018800CF089FB3D4B3D4A1880137843F0C7
:1044780002031370A8E10CF075FB02900CF086FBA8
:1044880083460CF083FB82460CF080FB81460CF0DF
:1044980073FB0CF071FB0CF065FB029BA3B9314B6D
:1044A8001020C3F800B0C3F804A006F0E5FF284ABE
:1044B800137843F001031370B9F1000F00F0848101
:1044C800294BC3F800907FE1102B40F07D81274BEA
:1044D800C3F800B0C3F804A0B9F1000F02D0224B12
:1044E800C3F800902148224B0222011D1A7003F0E4
:1044F8007DF969E1A0600CF049FBA3681843A0604E
:1045080062E10CF039FBA4F858010CF035FBA4F873
:104518005A010CF031FBA4F85C0155E10CF022FBC8
:1045280084F87A010CF01EFB84F87E010CF01AFB6B
:1045380084F87D010CF016FB84F87F0144E100BF8C
:10454800B8110020E4110020BA2A0020EE2700202C
:10455800901A0020961A0020941A0020921A00201F
:10456800EA110020EC110020FC110020F4110020B9
:10457800A00F0020981A00200CF0FEFAA4F8800181
:104588000CF0FAFAA4F882010CF0ECFA84F8840131
:104598000CF0F2FAA4F8860116E10CF0E3FA84F8BC
:1045A80090010CF0E9FAA4F89A010CF0E5FAA4F8E5
:1045B80096010CF0E1FAA4F898010CF0D3FADAF8B5
:1045C800003084F891015B79082B40F2FD800CF0F3
:1045D800D3FAA4F89C010CF0CFFAA4F89E01F3E0FA
:1045E8000CF0C0FA84F8D6010CF0BCFA84F8D701B4
:1045F8000CF0C2FAA4F8D801E6E092F8059003237B
:10460800B9FBF3F9B9F1120F3FF65FACDFF888A3F5
:104618004FF0000BCB4580F0D7800CF0A3FA8AF856
:10462800A0010CF0A9FA40F2ED23984205DD40F60E
:10463800CA039842A8BF184601E040F2EE20A0F253
:10464800EE2019230BF1010B90FBF3F00AF1020A9B
:104658008AF89F01DEE70CF085FA84F89201B3E04E
:104668000CF080FA04EB090309F10109B9F1080F0C
:1046780083F88801F4D1A7E00CF074FAC4F808B004
:1046880060710CF083FAA3681843A0600CF06AFA12
:1046980084F890010CF070FAA4F858010CF06CFA48
:1046A800A4F85A010CF068FAA4F85C010CF064FA5A
:1046B800A4F880010CF060FAA4F8820184E0537930
:1046C8004FF0070AB3FBFAF2C2EBC2029A1A12F0D1
:1046D800FF0F7FF4FAABB3FBFAFA0AF1FF3A5FFA7D
:1046E8008AFABAF1FF0F6FD00CF03CFA5FFA80FB40
:1046F8004FFA8BF004F06AFC814600283FF4E5ABE2
:1047080080F800B00CF038FAA9F802000CF02AFA88
:1047180089F804000CF026FA89F805000CF022FA52
:1047280089F807000CF01EFA89F80600D5E7DFF8CB
:10473800689209F1400A0CF01FFAA9F8A4020CF0DB
:1047480011FA89F8A6020CF00DFA09F1040989F8A2
:10475800A302D145EFD137E00CF004FA1F288146B7
:104768003FF6B3AB3B685B79082B7FF4AEAB0CF03C
:1047780003FA09F1880904EB890900F03F00A9F858
:1047880006000CF0F9F9B9F80630800100F4FE5083
:104798001843A9F806000CF0E5F9000189F80400AF
:1047A8000CF0E0F999F8043000F00F00184389F88C
:1047B80004000CF0D7F989F805000AF06DFD03E054
:1047C800624B012283F8352000200CF017FAFFF71E
:1047D800D5B95F4B98590CF0FDFD18B932200CF093
:1047E8002BFDF6E70CF06CFF06F06EFE594B5A4AAB
:1047F800DA60FFF7D1B90C2844D00A284BD1574DBD
:1048080057480CF083FA2846232111F03CF808B1E8
:10481800401B20602368002B60D150482360002192
:10482800302210F0FAFF98F80030002B2DD14D4BB4
:104838001B689B0615D54C4B44491B688A6B9A1A12
:10484800002A0EDB494A1278042A0AD9484A03F595
:10485800123303F5F8738B63938A9BB283F4804316
:104868009382444B9B68002B6BD043480FB0BDEC40
:10487800028BBDE8F04F18470BF0EEFBFFF77EB94F
:104888000C2804D13D480CF041FA3D480DE07F2842
:1048980012D1FFF7E0B80D28B1D07F2809D1013B2C
:1048A8002E4A384823600021D1540CF02FFAFFF724
:1048B800D2B82F2B3FF6CFA8A0F12002D2B25E2AA1
:1048C8003FF6C9A813B920283FF4C5A85A1C22608E
:1048D800224AD0540CF012FAFFF7BDB85A1EA95C50
:1048E800202901D1134696E71C4A23600021D154A0
:1048F800254B264DD3F800A0D5F800B0DFF85C9022
:10490800584610F0CEFF07463A464846594610F03A
:10491800D1FF1F4A28B919F8073053445B785B0761
:1049280003D010359542E7D306E0954204D2781CAF
:10493800EB684844984702E016480CF0E7F9002372
:104948006BE70FB0BDEC028BBDE8F08F3010002094
:10495800E029002000ED00E00400FA05781D0020A1
:10496800B6A101088C1A0020842F0020961A002076
:1049780000080048702700206C100020E995010805
:10498800E49501081096010808010020B87C010888
:10499800687E0108F49501087012002010F80A3C9E
:1049A8000133DBB20A2B84BF10F8131C044A00F849
:1049B8000A3C82BF002322F8113000F80A3C7047F5
:1049C800B42E0020334A136C90681944081A40F634
:1049D8008C23984270B513469160D06051603BD9E2
:1049E800127893F945108A4210460BD1111F0829F5
:1049F80008D893F84610182901D8013103E083F844
:104A0800442002E0002183F8461093F944402149EC
:104A1800A24219D191F84740B4B10C310024944214
:104A280006DA1D4D51F8046F25F814600134F6E7D5
:104A38000C2805D01849002421F810400130F7E768
:104A4800164801780131017083F8452000220121C0
:104A58001A7083F8471070BD92F84710C9B1A0F2D8
:104A6800EF2440F2DA518C4208D811780B2905D886
:104A78000B1D0131117042F8230070BD002283F82C
:104A88004720074B03F13002002143F8041F9342EB
:104A9800FAD170BDA0010020B42E00208D060020A0
:104AA800AC010020024A136C0133194411647047A9
:104AB800A0010020024B53F820301B681960704792
:104AC800182B0020064B53F820301A681B89A1F5D3
:104AD8007A7159434FF47A7391FBF3F1116070477F
:104AE800182B0020054B98420CBF054A054A13882D
:104AF80001339BB213800020704700BF0054004070
:104B0800781100207A110020F0B5046D86682368BA
:104B180023F0010323608379054613F0020F4079DF
:104B28000CBF4FF0000E4FF4005E13F0040F14BFDB
:104B38004FF48067002710F0010F14BF04210021F3
:104B48008307206820F001002060626822F4405248
:104B58004EEA02026260226822F4B05323F00C038A
:104B680048BF41F008013B430B432360A36895B05D
:104B780023F44073A360684605F05CFE284B9C4212
:104B880001D10C9B0EE0274B9C4201D10D9B09E003
:104B9800254B9C4201D10E9B04E0244B9C420CBF48
:104BA8000F9B109B2268A879170448BF5B00B3FBD2
:104BB800F6F206FB1233B3EB560F236828BF013217
:104BC8001E0441BF4FF6F073C2F34201134041EA9D
:104BD80003026B7992B213F0020FA28100F0010177
:104BE80014BF4FF400320022DC0748BF42F4803281
:104BF8002B6D11B159680A4302E0596821EA020293
:104C08005A609A6801074CBF42F0080222F0080275
:104C18009A601A6842F001021A6015B0F0BD00BF30
:104C2800003801400044004000480040004C00406B
:104C38003D4B1B78012B30B514BF00240324B1B9B8
:104C4800036A23F0010303628169036A21F0F30117
:104C580023F00A0341F0010142F001021A4341EA3C
:104C6800041181610262836923F00C031BE00429AB
:104C78001DD1016A4FF6EF730B4003628169056A23
:104C8800120121F473414FF65F7342F0100241F4B0
:104C980080712B4092B2134341EA0431816103626F
:104CA800836923F4406383618369836130BD082984
:104CB800016A1AD14FF6FF630B400362C169036AA8
:104CC8009BB289B223F4206343F4807321F0F3018B
:104CD80043EA022241F0010192B241EA0411C161A2
:104CE8000262C2694FF6F37319E04EF6FF730B4088
:104CF8000362C369056A40F6FF41194045F6FF7330
:104D08002B4043F4805343EA023241F4807192B25B
:104D180041EA0431C1610262C2694FF2FF331340B4
:104D2800C361C369C36130BD9C01002038B510F868
:104D38000E2C50F8043C044652B9012200F80E2CFF
:104D480020F80C1C997A18680222BDE838406FE7F1
:104D580030F80C2C20F80A1C891A89B220F8081C93
:104D6800074A10F80F0C002522F8101004F80E5C02
:104D78001868997A2A46FFF75BFF04F8065C38BD85
:104D8800B42E0020044B53F820301BB107289CBFD9
:104D98001B681960704700BFC8020020084A1368E2
:104DA8009B050BD5074B00211970074908684FF67A
:104DB800FE7303400B604FF400735360704700BFED
:104DC80000000240A52F0020300002402DE9F047E6
:104DD800664D2B6866490A78581C02F0FF068E4615
:104DE8000AB10346F6E72B60687BAB6895F80C8040
:104DF800AA7B374639B2202900F09B80DFF880C1B2
:104E08000CEB81033CF82110DC789B78C3F1FF039D
:104E18009BB2002B65D0C3F1FF0363434FF03C0CFA
:104E28001B12B1FBFCF9B9F1050F5DD8DFE809F0F9
:104E3800030B1A293A4AE01ADAB24143B1FBFCF0F3
:104E48001044C0B251E0B1FBFCF00CFB101189B268
:104E5800DAB2C1F13C01E31A4B432046B3FBFCFC38
:104E680094442CE0B1FBFCF00CFB10115FFA83F8C2
:104E7800E21A89B24A43B2FBFCF24244D2B220465B
:104E880032E0B1FBFCF90CFB191189B25FFA83F827
:104E9800E01AC1F13C014843B0FBFCF04044C0B209
:104EA800224621E0B1FBFCF80CFB1811D8B289B2FC
:104EB800E31A01FB03F2B2FBFCFC224684445FFACE
:104EC8008CF412E0B1FBFCF80CFB181189B2D8B2D3
:104ED800C1F13C01E31A4B43B3FBFCF20244D2B2EA
:104EE80003E02246204600E044464FEA042C4CEA00
:104EF800004C4CEA020C172306F117014FF0010889
:104F080008FA03F8C91A18EA0C0F89B2DFF8748096
:104F180014BF4FF011094FF0090913F1FF3308F8D6
:104F28000190E9D218360137B6B2BFB2114BA0468C
:104F380060E7AA73AB60104AE98001238EF800305D
:104F48000E4985F80C8040F22A336873AE805360AE
:104F580000234B620B889BB243F001030B8013685C
:104F680043F001031360BDE8F08700BF7010002014
:104F7800A52F00207C100020300002400044014092
:104F8800DA0D00203503002073B506460D460024CF
:104F980001232A88A34013421AD0AA78009302F06A
:104FA80003038DF80430EB78022B03D0032B0CBFDE
:104FB800032301238DF805303046C2F301136946F7
:104FC800C2F381028DF806308DF8072005F0A0FDA8
:104FD8000134102CDCD102B070BD2DE9F04F734EB6
:104FE800F57B07460C4687B011469A4600686B1C4D
:104FF800914622464FF0020BF37308F051FB3B89B0
:105008007868ADF8043001A98DF806B08DF807B0BE
:10501800FFF7BAFF0023ADF80A30ADF81230ADF84B
:10502800163070230193BA7A3C68CDF80CA001239E
:1050380006F110082D01ADF808304FF48073A8442C
:10504800ADF810B0ADF814300C2A7ED8DFE802F0C5
:10505800077D7D7D0F7D7D7D387D7D7D5E002046D1
:1050680001A905F0A9FBA36943F0080326E0236A18
:105078004F4823F010032362236A6168A26922F073
:10508800807222F4E642844242F4E04206D000F5FF
:105098000060844202D043F0300307E023F0E003CD
:1050A80021F4406143F0300341F480616160A26102
:1050B800C4F838A02362A36943F40063A36144E001
:1050C800236A3B4823F480732362226A6168E36998
:1050D800844223F0730343F0700306D000F50060A8
:1050E800844202D042F4407207E022F4606221F464
:1050F800405142F4407241F480516160E361C4F868
:105108003CA02262E36943F008031DE0236A2848B3
:1051180023F480532362226A6168E369844223F49A
:10512800E64343F4E04342F4405203D000F5006004
:10513800844201D141F480416160E361C4F840A038
:105148002262E36943F40063E3613A7B3B681AB186
:105158005A6C42F400425A641A8892B242F0010230
:105168001A80BA7A0C2A18D8DFE802F0071717173E
:105178000B1717170F1717171300721903F13401BC
:105188000AE0721903F1380106E0721903F13C01D3
:1051980002E0721903F14001116135444046A5F857
:1051A80018906B6107B0BDE8F08F00BF7010002049
:1051B800002C0140F8B53A4E3A4C4000C7B24FF4C3
:1051C80020453068C4F8D050D0F818E01EF4004FDD
:1051D80005D0AE46013DBEF1000FF5D116E0D0F87E
:1051E80004E0314D0EEA050545F490353D43456030
:1051F8004FF42045C4F8D050D0F818E01EF0020F44
:105208002DD1AE46013DBEF1000FF5D1C4F8D05006
:105218001FE02946013D0029F8D081694906F8D5E3
:10522800C4F8D05020494568294041F0007141F444
:10523800105141EA0241394341604FF42041A2B183
:10524800306885696D071ED411F1FF31F9D2C4F8B1
:10525800D010FFF747FC003018BF0120F8BD4FF40D
:1052680020458162C4F8D050D7E73068C4F8D01020
:105278000B46826992060CD41A46013B002AF8D1E3
:10528800C4F8D030E5E7416A03F8011B013AD2B20D
:10529800D3E7C4F8D0302023C3610120F8BD00BF94
:1052A8007411002070100020009800FC400070B5B8
:1052B800C5B23248324B00684FF42044C3F8D0409E
:1052C8008669360404D52646013C002EF8D113E041
:1052D80046682C4C344044F0807444F490342C4399
:1052E80044604FF42044C3F8D0408669B60729D4F7
:1052F8002646013C002EF8D1C3F8D0401CE02146D8
:10530800013C0029F8D081690E06F8D544681D498A
:10531800214041F0007141F48031294341604FF44C
:105328002041C3F8D0108469A40711D40C46013970
:10533800002CF8D1C3F8D010FFF7D4FB003018BF09
:10534800012070BD4FF420448162C3F8D040DAE7F1
:1053580082624FF42042C3F8D0208169890606D4BE
:105368001146013A0029F8D1C3F8D020E4E7C3F880
:10537800D0202023C361012070BD00BF741100201C
:1053880070100020009800FC2DE9F0474D282DED05
:10539800028B044600F0608600F2B980302800F0E5
:1053A800DB8651D8222800F09D8423D8032800F0FA
:1053B8000B8214D8012800F0FB81022840F00487F2
:1053C80004200BF01BFC43200BF0E9FB4C200BF0F6
:1053D800E6FB46200BF0E3FB4C2000F063BE0428FC
:1053E80000F0FB81052840F0EF861A200BF006FC40
:1053F800002402E2282800F0EE8515D8242800F0C1
:10540800D585262840F0E086D14C06200BF0F6FB27
:10541800B4F858010BF0F5FBB4F85A010BF0F1FBA6
:10542800B4F85C0100F0BFBD2C2800F0E7852E28F9
:1054380000F062862A2840F0C78601200BF0DEFBC8
:10544800C34B587900F02EBE3D2800F0FF821ED8CD
:10545800362800F038860BD8322800F01D8634280C
:1054680040F0B28648200BF0C9FB002500F05CBC78
:105478003A2800F0C2823B2800F02D84382840F0FA
:10548800A38604200BF0BAFBB14C00F095BD45286B
:1054980000F0878627D8402800F00786422840F089
:1054A8009386AB4C10200BF0A9FB60790BF077FBCF
:1054B800A0680BF0AFFB94F890010BF070FBB4F808
:1054C80058010BF09EFBB4F85A010BF09AFBB4F8A4
:1054D8005C010BF096FBB4F880010BF092FBB4F87A
:1054E800820100F060BD492800F0BB824B2800F023
:1054F800A485462840F068860D200BF07FFB00202D
:105508000BF04DFB00200BF085FB00F055BE70281A
:1055180000F0F68200F2E580692800F04C8200F283
:10552800B680662800F0A68100F2A680642800F004
:105538007D81652840F04886864C0B200BF05EFB89
:1055480020880BF05EFB6268834B9A420CBF20896F
:10555800608980B20BF055FB804B1B68C3F3C00019
:10556800C3F38002800040EA4200C3F340021043C4
:10557800C3F3401240EAC20003F0100318430BF0D3
:1055880040FB774B1A88E368247C02F0080103F497
:10559800475949EA010903F4804149EA010903F43A
:1055A800004149EA010903F4803149EA010903F499
:1055B800003149EA010903F4802149EA010903F4A9
:1055C800002149EA010903F4801149EA010903F0BD
:1055D800007349EA0303DFF8A89199F8009012F0E4
:1055E800010FC9F3800914BF4FF002084FF00008FB
:1055F80043EA090312F0020F43EA080314BF4FF00D
:10560800040C4FF0000C12F0040F43EA0C0C14BF0A
:105618004FF0100E4FF0000E12F0400F14BF20276D
:1056280000274CEA0E0E12F0100F14BF4FF400764C
:1056380000264EEA070712F0200F14BF4FF48065CA
:1056480000253E4312F4807F14BF4FF40060002011
:10565800354312F4007F14BF4FF400110021284392
:1056680012F4806F41EA000114BF4FF080630023F9
:10567800002019430346E9E0672800F023816828E1
:1056880040F0A28510200BF0B9FA00248AE16C28BA
:1056980000F0A48117D86A2800F008846B2840F02D
:1056A800938505200BF0AAFA2E4B18880BF0A9FA5F
:1056B8002D4B18880BF0A5FA264B93F87A0000F0CA
:1056C800010000F0EFBC6E28224D00F09A8100F234
:1056D800EF8106200BF092FAA86E0BF09BFA234B91
:1056E80089E1782800F0FB8018D8742800F03D8301
:1056F8000AD8722800F09A83732840F0658508203C
:105708000BF07CFA0124CAE3762800F0EF8300F25C
:105718006D832F200BF072FA154CD4E2A42800F008
:105728000E842FD87B2800F07482A02840F04C8586
:105738000C200BF063FA0F4B18680BF06BFA0E4B4A
:1057480018680BF067FA0D4B186800F039BD00BFF8
:105758007012002070110020005400408C1A0020A4
:10576800541B00200A1B00200C1B0020581200208C
:105778000F760108ACF7FF1FB0F7FF1FB4F7FF1F44
:10578800A62F0020F12800F0E680FE2800F0FE8316
:10579800F02840F01985B64C04200BF02FFAA36CC2
:1057A800B3F866000BF02DFAA36CB3F86400FAE3C3
:1057B80003200BF023FA00200BF0F1F920460BF040
:1057C800EEF90D2000F06EBC0BF018FA01200BF07A
:1057D800E6F90B200BF0E3F9AFE306200BF00EFA25
:1057E80043200BF0DCF94C200BF0D9F942200BF0E8
:1057F800D6F952200BF0D3F9D4E39E4B185D01344F
:105808000BF0CDF90B2CF8D100249B4B185D01341B
:105818000BF0C5F9082CF8D10024984B185D013419
:105828000BF0BDF9072CF8D100F0CCBC07200BF029
:10583800E5F9E7200BF0B3F9914B58790BF0AFF984
:1058480000200BF0ACF9042000F0BABCA3420AD245
:105858008C4A9D5C012202FA05F50D421CBF9A4054
:1058680010430133F2E70BF0D5F9854B93F8D007D5
:1058780000F018BC12200BF0C1F9834B1B88B3F55C
:10588800806F8CBF082501250024804B33F9140054
:1058980090FBF5F0013480B20BF0B3F9032CF4D18E
:1058A800734CA08D0BF0ADF9E08D0BF0AAF9208EAA
:1058B8000BF0A7F9608E0BF0A4F9A08E0BF0A1F9FC
:1058C800E08E70E310200BF099F90024704B185DFE
:1058D80001340BF064F9102CF8D100F073BC70207F
:1058E8000BF08CF90026624D0E24AB6C74432344F4
:1058F8000136B3F825010BF084F9AB6C2344B3F8F7
:1059080027010BF07EF9AB6C2344B3F829010BF0A7
:1059180078F9AB6C234493F82B010BF040F9AB6C8E
:10592800234493F82C010BF03AF9AB6C234493F819
:105938002D010BF034F9AB6C234493F82E010BF0D6
:105948002EF9AB6C1C44D4F82F010BF063F9082E28
:10595800C9D100F037BC7020494C0BF04FF904F165
:10596800700594F8D0000BF01AF994F8D1000BF0F8
:1059780016F994F8D2000BF012F994F8D3000BF052
:105988000EF994F8D4000BF00AF994F8D5000BF04E
:1059980006F9073494F8CF000BF001F9AC42E0D1D6
:1059A80000F010BC3B4B185D01340BF0F8F8102CDC
:1059B800F8D100F007BC384D2878400000F0FE0010
:1059C8000BF01CF900242B789C4280F0FB83334BAE
:1059D80033F814000BF015F90134F4E7244C0620D1
:1059E8000BF00CF9B4F864000BF00BF9B4F866008E
:1059F8000BF007F92A4B1888D5E204200BF0FEF8C3
:105A0800DDE307200BF0FAF8264B1888FF28A8BF1B
:105A1800FF20C0B20BF0C3F8234B186880F31000C6
:105A280080B20BF0EEF8B5F86C000BF0EAF8144B06
:105A380093F885211D4B186822B10A23584380F337
:105A4800100001E000F30F0080B2ACE20C4C022021
:105A58000BF0D4F894F8E0010BF0A1F894F8DF010A
:105A680020E302200BF0CAF8014BB3F870009AE269
:105A78007011002037930108439301081B93010814
:105A88007012002081110020040000205212002012
:105A9800A8110020BC1100207C2A0020202F002003
:105AA800601200207C1A0020881A0020841A002026
:105AB8000B200BF0A3F86B6F18780BF070F86B6F76
:105AC80058780BF06CF800266B6FC44C33440136E1
:105AD80018790BF064F8032EF6D1636FD8790BF0C0
:105AE8005EF8636F98780BF05AF8636FD8780BF00C
:105AF80056F8636F58890BF084F8636F187AD1E20F
:105B0800B64C1E200BF07AF8A36C1B78022B4FF0D2
:105B180000056BD1A36C03EB850393ED080AB2EE85
:105B2800048A20EE080A10F087F880F30800C0B253
:105B38000BF035F8A36CDFEDAA7A03EB850393ED40
:105B48000B0A20EE270A10F077F880F30800C0B29D
:105B58000BF025F8A36CDFEDA37A03EB850393ED37
:105B68000E0A20EE270A10F067F880F30800C0B28A
:105B780001350BF014F8032DCCD1072DA36C23D1DC
:105B880093ED110A20EE080A10F056F880F3080089
:105B9800C0B20BF004F8A36C93ED120A20EE080AC9
:105BA80010F04AF880F30800C0B20AF0F8FFA36CBE
:105BB80093F84C3000EE103AB8EE400A10F03CF87A
:105BC80080F30800C0B20BE02B4458780AF0E7FFD6
:105BD800A36C2B44D87A0AF0E2FFA36C2B44587DBF
:105BE80001350AF0DCFF0A2DC7D1EBE2A36C2B4488
:105BF80058780AF0D4FFA36C2B44D87A0AF0CFFF68
:105C0800A36C2B440135587D0AF0C9FF0A2DEDD14C
:105C1800D8E23C200AF0F2FF0024704D9FED718A13
:105C2800AB6C03EB840393ED080A20EE080A10F02E
:105C380003F880B20AF0E5FFAB6C03EB840393ED45
:105C48000B0A20EE080A0FF0F7FF80B20AF0D9FF1E
:105C5800AB6C03EB840393ED0E0A20EE080A0FF0F9
:105C6800EBFF013480B20AF0CCFF032CD5D1072C0E
:105C7800AB6C16D193ED110A20EE080A0FF0DCFF89
:105C880080B20AF0BEFFAB6C93ED120A20EE080A50
:105C98000FF0D2FF80B20AF0B4FFAB6C93F84C005F
:105CA8000BE0234458780AF0ACFFAB6C2344D87A55
:105CB8000AF0A7FFAB6C2344587D01340AF0A1FF1A
:105CC8000A2CD4D17EE214F8010F002800F07A8261
:105CD8000AF065FFF7E701200AF090FF3F4B9B6C45
:105CE8001878DFE150200AF089FF00253B4B9C6CB7
:105CF8003D4B04EB85040C2194F8852001FB02330D
:105D0800013593F838000AF04AFF94F886000AF043
:105D180046FF94F887000AF042FF94F888000AF0DA
:105D28003EFF142DE2D14DE22C4B9C6C062303FB65
:105D38000544013594F8DA000AF031FF94F8D500EB
:105D48000AF02DFF94F8D6000AF029FF94F8D7003E
:105D58000AF025FF94F8D8000AF021FF94F8D9003A
:105D68000AF01DFF0C2DDFD12CE24FF000080126B0
:105D780000271A4B1A7C974227DA11330024FA5C61
:105D8800194D0C2305F130016343595C914207D149
:105D98002B44586B0FF085FD82462EB9B14605E0BD
:105DA80001341C2CECD10EE080440CE0D1450ADA19
:105DB8000C2303FB04535B6B13F809000AF0EFFE96
:105DC80009F10109F2E70137D3E7002E00F0FA8163
:105DD8005FFA88F00AF012FF0026C9E77011002068
:105DE8000000C84200007A4410760108CD4D287C96
:105DF8000AF004FF00242B7C9C4280F0E381CA4B0C
:105E0800E65C0021C9480C2200F1300702FB01F3CF
:105E1800DA5DB24205D1034493F838000AF0BFFEB8
:105E280002E001311C29EDD10134E4E7C04C162011
:105E38000AF0E4FEB4F896010AF0E3FEB4F8400173
:105E48000AF0DFFEB4F842010AF0DBFEB4F84401C0
:105E58000AF0D7FEB4F8D8010AF0D3FE94F8ED01A1
:105E68000AF09DFE00200AF09AFE94F8EE010AF06E
:105E780096FE94F885010AF092FE94F892010AF0D1
:105E88008EFE00200AF08BFEA64B9B6C0A20B3F90D
:105E9800623093FBF0F080B20AF0B3FE8CE0E0B21F
:105EA80001340AF07CFE092CF9D18BE110200AF0AC
:105EB800A5FEA04BA04C187800F002000AF06FFE77
:105EC8009E4B18780AF06BFE20680AF0A3FE606803
:105ED8000AF0A0FE9A4B18880AF093FE994B18888E
:105EE8000AF08FFE8F4BB3F878005CE00AF03AFEB8
:105EF800074612200AF082FE8A4C1FB9E66FD4F8D2
:105F0800805007E0102F13BF0025D4F88460D4F820
:105F180088502E4638460AF042FE30460AF07AFE8D
:105F280028460AF077FED4F88C000AF073FE0020A9
:105F38000AF067FE00200AF064FE0020B2E0794D06
:105F480095F8900080000130C0B20AF057FE95F82D
:105F580090000AF024FE00242E4696F890309C42C9
:105F680080F03081784D285D0AF019FE05F11003A4
:105F7800185D0AF014FE05F120033035185D0AF0AB
:105F88000EFE285D0AF00BFE0134E6E708200AF051
:105F980035FE00200AF035FE00200AF032FE00200F
:105FA8000AF02FFE00200AF02CFE0BE104200AF074
:105FB80025FE5F4B986803E194F87A010AF0EFFD3B
:105FC80094F87E010AF0EBFD94F87D010AF0E7FDF4
:105FD80094F87F0166E0564C07200AF00FFEB4F8EB
:105FE80080010AF00EFEB4F882010AF00AFE94F865
:105FF80084010AF0D4FDB4F88601D4E74C4C0C2097
:106008000AF0FCFD94F890010AF0C9FDB4F89A0171
:106018000AF0F7FDB4F896010AF0F3FDB4F8980118
:106028000AF0EFFD94F891010AF0B9FDB4F89C016B
:106038000AF0E7FDB4F89E01B5E73D4C04200AF0EC
:10604800DDFD94F8D6010AF0AAFD94F8D7010AF00C
:10605800A6FDB4F8D801A6E73C4C3D4D207800EBEE
:106068004000C0B20AF0CAFD002623789E4205F11E
:10607800020580F0A78015F8020C0AF090FD15F8CB
:10608800010C00EB800000EB800000F2EE2080B2F3
:106098000AF0B7FD0136E8E701200AF0AFFD244B0E
:1060A80093F892010AF07BFD8CE008200AF0A6FD27
:1060B80000241F4B2344013493F888010AF06FFD34
:1060C800082CF6D17EE0174B194C93F8D100C0EBA1
:1060D800C000C0B20AF092FD04F1200594F8F40162
:1060E80000231C4AD25C904270D00C33302BF8D17C
:1060F8000834AC42F2D165E040200D4C0AF07EFD38
:1061080004F14005B4F8A4020AF07BFD94F8A60255
:106118000AF045FD043494F8A3020AF040FDAC42AD
:10612800F0D14FE070110020811100201076010895
:1061380070120020901A0020981A0020961A002049
:10614800941A0020921A0020011200207C2A0020B4
:1061580010140020882A0020E0202A4C0AF04EFD66
:1061680004F18005B4F8260200F03F000AF049FD6A
:10617800B4F82602C0F386100AF043FD94F824020E
:1061880000090AF00CFD94F8240200F00F000AF050
:1061980006FD043494F821020AF001FDAC42E1D175
:1061A80010E013200AF02AFD0024174B185D013473
:1061B8000AF0F5FC0B2CF8D100200AF02BFD00208A
:1061C8000AF028FD012018E0002016E00AF0E7FC9C
:1061D800B4F8F6010AF015FD94F8F8010AF0DFFCAE
:1061E80094F8F9010AF0DBFC94F8FB010AF0D7FCFB
:1061F80094F8FA010AF0D3FC7AE7BDEC028BBDE80B
:10620800F08700BF70120020379301082DE9F04392
:10621800C34C237887B00746002B00F004826268DD
:10622800A368D31A7C2B40F2FE81237BA260013342
:106238002373002606F12400B94DC0B20BF0BEFE50
:1062480005F10E0333F9163007EE903AB54B1B886B
:10625800B8EEE77A07EE903AF8EEE77A0136C7EE3D
:10626800277A9FEDB17A67EE877AFDEEE77ACDED72
:10627800037ABDF90C000BF08FFE032EDAD1302023
:106288000BF09CFEB5F914000BF086FE0BF08EFEA9
:106298002B7B9E072BD1AA6841F288339A4217D9E3
:1062A80010200BF08BFE6426A86990FBF6F000B274
:1062B8000BF072FE21200BF081FEA86990FBF6F32B
:1062C80006FB13000028B8BF404200B20BF064FE82
:1062D80014200BF073FEB4F91C000BF05DFE1C20BB
:1062E8000BF06CFE00200BF057FE0BF05FFE237BDB
:1062F8008B4E580740F0748102200BF05FFE306A25
:106308006423323090FBF3F000B20BF045FE03201B
:10631800B6F92A500BF052FE844B1B7859074FF000
:10632800050895FBF8F5ADB20DD506F5DA703946D6
:106338000AF022FF28B9D6F8303813F0100F18BF2A
:10634800002528B205E0D6F834389889B0FBF8F073
:1063580000B20BF021FED4F83038714D9A0740F1A5
:106368008880DFF8D881B5F83A6898F80030B5F831
:10637800382836016427B6B207FB02325B00B2FB4D
:10638800F3F346EA0326B6B2C3F303231E430620FB
:106398000BF014FE30B20BF0FFFDB5F83A3898F860
:1063A800001001339BB293FBF1F201FB1233A5F805
:1063B8003A38D5F83C389B7B012B05D139200BF0B6
:1063C800FDFDB5F938081AE0B5F838586E233A20BB
:1063D8005D4315260BF0F2FD95FBF6F5AEB2B6FB64
:1063E800F7F528B20BF0D8FD07FB15653B200BF03D
:1063F800E5FDA8B2451D0A2095FBF0F000B20BF0B0
:10640800CBFD28200BF0DAFDD4F84038444D0A20A3
:1064180093FBF0F000B20BF0BFFD04200BF0CEFDB3
:10642800D4F83438D5F844089A894FF6FF7398425F
:10643800A8BF1846C2B10028ACBF131A134607EE0E
:10644800903A9FED3B7AF8EEE77A67EE877A07EEA7
:10645800102AB8EEC77AC7EE877AFDEEE77A17EE0C
:10646800900A6428A8BF642020EAE07000B20BF00C
:1064780093FDD4F848382A4E9B0640F1A68096F83A
:106488004C389F071DD511200BF098FDB6F84E0823
:10649800284B4FF4F365684390FBF3F000B20BF020
:1064A8007BFD19200BF08AFDB6F84E0845436420A1
:1064B80095FBF0F595FBF0F300FB135000B20BF0E1
:1064C8006BFD94F84C38B4F8505813F0020F08BF1D
:1064D800002501200BF072FD28B20BF05DFD0920AC
:1064E8000BF06CFD00200BF057FD134B94F852583D
:1064F8001A88B2F5967F0AD9094B1B7B03F00F0364
:10650800072B04D842F20F75954228BF154605207F
:106518000BF054FDD4F83C385B7B9BB928B22EE0D5
:10652800441200200400002000007A44A62F002016
:106538000000C842A0860100FE000020FC000020E8
:106548006666E63FA5F1200307EE903A1FED047A50
:10655800F8EEE77AF6EE006AC7EE877ABEEE007AC2
:10656800F5EEC07AF1EE10FA58BFB0EE667A77EE23
:10657800877AFDEEE77ACDED037ABDF90C000BF0D2
:106588000BFD94F84C28C84B950703D493F853286F
:10659800012A04D1012384F85338C4481CE0D3F8F5
:1065A8003C38DFEDC36A93ED017AD3ED027A27EE2A
:1065B800267A67EEA67ABDEEC77AFDEEE77A8DED0C
:1065C800047ACDED057A04A806E0BA4A92E80300F9
:1065D80004AB83E80300184602F030F80BF0E6FC41
:1065E800227BB14B282A1ED100221A733C265B68F5
:1065F8004FF47A70B3FBF0F717200BF0DFFCB7FB12
:10660800F6F5B5FBF6F006FB1050000200B20BF0F1
:10661800C3FC18200BF0D2FC06FB157000B20BF07F
:10662800BBFC0BF0C3FC94F85C389F4D002B00F0CA
:106638005E810AF0E5FDD5F860389F4AC31A934297
:10664800064640F2C580002385F8663885F8683824
:10665800B5F83838DAB21B0A85F8822885F8833805
:1066680085F8782885F87938D5F890286B689A1ACB
:10667800D5F89438D97B4FF47A734B439A420DD3AB
:106688006B68C5F8903895F89838013B012B9FBF87
:10669800102385F86638022385F868380A20D4F86C
:1066A800402892FBF0F284F88028121284F881289E
:1066B80094F84C28D4F8443893FBF0F384F88438E1
:1066C8001B1284F88538900794F85238764984F874
:1066D800B33803D42D2381F8B43877E0042BD4F8E9
:1066E8005498D4F85878DFF8E081744A8CBF332383
:1066F800322381F8B4384FF0060C714B99FBF3F054
:1067080097FBF3F308FB009108FB037803EB830383
:106718000CFB01F103EB830391FBF2FE642502FB02
:106728001E119B0091FBF5F184F8A51809120CFBCA
:1067380008FC84F8A6189CFBF2F143FA81F39BB29B
:1067480002FB11C292FBF5F284F8AA28121284F80F
:10675800A83884F8AB281B0AB4F84E2884F8A9385E
:106768002423534393FBF5F5B4F8C63884F8AC38C2
:1067780000EB80001B0A00EB8000800084F8AD3835
:106788000A22B4F85038B3FBF2F303F5FA739BB25C
:1067980040FA8EF080B284F8AE381B0A4FEAD979F5
:1067A80084F8A308FF0F000A84F8A05884F8AF38CB
:1067B800C5F30725B4F8C83884F8A29884F8A40863
:1067C80084F8A77884F8A15884F8B538C4F86068C4
:1067D80094F8CA88344DB8F1000F0DD1D5F8D00817
:1067E8000AF001FE012807D90228364F00F060821E
:1067F80001F016FF0123BB70D4F8D4282A4D002AD3
:1068080075D095F8CA783FB1D5F8DC3840F6B7317D
:10681800F31A8B4219D86AE00123D5F8D00885F815
:10682800CA3802F0C0FAD5F8E03893F9000002231C
:106838008DE8880008213A464FF4964302F0C6FADC
:1068480085F8E478C5F8D0084FE095F8D878CFB93E
:10685800D5F8D008C5F8D47885F8CA7802F0A3FA34
:10686800D5F8E03893F9000001238DE88800082165
:106878003A464FF4964302F0A9FAC5F8D00801F059
:10688800CFFE32E0013FFFB285F8D87895F8E418DA
:1068980095F8E538D7B94A1C013385F8E42885F816
:1068A800E538D5F8D0081EE044120020981A0020D8
:1068B8008096184B9C7701083F0D030040420F005B
:1068C8008096980004000020806967FF12F8017B19
:1068D800C5F8D428781885F8E4080133D5F8D00825
:1068E80085F8E53839460AF081FDC4F8DC6894F883
:1068F800E638A54DF3B1D5F8E838DBB1D5F8EC3872
:10690800C3B1C5F8F0381B68A04AC5F8F438D5F803
:10691800F8381344187AFEF737FDD5F8F038987927
:106928000AF03DF9D5F8F8380133092B88BF002360
:10693800C5F8F83894F8FC28934B6568002A00F0ED
:10694800F281D3F80029002A00F0ED8193F8043988
:10695800013B012B00F2E781D4F800098A4E0AF0C6
:1069680042FDE0B1D6F800090AF03AFD96F805397B
:10697800D6F804807E2B07460ED102231B2886F802
:10698800043909D1D6F800090AF02DFD20B90123F0
:10699800C6F8088986F80C3984F80579DCE7D6F852
:1069A800082973689B1A41F6583293421FD903236A
:1069B80086F80439B7E1764A32F8130010B903466D
:1069C8004FF403600133B0F5C06FDBB27ED020D93D
:1069D800B0F5006F00F0848033D9B0F5036F40D173
:1069E80084F80D39D4F84838674E9B0640D494F89B
:1069F8000C6994F80D39002E00F0578162686249DD
:106A0800521B012AD7D981F80D39002381F80C3996
:106A180089E1B0F5007F43D007D8B0F5807F4CD02E
:106A2800B0F5887F00F09180E5E7B0F5806F00F061
:106A3800B180B0F5826F00F0F680B0F5047FDAD14E
:106A480023E0B0F5E26F00F09180B0F5E46F00F05C
:106A58009280B0F5E06FCED184F80D39B4F90E10FC
:106A68008DE0B0F5046F7AD0B0F5026FC3D105E1BF
:106A780096F84C389F07BAD5B6F84E1824234B43DE
:106A88001233642193FBF1F109E184F80D39D4F84C
:106A980030383D4E9907AAD5B6F838380A21FDE0B6
:106AA80084F80D39D4F83038374E1A059FD5D6F802
:106AB80040180A2391FBF3F1F1E084F80D39D4F87A
:106AC8004838314E5B0792D5B169E8E084F80D3952
:106AD800D4F830382C4E1F0589D5D6F84418DEE096
:106AE800D4F84818284A84F80D3988067FF57FAF0E
:106AF80092F84C1889077FF57AAFDB0712D5D2F8E0
:106B0800583883EAE371002BA1EBE37101EB5101E3
:106B18004FF01902B1FBF2F1ACBF41F0004141F076
:106B280040410FE0D2F8543883EAE371A1EBE371F6
:106B3800002B01EB51014FF01902B1FBF2F1B8BF84
:106B480041F080414FF4006087E084F80D39D4F8B3
:106B580048380D4E5F077FF54AAF71699FE0B4F979
:106B68001C1084F80D396423594376E084F80D39F4
:106B7800B4F9101003E0B4F9121084F80D392C237D
:106B880091FBF3F169E000BF441200209C770108F3
:106B98002E97010884F80D3994F80E39634A0133A9
:106BA800DBB2032B88BF012382F80E3994F80E1943
:106BB80042F2107359435E4B1B78D80748BF013126
:106BC8009A0748BF02315F07B4F8103948BF04314B
:106BD800DE0748BF0A31980748BF14311A0648BF74
:106BE8002831DF0548BF28315E0748BF64311807E0
:106BF80048BFC8319A0548BF01F5C8719F0648BF0C
:106C080001F57A71DE0648BF01F5FA61580648BFFA
:106C180001F57A614FF4806001F0CEFC434B00220D
:106C280083F80C29E3E6D4F84818404F84F80D3966
:106C380011F0200617D097F84C2812F0020F14BF55
:106C48004FF47A71002112F0010F14BF4FF4FA6368
:106C580000230B4494F85218194401F0ADFC0023AA
:106C680084F80C39C3E6D7F8303819067FF5BFAE7B
:106C7800314601F0A1FC87F80C69B8E684F80D39B3
:106C8800D4F84838294E9A067FF5B1AE96F84C38B4
:106C98009B077FF5ACAEB6F850386421594301F034
:106CA8008BFC002386F80C39A1E684F80D393AE00C
:106CB800BB7823B1C5F8CC6887F802809CE5D5F885
:106CC800CC38F31AB3F57A6FFFF496AD0123D5F8F3
:106CD800D008BB700AF084FB0746D5F8D0080AF044
:106CE8007FFB79067FF488AD8A2802D08E280DD0E4
:106CF80082E5D5F848389A067FF57EAD95F8CA380A
:106D0800002B7FF479AD05F6990306E095F8CA38AB
:106D1800002B7FF471AD05F66403C5F8D4382D2334
:106D280085F8D83868E507B0BDE8F083441200203C
:106D3800A62F0020FF20704790F844305A1C0344C7
:106D4800D2B22DE9F04380F8442083F8301090F84F
:106D580045300BB1132A4FD9002380F84430002A5C
:106D68004AD0264B1968002946D01B68052B43D109
:106D78002349202A144628BF2024651C0E686D105C
:106D8800204F3B6883BBDFF88CC000F13203AE466E
:106D980013F8019C13F8028CBEF1010E48EA092889
:106DA8002CF8048C03F102030CF1040CF0D1164BFF
:106DB8001B681FFA83FE154B73445B00A646D3F885
:106DC80000C01C603B6823443B60114F3B6823F4C0
:106DD800E04323F040039BB283F0300343F40043C5
:106DE80043F080033B6001E04FF0000E964503D06E
:106DF8000B689B1B312BC3D9BDE8F083882F00207B
:106E080048120020D8290020505C00400A30002099
:106E1800045C004084610040014B1868C0B27047B0
:106E280094290020012070477047704707EE900AA8
:106E3800F8EEE77ADFED0C6A9FED0C0AF5EEC07A02
:106E4800F1EE10FAD4BFB1EE677AC7EEA67A08B5AC
:106E5800D8BFC7EE267A27EE800A04F005FB044B5C
:106E680083ED000A08BD00BF8096184B35FA8E3CAA
:106E78006C000020F7B51C4B1A680AB91C6800E0C2
:106E880001241A490E780022D0B2A04202F1010270
:106E980007D202AD2F18164D3544285C07F8040CAC
:106EA800F2E71A68121B1A600A781D6822440A70F1
:106EB8009DB90320402103F013FB0E4A136823F405
:106EC800804323F070039BB283F4405343F40043A0
:106ED80043F080031360054B1D70002CCBD09DF848
:106EE800040003B0F0BD00BF94290020581B002007
:106EF800982900200C5C004013B5062204460321A3
:106F08001E206B46FEF756F900283DD09DF800205C
:106F18009DF801309DF8021043EA02231BB21B4A78
:106F280007EE903A92ED007AF8EEE77A012067EEE4
:106F3800877A92ED027AFDEEE77A17EE903A23808F
:106F48009DF8033043EA01231BB207EE903AF8EEAE
:106F5800E77A9DF8041067EE877A92ED017AFDEEE4
:106F6800E77A17EE903AA3809DF8053043EA0123AB
:106F78001BB207EE903AF8EEE77A67EE877AFDEEF5
:106F8800E77A17EE903A638002B010BD080000203F
:106F98002DE9FF41634B1B6893B11A681AB1624926
:106FA800486902434A619A88ADF8042002228DF8A4
:106FB80007209868002201A98DF80620FDF7E4FF54
:106FC80032200AF039F9002111221E20FEF76EF94D
:106FD800012160221E20FEF769F964200AF02CF9CD
:106FE80002A8FFF789FF00240A2726462546022122
:106FF80001221E20FEF75AF932200AF01DF902A8D4
:10700800FFF77AFFBDF90820BDF90A10BDF90C3069
:107018008A421444A8BF0A4693421D44A8BF134697
:1070280013F5805F0E440ADD404A938A9BB283F4CD
:107038008043013F9382DAD14FF0010801E04FF01D
:1070480000081E2000211222FEF730F90A2702212B
:1070580001221E20FEF72AF932200AF0EDF802A8D4
:10706800FFF74AFFBDF90820BDF90A10BDF90C3039
:107078008A42A4EB0204A8BF0A469342A5EB030583
:10708800A8BF134613F5805FA6EB010608DD274A63
:10709800938A9BB283F48043013F9382D7D101E066
:1070A8004FF0000807EE904A9FED217A214FF8EE45
:1070B800E77A0021C7EE277A70221E20F0EEE77AE1
:1070C800C7ED007A07EE906AF8EEE77AC7EE277AFE
:1070D8009FED197AF0EEE77AC7ED017A07EE905A3C
:1070E800F8EEE77AC7EE277AF0EEE77AC7ED027A8C
:1070F800FEF7DCF8012120221E20FEF7D7F81E201B
:1071080002210022FEF7D2F864200AF095F8B8F1BF
:10711800000F04D14FF07E533B607B60BB6004B02E
:10712800BDE8F0811003002000100240000800486C
:1071380000406F460800002001C05E46F8B59B4B32
:107148001B680546187818B1012800F06581DCE253
:10715800242D974C0CD006D80A2D00F0D8800D2D80
:1071680000F0D58042E12A2D06D02C2D04D03DE137
:107178006070A070E0704BE18E4BA17867788C4A04
:10718800002058542FBB19781771472921D15978F5
:1071980050291ED19978472907D1D978472904D190
:1071A8001979412901D1012111719978814A52290E
:1071B80003D1D1784D2900F0AA8299787D4A4729D0
:1071C80007D1D178532904D11279562A04BF032252
:1071D80022712279764E022A38D0032A4BD0012A0E
:1071E80040F08380BA1E072A7FD8DFE802F004083F
:1071F8000F131A257E2A0AF0D9FDA06075E01B78C6
:10720800532B72D1A3685B42A3606EE00AF0CEFDF7
:10721800E0606AE01B78572B67D1E3685B42E36064
:1072280063E01B78302B644B1A788CBF42F0020263
:1072380022F002021A7058E000200AF017FE2074AB
:1072480053E000200AF012FE60824EE0072F06D0BD
:10725800082F4AD101200AF009FEF08245E00120FA
:107268000AF004FE41F2184358434FF47A73B0FB16
:10727800F3F0B08239E0022F07D0032F0AD10020A3
:107288000AF0F4FD4D4B18702FE000200AF0EEFDD7
:1072980030762AE029D93A1F9210337E0132D2B2D1
:1072A800013B02EB8303DBB2102B1ED8F91EC2F19F
:1072B800010201EB8202D2B2012A0BD0042A11D1B9
:1072C80000205E1E0AF0D2FD3D4B98553D4B002232
:1072D8009A5507E05E1E3C4A002093550AF0C6FD09
:1072E8003A4B9855E3690133E361314B2A2D18BFB6
:1072F800DA7807F101074FF000000CBF0122554072
:107308006770A0700CBF83F82020DD7080E094F8CF
:107318002000002846D02E4B13F8012D2D495A7015
:107328008B42F9D1234A224D13785278402B85BFDE
:10733800373B1B011B01DBB298BF03F0F003402A67
:107348008CBF373A303AD2B21344E278DBB29A4271
:1073580025D121230B7028796B6A1E4A0133012835
:107368006B620AD002281CD1722313701A4BAA8AA6
:107378001A801A4BEA8A1A8013E0672313700E4B9F
:107388001B789F070ED5164BAA681A60EA685A60E0
:10739800144B2A7C1A70144B6A8A1A8002E03F2325
:1073A8000B700020002384F8203031E024080020EE
:1073B800581B0020222E0020901A002000120020C6
:1073C8003112002021120020011200201112002089
:1073D8003403002020030020921A0020E811002026
:1073E800981A0020961A0020941A0020A37894F87E
:1073F80020000E2B9FBFAA4A591C9170A94A98BF1A
:10740800D554A74A18B9D3785D40D57000E000205C
:10741800003018BF0120F8BDA14B93F828100022B6
:10742800082900F27281DFE801F0050C101A2B3BE5
:107438005F7B8800B52D40F0688183F82920012200
:107448004FE0622D08BF02224BE0032283F8282078
:1074580083F82A5083F82B5083F82C5055E10422E6
:1074680083F8282093F82B2093F82C1083F82D50BC
:107478002A44D2B283F82B200A4483F82C2044E112
:10748800052283F8282093F82B2093F82C10DD850B
:107498002A44D2B283F82B200A4483F82C2034E102
:1074A800062283F8282093F82B2093F82C102A44DE
:1074B800D2B283F82B200A4483F82C20DA8D02EB11
:1074C8000525ADB2B5F5AC7F88BF754ADD8584BFAB
:1074D800012182F8291000221A86002D40F015811A
:1074E800072283F8282010E193F82B2093F82C101A
:1074F8002A44D2B283F82B200A4483F82C201A8E0F
:10750800B2F5AC7F3CBF6649891802F1010238BF69
:1075180081F83450D98D92B291421A86E0D9F4E0BC
:10752800082283F8282093F82B30AB4200F0ED8036
:107538005B4B012283F829200FE05B4C83F828205D
:1075480014F8012D6270594A9442F9D193F82C101D
:10755800534AA94206D03F232370554A5368013342
:107568005360D2E0516A92F829000131516210B19A
:107578003E232370C9E02121217092F82D1006299D
:1075880041D004D8022907D0032923D0F8BD1229F5
:1075980059D0302967D0F8BD502121704549946BE6
:1075A8004C60D46B0C60516C4FF47A7491FBF4F11D
:1075B800414C218092F88C11404A19B1117841F060
:1075C800020102E0117821F002011170012283F812
:1075D8008D218CE05321217092F83910CE0705D502
:1075E80092F83820D51E6A426A4100E0024602F04D
:1075F800010183F88C11002A79D130490A7822F0E8
:1076080002020A7073E04F21217092F83F10CC07F4
:1076180005D592F83E20D11E4A424A4100E0024672
:1076280002F0010183F88C1122B924490A7822F06A
:1076380002020A70224A93F863101170214AB3F8C3
:107648006010118053E0562121701F49946C0C8002
:1076580042F21074D16C91FBF4F11C4C2180012191
:1076680082F88E1143E04921217092F83810184AA7
:10767800102988BF10211170164914780022A242DF
:1076880032D2154D0E7A5655144D4E7A5655144D24
:10769800CE7A5655134D11F80C6F56550132EEE758
:1076A800581B0020222E0020340300202003002035
:1076B80004080020981A0020941A0020901A00202C
:1076C800961A0020FE000020921A0020E8110020DF
:1076D800001200208C1B0020011200201112002033
:1076E8002112002031120020DA690132DA6193F8A0
:1076F8008D310B4A93B192F88E317BB1002182F81B
:107708008D1182F88E111846F8BD0020F8BD127947
:10771800432A7FF452AD022222714EE5F8BD00BF24
:10772800581B00200449054B0968187000225A614B
:1077380099611A77704700BF48120020040800209A
:1077480010B5121A07EE902A5B1A2DED028BF8EE8F
:10775800E78A07EE903A184B059CB8EEE78AD3ED16
:10776800007A28EE278A28EE080AA8EEA80A0EF062
:10777800ADFCDFED127A049B20EE270AF0EE480AF2
:10778800BCEEC00A83ED000AB1EE680A03F099FD69
:10779800DFED0B7A9FED0B7AE0EE077ABDEC028BFA
:1077A800FDEEE77A17EE903A002BBCBF03F50C43C9
:1077B800A033236010BD00BF6C0000202C7D8E3FDD
:1077C80000A00C46A00CB34544F25063984203DD78
:1077D800A0F50C40A0387047034B9842BCBF00F599
:1077E8000C40A030704700BFB0B9FFFF73B51A4C0A
:1077F800036823600B686360184D0068184EFFF734
:1078080015FB184B009395E8030094E80C000196CB
:10781800FFF796FF144B32681A606868636813496B
:107828001B1A07EE903A124B286893ED007A2368EA
:107838001B1A0B600F4BF8EEE77A1A600E4B67EED7
:10784800877A1B68FDEEE77ADA880C4BC1ED017A7E
:107858001A8002B070BD00BF14290020981A0020B9
:10786800202900201C2900205C2900202429002030
:107878006C00002054290020A40F0020502900206B
:107888004279DFED2A5A2A4B9FED2A5A07EE902AB1
:10789800F8EE677AC27BC7EEA57AB2EE047AC3ED3A
:1078A800007A07EE902AF8EE677A234ADA60C7EE84
:1078B800A57AC3ED017A8179204B07EE901AF8EE8C
:1078C800677A017CDA60C7EE877AC3ED007A07EE43
:1078D800901A817E06EE101AF8EE677AB8EE466ABC
:1078E800C7EEA57A86EE056AC3ED017A83ED026AD2
:1078F800C179134B06EE901A417CDA60F8EE666A9D
:10790800C6EE876A07EE101AC17EC3ED006A07EE5D
:10791800901AB8EE477AF8EE677A87EE257AC7EEBE
:10792800857A83ED017AC3ED027A70470000C84278
:107938002C29002000007A440000FA443C29002049
:107948006029002010B50C4C23789B0713D50B4BEE
:107958001B78042B0FD90A4A0A4B106852685A60E0
:107968001860FFF763FA084B1A88084B1A802378C7
:1079780043F00103237010BD901A0020961A0020CE
:10798800981A0020EC1100206012002070290020B5
:107998002DE9FF47734B744933F9103004462BB96E
:1079A80002280CD0714B1B88980708D0704B002216
:1079B80023F814206F4B1B8821F81430CFE031F8DE
:1079C800143023B96C4A02EB8402C2F890310133B7
:1079D8009BB221F814301BB2002B1CDD022C664A26
:1079E80066480BD1D2F89861B0F90450202095FB75
:1079F800F0F505FB0060C2F898010CE002EB840288
:107A080030F91450D2F89061802095FBF0F505FB11
:107A18000060C2F890015A4F386890F85E2093428F
:107A280040F09D80544ADFF8488102EB840200EB65
:107A3800040E022CD2F8905195FBF3F39EF85750A0
:107A4800C2F8903108BF5E424FF0000221F81420BE
:107A580007BFB6B214219EB20A21002D7DD0002E98
:107A68007BD038F81420002A77D00FFA86F90FFA5D
:107A780082FCE14571D089EAE9728CEAEC7AA2EBE2
:107A8800E972AAEBEC7ACAEB0202B9F1000F12B262
:107A980009B2DFF8F89003DDBCF1000F03DC20E049
:107AA800BCF1000F1DDA8A420BDD022C90F85A2037
:107AB80002D102F580720EE039F8141040320A44FF
:107AC80019E049428A4218DA022C11D190F85A205A
:107AD800C2F57F42C032B9F804100A44A9F804205C
:107AE8000BE0002AB8BF52428A4206DD022C04D0BD
:107AF80039F81420203A29F8142039F914209EF86E
:107B0800549092114A4503DBAA42A8BF2A469146DF
:107B18001C4A126812031FFA89F508D5142001A916
:107B28008DF804400293ADF80C5000F0AFF9164BF5
:107B38001B7873B12AB207EE902AF8EEE77AB2EE14
:107B4800047AC7EE877A3B6803EB8403C3ED087AAF
:107B580003E03B68234483F8019028F8146004B0DC
:107B6800BDE8F0876812002088080020541B002018
:107B7800820800207A080020581B00209C11002051
:107B880074080020741A0020780800207C0800205F
:107B98002E4B2F4A1B68126810B51A602D4A1168BF
:107BA800596051689268DA602B4A996011681961C6
:107BB800516892689A61294A59611168D961516876
:107BC80092685A62264A196211881985518859851E
:107BD8009188D288DA85234A99851188198651882F
:107BE800598692889A86204A1188D9865188198799
:107BF8001946928821F83A2F1C4A107800228242AE
:107C080006DA1B4C34F8124021F8024F0132F6E72D
:107C1800184A1288A3F86420174A1288A3F8662025
:107C2800164A1188A3F86C1051889288A3F870201E
:107C3800134AA3F86E1012689A66124A1288A3F8BB
:107C48007220114A5289A3F85E2010BD8C2C0020A6
:107C5800842F00204C27002058270020642700206C
:107C6800681200209C11002052120020482B00208E
:107C7800BC110020F41E002054100020A211002086
:107C88005C120020DC110020A81100202DE9F84327
:107C98000E4B93E8800305460E460024B44213DADF
:107CA8007B1933F9140008EB050333F9142009EBA9
:107CB800050333F914301344022293FBF2F3C01A7C
:107CC80008F001FE0134E9E7BDE8F8838C2C0020B8
:107CD80070B5472008F050FD174B1B681B0307D5EC
:107CE800164B174A5B6810681B68C01A08F0DCFD61
:107CF800144E154C154D307808F0D6FD23682868C9
:107D0800C01A08F0E0FD63686868C01A08F0DBFD77
:107D18000F4B188808F0C8FD0E4B188808F0C4FDF2
:107D28000D4B188808F0C0FD337823742B68A360C6
:107D38006B68E36070BD00BFF82D00208C2C00201C
:107D4800842F0020961A0020782C0020981A0020F2
:107D5800941A0020921A0020E81100207FB5264CC2
:107D6800264E274D2749284A284B20B12848008805
:107D7800B0F5805F31D23088ADF8040028781E4D08
:107D880091F8201012788DF806008DF807108DF8FC
:107D980008201B788DF8093001A8294606220DF025
:107DA80021FD30B30198BDF808302860AB8053201E
:107DB80008F0E2FC208808F077FDA07808F074FD50
:107DC800E37801932379029301A86379039308F078
:107DD800DBFC0F4B00221A800BE03088208091F8E2
:107DE8002010287812781B78A070E17022716371D6
:107DF800DDE704B070BD00BFF41C0020541B002058
:107E0800901A00204C2F0020880E0020360F0020EA
:107E18001C2E0020A0F17D03012B70B504460D46F1
:107E28000A4E05D830687D2109F0E0FA84F0200474
:107E38003068214609F0DAFA35B12B881C4404EB86
:107E4800142404F0FF042C8070BD00BF441B0020E4
:107E58000A4A138801331380094A136801331360EF
:107E6800084A138801339BB2202B01BF00231380DB
:107E7800054A138808BF0133138070471C2E002061
:107E8800002E0020042E0020062E002038B52A4B94
:107E98001B78083B012B05460C464BD8452008F0BB
:107EA8006BFC284608F068FC0E2D33D003D83DB192
:107EB8000D2D07D038BD142D20D0FF2D32D038BD60
:107EC80020682BE0637820789BB180F0800008F070
:107ED80053FCA568E8B208F04FFCC5F3072008F08A
:107EE8004BFCC5F3074008F047FC280E08F044FC9B
:107EF80004E008F041FC606808F0E5FC207808F030
:107F08003BFC606808F0DFFC2489E0B208F034FC30
:107F1800200A0BE0206808F0C7FC6068BDE838401C
:107F280008F0C2BC054808F005FC0020BDE8384050
:107F380008F022BC38BD00BF6C2C00204E97010809
:107F48002DE9F04FB74BB84F1A888BB00193002A30
:107F580040F0A380B7F8F607B44E42F20103C21A04
:107F680050425041FFF7FAFEFFF712FE34684920ED
:107F780008F002FCAE4B2546186808F095FC55F849
:107F8800040B08F091FC284607F066FF04F1100086
:107F980007F062FF04F11C094FF01008A54D0123FA
:107FA8002A6803FA08F3134203D0D9F8000008F04E
:107FB8008AFC08F10108B8F1130F09F10409EDD1A1
:107FC80004F1280007F038FFB7F84031B4F92E0063
:107FD800C01A08F069FC2B68DB0408D5964BB4F886
:107FE80064001B88181AC0F30D0008F05DFC2B68AC
:107FF800980403D5B4F8660008F056FC2B685905B8
:1080080003D504F16C0007F017FF2B681A0502D599
:10801800A06E08F058FC2B681B0403D5B4F8720056
:1080280008F042FC04F13000A04607F005FF04F117
:10803800360007F001FFB7F8403138F93C0FC01A95
:1080480008F032FC01277D4B1B789F4208DA38F98B
:10805800020FB4F93C30C01A08F035FC0137F2E7DA
:108068002B68980505D5B4F95E00A0F2DC5008F03D
:108078002AFC326872487260B260121A9110714A12
:108088004A43531C032293FBF2F202EB42029A1A70
:10809800742303FB02033360C9E16B4B6B4A1B6813
:1080A80011688B4206D00AA9002041F8203D1360D0
:1080B800FFF7ECFE019B97F8F6171B8897F8F70770
:1080C8000B44013BB3FBF0F200FB12338B4280F010
:1080D8007981564C0120FFF741FEFFF759FD5020EA
:1080E8002668656808F048FBA268236810681B6862
:1080F800626803441068A3EB400008F0E4FB6A6878
:1081080073689B1A0293AA68B3689B1A0393EA6878
:10811800F36802A89B1A049307F09EFE2A69336944
:108128009B1A02936A6973699B1A0393B369AA69D4
:1081380002A89B1A049308F027FB06F11C0905F115
:108148001C0B1027A0463B4801210368B94019427F
:10815800824606D0D9F80000DBF80030C01A08F0D3
:10816800B2FB0137132F09F104090BF1040BEAD113
:1081780006F1260005F12601002331F9024F30F9F6
:10818800022F121B02AC44F823200133042BF4D134
:108198000322002702ABBF0053F82230FFB26BB1B5
:1081A80003F108010F2902D847F0010706E08033E0
:1081B800FF2B94BF47F0020747F0030712F1FF3285
:1081C800E8D2384608F0D8FA00240DF10809A34689
:1081D80007F00302022A10D0032A17D0012A4AD135
:1081E800BBF1000F41D0D9F8000000F00F00204388
:1081F80008F0C2FA4FF0000B3DE0BBF1000F0CD0C5
:10820800D9F80000C0F3031020432CE0BBF1000FA5
:108218001ED199F8010008F0AFFA99F8000008F0AB
:10822800ABFA28E0042E0020701200208C2C0020CD
:10823800002E0020F82D0020F42D0020482B0020CF
:10824800982C002035C2724F0C2E0020082E0020DA
:10825800D9F80000C0F30330204308F08DFAD9F8AC
:108268000000C0F3071008F087FAD9F8004024018D
:10827800E4B24FF0010B09F1040906AB99454FEA46
:108288009707A5D1BBF1010F02D1204608F074FA77
:10829800DAF8003013F480541FBFB6F86420B5F83C
:1082A8006410521A029218BF012499040AD50AAA26
:1082B80002EB8401B5F86600B6F86620121A41F898
:1082C800202C01345A0513D502AA02EB840E06F1BC
:1082D8006A0705F16A00002237F9021F30F902CF58
:1082E800CCEB01014EF822100132032AF4D10334F9
:1082F8001F0508D50AAA02EB8400A96EB26E521AAD
:1083080040F8202C013418040BD50AAB03EB840287
:10831800B5F87210B6F872305B1A42F8203C013496
:1083280000E0F4B1012C03D1029808F0CCFA18E06F
:10833800631E002002AA400052F82320C0B20AB1EE
:1083480040F0010013F1FF33F4D208F015FA0027CA
:1083580002AB53F8270008B108F0B5FA0137A74275
:10836800F6DB30200321FFF791FC36200321FFF7CD
:108378008DFC314B3C201978FFF788FCDAF8003087
:10838800990506D5B6F95E00B5F95E30C01A08F051
:108398009AFAD8F800202948D8F80430C8F80420F8
:1083A800121A9110264AC8F808304A43531C03226F
:1083B80093FBF2F202EB42029A1A742303FB0203C4
:1083C800C8F800301F4B1B681A0630D51E4C1F4DCD
:1083D80022682B689A420BD162686B689A4207D16F
:1083E800019B1B88102B11D1194B1B885B060DD1E3
:1083F800482008F0C1F9206808F065FA606808F0BC
:1084080062FA23682B6063686B600EE0114A0F4BB9
:1084180011782A7C914208D10F4A996810688842DD
:1084280003D15268DB689A4201D0FFF751FC08F08B
:1084380073F90BB0BDE8F08F482B0020982C002072
:1084480035C2724F741A0020EC110020782C0020DD
:10845800062E0020961A0020981A00202DE9F74FC2
:108468000E9F4D4CC2EB030B0D9BFF1A636800294E
:1084780014BF4FF006094FF004090133824616462F
:1084880034D123684B4580F08280444A019152F8E8
:108498002380009340460DF004FA0B3008F004F9ED
:1084A800009B0199054608B1012071E0032B98BF94
:1084B800514642463A4808F04DF93A4A1368181AA4
:1084C8006368106001336360374B9D710EE00D9A4D
:1084D80092B103FB07F20D99895C01228A40334966
:1084E80009680A4208D163680133636063680C9ABB
:1084F800294D9342EBDB32E003FB0BF5236806EBD7
:10850800050A2BB970590DF0CCF900F1050801E006
:108518004FF00308404608F0C7F80028C4D1214AA4
:10852800214B1068C8EB000010609A791AB12C2012
:1085380008F022F901E001229A71236843B97059C1
:1085480008F0F8F89AF904104B1CCCD0184803E04E
:108558009A4418489AF8041008F0FCF8C3E710D1B8
:10856800012008F0A1F860B90E4A13680A20013BFF
:10857800136008F001F92B6801332B604FF0FF33CB
:108588006B60206848452CBF0020012000E00020D7
:1085980003B0BDE8F08F00BF142E0020B0770108AB
:1085A80059970108102E0020F41C0020F82D0020F7
:1085B8006897010810A1010830B585B004AC002502
:1085C80024F8025D0091ADF8060021461020FFF75F
:1085D80021FC9DF806002146FFF71CFC9DF80700CA
:1085E8002146FFF717FC9DF800002146FFF712FC13
:1085F8009DF801002146FFF70DFC9DF80200214679
:10860800FFF708FC9DF803002146FFF703FC9DF8DF
:108618000E00C043C0B22946FFF7FCFB05B030BDD1
:1086280010B5054C206808F0DEFE18B1206808F087
:10863800D7FEF6E710BD00BF141B002013B5044693
:1086480001A9006809F07EFC132009F0B7FCBDF908
:10865800040009F0A1FC1B2009F0B0FCBDF90600DC
:1086680009F09AFC232009F0A9FC2368002BB4BF69
:1086780053204E2009F090FC01A9606809F062FCC3
:10868800122009F09BFCBDF9040009F085FC1A20B2
:1086980009F094FCBDF9060009F07EFC222009F0DF
:1086A8008DFC6368002BB4BF5720452009F074FC8B
:1086B80002B010BDF8B504460E4617460025204600
:1086C80020210DF0E0F80446D0B1013420460DF029
:1086D8003FF9B0F5617F05DB40F634039842A8BF47
:1086E800184601E04FF46170A0F56170192390FB02
:1086F800F3F00DB9307000E070703B7801333B70D7
:108708000DB90125DBE72046F8BD30B505460C4616
:108718001346294622460248BDE8304002F0A3BD70
:108728005C9801087FB504780646E4B9354B1B68A8
:1087380003EB8403192193F8870093F8886093F872
:10874800852093F886304FF4617511FB005011FBBA
:108758000651009001912C482146013402F083FD16
:10876800142CE3D14BE00DF0F3F81328054641DC57
:10877800244B701C1C68202100238DF80F300DF04D
:1087880082F82035064670B1013630460DF0E0F823
:108798001A289FBF04EB850358719DF80F300133E9
:1087A80098BF8DF80F30304620210DF06CF8064642
:1087B80070B1013630460DF0CBF80D289FBF04EBA1
:1087C800850398719DF80F30013398BF8DF80F30ED
:1087D80004EB85043046E11D0DF10F02FFF76AFF37
:1087E8009DF80F30042B0AD0601D002104220DF0E3
:1087F80014F804E0054800211322FFF786FF04B0AF
:1088080070BD00BFB81100207B980108909801083E
:10881800014808F07BBA00BF96980108F8B50478BB
:10882800064674B9304DB5F8C421B5F8C6312F489D
:108838002146013402F017FD042C05F10405F2D19C
:10884800F8BD2B490CF0F2FFA8B9274B4FF47A7109
:108858004FF4FA62A3F8C411A3F8C621A3F8C8110B
:10886800A3F8CA21A3F8CC11A3F8CE21A3F8D011FC
:10887800A3F8D221F8BD30460DF06AF80328054662
:108888002BD8304620210CF0FEFF044630B10134CD
:1088980020460DF05DF80126074600E00646204612
:1088A80020210CF0F0FF10B9BDE8F840B0E7013026
:1088B8000DF04EF8012EF7D1A7F2EE2240F2DC536C
:1088C8009A42F1D8A0F2EE229A42EDD8064B7035C2
:1088D80003EB85039F80D880F8BD0648002103225A
:1088E800BDE8F84011E700BF70120020A498010805
:1088F800B7980108BCA301082DE9FF410478054693
:10890800002C39D17348744D08F000FAD5ED047A7B
:10891800F5EE407AF1EE10FA00F0D88021466F4863
:1089280002F0A1FC95ED040A684602F031FB01460D
:108938006B4802F098FC95ED050A684602F028FBA2
:108948000146674802F08FFC95ED060A684602F07A
:108958001FFB0146624802F086FC95ED070A68464F
:1089680002F016FB013401465E4802F07CFC0C2C38
:1089780005F11005CAD1A9E05B4905220CF09AFF60
:1089880040B9554B03F1C002002143F8101F934230
:10899800FAD19BE02846554904220CF08BFF044687
:1089A8002846002C40D120210CF06DFF002800F053
:1089B8008D80451C28460CF074FF07464C4B53F835
:1089C80024601EB94B4808F0A1F97FE028463146DB
:1089D800FAB20CF06FFF01340028EFD13E4B03F1DF
:1089E800C0029E46002143F8101F9342FAD1424B21
:1089F80003EBC4029846D2F804C0BCF1000F04D1BE
:108A080031463E4802F02FFC57E0002718F8343072
:108A18009F42F5DA3B010EEB030563440FCB10359B
:108A280085E80F000137F1E70CF092FF0B280646A6
:108A380047DC284620210CF026FF054650B10135B9
:108A4800284602F01BFA244B03EB061383ED040AB5
:108A5800012400E00446284620210CF014FF0546B6
:108A680048B10135284602F009FA1B4B03EB0613FF
:108A780083ED050A0134284620210CF004FF054641
:108A880048B10135284602F0F9F9134B03EB0613F8
:108A980083ED060A0134284620210CF0F4FE10B9B3
:108AA800FFF7B6FE12E0013002F0E8F90A4B032C9A
:108AB80003EB061686ED070AF2D11148FFF71CFFF3
:108AC80004E0104801210C22FFF71FFE04B0BDE8A6
:108AD800F08100BFBD98010870120020D8980108E5
:108AE800DE980108F8A00108B7980108E298010883
:108AF80070910108E79801088C970108F698010819
:108B08001396010890980108F0B5047887B00646D6
:108B18001CBB514B1968062303FB0411192091F85B
:108B2800D65091F8D77091F8DA2091F8D5304FF4F3
:108B3800617610FB056510FB07600095019091F8C0
:108B4800D8000290D0314548497A03912146013432
:108B580002F089FB0C2CDCD17CE00CF0F9FE0B2830
:108B6800044672DC3C4B701C1D68202100238DF8E4
:108B780017300CF088FE064680B1013630460CF0FE
:108B8800E7FE03289FBF062303FB045383F8DA009C
:108B98009DF817309CBF01338DF8173030462021DF
:108BA8000CF071FE074680B1013738460CF0D0FE54
:108BB8000D289FBF062303FB045383F8D5009DF8B7
:108BC80017309CBF01338DF8173006266643A91964
:108BD8003846D6310DF11702FFF76CFD20210CF055
:108BE80052FE074670B1013738460CF0B1FE142822
:108BF8009FBF9DF817307619013386F8D80098BFC3
:108C08008DF81730384620210CF03DFE78B1013040
:108C18000CF09EFE0D289FBF062303FB045383F828
:108C2800D9009DF817309CBF01338DF817309DF897
:108C38001730062B0ED0062202FB04500021D53037
:108C48000CF0EBFDFFF7E4FD04E0054800210B22E2
:108C5800FFF75BFD07B0F0BDB811002002990108CD
:108C6800909801082DE9F347047807464CB9204647
:108C780001A907F09BF90134FFF7F4FF122CF6D194
:108C880079E00CF065FEC5B2112D6FD8781C202153
:108C98000CF0F9FD394C3A4F05F1D006034614F8AB
:108CA800168030B9A8F10202D2F1000848EB020898
:108CB80043E000F1010A597838460CF0E4FD60B150
:108CC800032D8CBF03230023C01B3B4453FA80F0C1
:108CD80090F80490B9F1030F02D1FFF799FD4AE02B
:108CE800A9F10203D3F1000850464FF0200148EBE8
:108CF80003080CF0C8FDD8B1B8F1000FEDD0013071
:108D08000CF026FE40F2ED2380B2984205DD40F6D5
:108D1800CA039842A8BF184601E040F2EE2004EBCF
:108D28004603A0F2EE20192290FBF2F0587002E000
:108D3800B8F1000FD1D104F8169014F81630FA5C87
:108D4800B8F1000F0DD00D4B0E4803EB460629462F
:108D5800737840F2EE24192505FB034302F083FAE9
:108D680009E02946084802F07EFA04E00748002195
:108D78001122FFF7CAFC02B0BDE8F087701200208C
:108D8800C87701082299010834990108BCA3010891
:108D980010B50446204608F01DFB18B90A2008F053
:108DA8004BFAF7E710BD002207490C2303FB021317
:108DB8005968814204D10022C2621A725A6070470F
:108DC8000132042AF0D17047882A00202DE9F04F9B
:108DD80087B0074602919DF8444011461A469DF80F
:108DE800403000250C20674E684300EB060E805784
:108DF800B842B14605D19EF808A0BAF1000F04D0D8
:108E0800BBE00135042DEDD1B7E0012F00F0A480BF
:108E180005DC002F40F0B18000945B48A1E0022FF0
:108E280000F09D80142F40F0A880584EB36943F09D
:108E38000103B36173694FF0904443F400337361E5
:108E480003224FF0010B4FF4805804A94FF09040D3
:108E58008DF815200392CDF810808DF814B08DF898
:108E680016B08DF817A001F053FEA4F82880C8208A
:108E780008F0E2F9C4F818807369039A43F40033E0
:108E8800736120464FF4C0538DF8152004A90222BF
:108E98008DF81420039204938DF816A08DF817A06E
:108EA80001F036FE636A23F470436362636A43F435
:108EB80060436362636A23F470236362636A43F402
:108EC80060236362324B334C4FF4802119601223C4
:108ED800A36404F14800082384F84D3084F84EB0A8
:108EE80008F0F6FE2C4B2D49C3F800A0F369039A4D
:108EF80043F40003F3612A4B04A8D9608DF810707D
:108F08008DF811208DF812A08DF813B008F096FE98
:108F18002A238DF810309DF813308DF811B08DF894
:108F280012A01BB104A808F089FE04E01D4B4FF401
:108F38008062C3F884201C4A1C4B136002221A72F8
:108F48001B4A1C4B13601C4A1C491B68116098473C
:108F58001B4B23600F4807E000941A4801E01A48A9
:108F6800009404F047FD40B10C2303FB05959DF8E0
:108F7800083007712B72686000E0002007B0BDE878
:108F8800F08F00BF882A00200038014000100240FE
:108F980014040140FC1C0020D80042420005FA05D8
:108FA80000ED00E000E100E07429002078290020AD
:108FB8009C280020A80000209828002014000020E9
:108FC800D4770108004400400048004010B5084B21
:108FD8001968002201EBC20393F90240844201D1CF
:108FE800981C10BD0132042AF4D1002010BD00BF26
:108FF800842A0020F0B5027887B08AB94A4C04F177
:10900800200694F8F42100234849595650B2814269
:109018006ED00C33302BF7D10834B442F1D181E053
:10902800002204920592451C0CF092FCC4B260B276
:10903800FFF7CCFF074618B18DF81040012400E077
:109048000446284620210CF01EFC054638B101359F
:1090580028460CF07DFC0134ADF81200E4B200267D
:10906800284620210CF00FFCB0B3451C28460CF014
:109078006FFC00222E4951F8223083425FFA82FEAB
:1090880004D00132082AF5D1002300E0734651F8D4
:109098002320824220D1022E0FD0032E12D05A1E36
:1090A800012ED2B204D0042A13D88DF814300EE061
:1090B800042A0ED88DF8153009E0052B09D88DF84B
:1090C800173004E09A1E052A03D88DF816300134AB
:1090D800E4B20136042EC3D1052C04D807B0BDE88C
:1090E800F040FFF795BB04AB03CB3860796019E01B
:1090F80094F8F9010E4B94F8F85153F82000B4F89D
:10910800F621009094F8FB0153F82000019094F8A0
:10911800FA0153F82000029053F82530054802F070
:10912800A2F879E707B0F0BD70120020882A002065
:10913800048101084399010838B1438811EA030002
:1091480003D08B420CBF01200220704730B50B4B77
:109158000B491C6891F85020032A0BD8134604EBDE
:10916800C303551CEAB29D882842F5D081F85020E7
:10917800981C30BD81F85020002030BD842A002082
:10918800FC1C0020024B002283F85020DEE700BFC1
:10919800FC1C00202DE9F047877890F803C0214D8A
:1091A800BBB2C7F1640E03EB83065C42C3F17800DF
:1091B8005FFA8EFE7600CCF16408A4B280B2A3B246
:1091C8000FFA83F9B9F1000F05DC002B14BFBA467A
:1091D8004FF0010A00E0F24613FB03F303FB0CF225
:1091E8001AFB0AF392FBF3F3434403FB09F30A2245
:1091F80093FBF2F333449BB225F8023FB1F8009099
:109208004A880A34C9EB020AA4B21AB202FB0AF26B
:109218004FF47A73844292FBF3F34B442B80CED104
:10922800BDE8F0874C1D002010B544780078002276
:1092380002FB02F3193B634303F6C413534340F69E
:10924800C411434393FBF1F3034921F8123001326F
:10925800072AEDD110BD00BF661D00200430114B58
:1092680033F91000B0F5617F10B506DB40F6330323
:1092780098420246A8BF1A4601E04FF461720C7882
:10928800192340F2833013FB0404944207DA497827
:1092980013FB01039342B4BF0020012010BD00203E
:1092A80010BD00BF202F002010B500F15003027838
:1092B8008A4203D18478C278944204D30430984215
:1092C800F5D1002010BD012010BD00BF38B5002425
:1092D8000B4D6059254407F019FD696811B109481B
:1092E80001F0C1FFA96811B1074801F0BCFF0748A8
:1092F800103407F00BFDB4F5D87FE9D138BD00BFB5
:10930800B87C01086299010868990108B6A10108AA
:10931800F0B585B004460CF0C4FA082826D1621EC0
:10932800E01D1F4912F8013F09681944497801F006
:109338000301022908BF203B82421370F1D1254660
:1093480004F1080715F8016B164831460CF09BFA32
:1093580020B1284631460CF096FA10B1FFF758FABA
:109368001CE0BD42EED1204606F002FE0E4807F092
:10937800CDFC00230D4A1A4404A992F888210A4416
:109388000849595C02F80C1C0133082BF2D1002360
:1093980007488DF80C3001A901F065FF05B0F0BD54
:1093A800080100204FA001086E99010870120020E2
:1093B800F8A00108234B244C1D68206880B5FFF7EE
:1093C800E7FC2846FFF7E4FC206841798B0704D4C2
:1093D800036841F002019B6998471C4B4FF4004217
:1093E8009A614FF480429A61206807F0FCFFA0B1AF
:1093F800164E4FF400433385134B186807F0F0FFFF
:109408000746FDF79BFE08B105F0A0FF2846394640
:1094180007F0ECFF4FF40043B361284607F0E3FF81
:109428000028E1D0094ED4F800804FF480473785F2
:10943800284607F0D5FF0146404607F0D7FFB76139
:10944800D2E700BFD42A0020741D0020000800487D
:109458002DE9F04705460CF024FA314E0446D6F8BB
:10946800088090B92F4807F051FC2F4B53F824106F
:1094780049B10123A34013EA080F02D02B4801F099
:10948800F2FE0134F1E72A4822E02846294922461B
:109498000CF010FA58B92848284C07F037FC54F853
:1094A800041F0029EFD0214801F0DDFEF7E72B78F3
:1094B8002D2B03BF013504F1FF344FF0010A4FF0A3
:1094C800000A4FF00009184B53F8297027B91C48B7
:1094D800BDE8F04707F01ABC2846394622460CF08A
:1094E800E9F9C8B9012000FA09F0830501D5154842
:1094F800EEE7BAF1000F03D001F0DEFF124803E0F7
:1095080040EA0800B060114807F000FC39461048EE
:10951800BDE8F04701F0A7BE09F10109D3E700BF94
:109528007012002074990108687E01087E9901086C
:10953800B6A101088299010887990108647E01088B
:10954800E798010893990108A1990108AA990108C7
:10955800F7A0010810B5084807F0D8FB074B00240E
:109568001C715C63064B1C7008F0CEF807F0B2FD66
:10957800044B1C6010BD00BFB2990108741D002087
:10958800A72F0020D42A002070B5064600240B4BD4
:10959800E518AA8816420AD0E158094801F063FE86
:1095A8002846002107F03FFB064807F0AFFB1434BC
:1095B80040F634539C42EAD170BD00BF3C84010898
:1095C800DE990108B6A10108F0B504788BB005460C
:1095D8000CB1002436E04B4B19680E2303FB041131
:1095E80001F59070B1F92951B1F92521B1F9273167
:1095F800009591F82C51019591F82D51029590F90B
:109608000B00039001F594713F4891F906100491FD
:109618002146013401F027FE082CDCD170E02D2B07
:1096280014D1072C1BDC28460CF092F90AAB661CF7
:1096380003EB440424F8100C15F8013F303B092BC8
:10964800FAD934462B78002BE9D104E0A3F1300293
:10965800092A09D8E5E7082CBDF8182009D00BB06D
:10966800BDE8F040FFF7D4B8202BF8D101352646E5
:10967800E7E7072AF3D8BDF81A00224BA0F2EE213B
:1096880089B240F2DC55A9421B68E8D8BDF81C1025
:10969800A1F2EE24A4B2AC42E1D8BDF81E6004B237
:1096A80037B2A742DBDB0DB2AF42D8DCA542D6DB2E
:1096B800BDF8247007F16404A4B2C82CCFD8BDF853
:1096C80026E00FFA8EF4112CC9DCBDF82050B42D19
:1096D800C5D8BDF82240B42CC1D812B24FF00E0C38
:1096E8000CFB0233A3F82501A3F82711A3F829617D
:1096F80083F82C5183F82D4183F82B7183F82EE1E0
:109708000BB0F0BDB8110020E8990108F0B5044687
:109718008FB020460CF0C5F8C5B225BBAF48B04C99
:1097280007F0F4FA94F8D21009B9AE4854E049B2F7
:1097380094F8D02094F8D130009194F8D310019186
:1097480094F9D410029194F9D510039194F8D61095
:109758000491A5482946013501F085FD102D04F135
:109768000704DFD1E1E72046A04905220CF0A2F862
:109778000546B8B929469E4870220CF04EF89D4B14
:10978800196828460E2303FB00130130002208281D
:1097980083F82F2183F8302183F8312183F832218F
:1097A800F0D119E12046944904220CF083F80546CB
:1097B8002046002D4AD120210CF065F8002800F041
:1097C8000B81461C30460CF06CF82C4607468B4B38
:1097D80053F824502DB98A480FB0BDE8F04001F085
:1097E80042BD30462946FAB20CF064F8013400282C
:1097F800EDD17B4A02F170011646002382F8D6307B
:1098080082F8D23082F8D13082F8D03007328A42DA
:10981800F3D17C4901EBC40191F80822934210DA94
:10982800D1F80C72C3EBC302B0183A4400F1D0016E
:109838001768C0F8D0709088888092798A7101334F
:10984800E7E72946704801F00EFD96E06F490722C8
:109858000CF030F805462046002D4AD120210CF0A6
:1098680012F806460CF01DF8C4B274BB684801F043
:10987800FAFC21466748013401F0F5FC0E2CF8D1BA
:10988800584801F0F0FC00246348214601F0EBFC45
:109898000025584A614811680E2202FB0412012370
:1098A800D2F82F215E49AB4013425E4B05F101050A
:1098B80008BF194601F0D7FC0E2DEAD149480134FA
:1098C80001F0D1FC082CDFD186E0304656490CF077
:1098D80043F82C46002852D0022C55D00CF038F80A
:1098E80006AB514943F8240000200CF035F8013448
:1098F800F0E74D490CF030F8002460B1082C3ED058
:109908000CF026F806AB484943F8240000200CF078
:1099180023F80134F1E7082C31D1069B0F2B2ED800
:10992800DDF81CE0BEF1070F29D8089F0D2F26D8B7
:10993800099E06F16402C82A21D80A9DFF2D1ED867
:109948000B9864281BD80C99642918D8884216DA11
:109958000D9C032C13D8224AC3EBC303134483F88A
:10996800D0E083F8D17083F8D26083F8D35083F8BD
:10997800D40083F8D51083F8D6402C4CC9E60FB034
:10998800BDE8F040FEF744BF069B072B20D8079997
:109998000D291DD80278722A0DD06E2A18D1154AC1
:1099A80012680E2000FB032301228A40D3F82F11EE
:1099B80021EA020209E00F4A12680E2000FB032385
:1099C80001228A40D3F82F110A43C3F82F2101E05E
:1099D800FEF71EFF0D4C9CE60FB0F0BD109A010873
:1099E80070120020B6A101083B9A0108B798010837
:1099F80040130020B8110020E29801087091010876
:109A0800E7980108B87C0108F6980108089A010847
:109A18006C990108579A010810A101085C9A01087D
:109A2800FFA40108B9A50108609A01081396010866
:109A38002DE9F743047805468CB9324D95F8A712FD
:109A4800B5F8A42295F8A6322F4800912146013492
:109A580001F009FC102C05F10405EFD14EE00BF0E4
:109A680077FF0F28044636DC284620210BF00BFF31
:109A7800264EE4B2D6F83880451CA40000272846B4
:109A88000BF066FF5FFA87F9B9F1010F83B208D0CE
:109A9800B9F1020F0BD0B3F5B47F24D2B26B1353D4
:109AA8000AE0FF2B1FD8B36B2344987004E0FF2B08
:109AB80019D8B36B2344D87028462C210BF0E3FE49
:109AC800054608B1013502E0B9F1020F0BD10137A3
:109AD800032FD4D112E00E4800210F2203B0BDE8B5
:109AE800F043FEF712BE08EB0400002104220BF03D
:109AF80094FE03B0BDE8F043FEF78ABE03B0BDE8AC
:109B0800F08300BF70120020629A0108741D0020C3
:109B1800909801082DE9F04304788FB00546002C91
:109B280059D17C4B0021142209A807AED3F83C80F8
:109B38000BF073FE0722304600210BF06EFE05A8DD
:109B48000023A700059308EB070583801A4672498E
:109B5800B5F802E031F813C01CEA0E0F0AD00DF177
:109B6800380C0E3102F1010E6244595C02F81C1CDB
:109B78005FFA8EF20133072BE9D100210B46674AC1
:109B8800B5F802E011F802C01CEA0E0F0AD00DF178
:109B9800380C063203F1010E63448A5C03F8242C66
:109BA8005FFA8EF301310629E9D118F807305C49CC
:109BB8008DE841006A78029209A81A0903F00F0398
:109BC80008F078F92146574809AA013401F04BFBFF
:109BD800202CA6D19BE00BF0BBFE1F28044600F307
:109BE800898028462021E4B20BF04DFE1F2C02D9B3
:109BF800FEF70EFE8BE0474BDB6B03EB8404451C42
:109C08000021204604220BF008FE0027464B09AE2F
:109C1800304600210A2217F803905FFA87F80BF004
:109C2800FCFD002315F8012B32B10A2B04D04A455C
:109C380002D0F2540133F5E74A4561D108F1FF3308
:109C4800032B09D8DFE803F0100502420DF12300C9
:109C580037E00DF123011FE030460BF079FE237841
:109C6800C0B243EA001006E030460BF071FE2378DC
:109C780000F00F001843207034E00133062B0BD09E
:109C88002A4800F2F3269E5D9642F6D1034493F8E3
:109C9800ED2263881343638011F8012F12B3002368
:109CA800EEE70133072B0CD0204A02F2E6269E5D30
:109CB8008E42F6D102EB4303B3F8D82263881343EC
:109CC800638010F8011F69B10023EDE730460BF0FF
:109CD8003FFE0F2804DC30460BF03AFE607001E0CE
:109CE800002363700137052F90D1012405F0D4FAC1
:109CF8006CB97DE70E4800211F22FEF706FD06E03D
:109D08002046002104220BF088FD0024EEE70FB066
:109D1800BDE8F083741D0020907F0108A57F01082D
:109D2800769A0108859A0108B17F0108B87C010874
:109D3800909801082DE9F0412DED048BB1498AB0C6
:109D480004460BF073FDB049002820460CBF0126DD
:109D580007260BF06BFDAD490028204608BF0226F8
:109D68000BF064FD002808BF0426F10740F1EF80DE
:109D7800A748A84C06F0CAFF002006F0D3FDA64865
:109D880006F0C4FFA54806F0C1FF6379A44AA548B8
:109D9800013B254652F8231001F065FAA24801F06C
:109DA80062FA4FF00008274695ED048AB5EE408A1E
:109DB800F1EE10FA04D19D4801F055FA002570E043
:109DC8009B48D5ED059A95ED069AD5ED078A41464B
:109DD80001F049FAB5EEC08AF1EE10FA02D520205A
:109DE80006F08CFFB0EE480A06A801F0D1F801464B
:109DF800904801F038FAF5EEC09AF1EE10FA02D563
:109E0800202006F07BFFB0EE690A06A801F0C0F832
:109E18000146884801F027FAB5EEC09AF1EE10FA2B
:109E280002D5202006F06AFFB0EE490A06A801F024
:109E3800AFF801467F4801F016FAF5EEC08AF1EE58
:109E480010FA02D5202006F059FFB0EE680A06A8DD
:109E580001F09EF808F101080146774801F003FA7D
:109E6800B8F10C0F05F110059ED1A4E749B294F89A
:109E7800D02094F8D130009194F8D310019194F93E
:109E8800D410029194F9D510039194F8D610049146
:109E98006A482946013501F0E6F9102D04F1070456
:109EA80003D094F8D2100029E0D16548654C06F03B
:109EB8002DFFD7F8088054F8041F19B1624801F043
:109EC800D2F9F8E70D46614B53F8254054B1012308
:109ED800AB4013EA080F03D05D48214601F0C3F9EF
:109EE8000135F0E75B4806F011FF21467B180AAA06
:109EF80093F888311344584A8A5C03F8102C0131CE
:109F08000829F3D1002306A954488DF8203001F020
:109F1800AAF9534806F0FAFE5248FFF76BF8524880
:109F280006F0F4FE4F48FFF7F5FD504806F0EEFE48
:109F38004C48FFF77DFD4E4801F095F94020FFF7AA
:109F480023FB4C4806F0E2FE4648FEF78BFEB207BC
:109F580039D5494806F0DAFE484806F0D7FE4148A8
:109F680006F020FD464806F0D1FE3E48FEF7DAFB33
:109F7800444806F0CBFE3B48FEF7C6FD424801F0D8
:109F880072F93848FEF74AFC404806F0BFFE3548EB
:109F9800FFF71AFB00270E257D4300243C4A126C6C
:109FA8002A440123D2F80A20A34013421ED10134C7
:109FB8000E2CF3D10137082FEDD12D4801F053F9BC
:109FC8008020FFF7E1FA730716D5324806F09EFEA7
:109FD800314806F09BFE234806F0BEFC244801F0F9
:109FE80042F94FF48070FFF7CFFA05E03946224670
:109FF8002A4801F038F9DAE70AB0BDEC048BBDE86D
:10A00800F08100BF919A0108A19E0108989A010861
:10A018009E9A010870120020AC9A0108BE9A0108A5
:10A0280070910108CA9A0108D59A0108E29A0108B4
:10A03800EF9A01086B990108F8A00108079B01082D
:10A04800F79A0108647E0108269B0108687E0108CA
:10A05800349B0108419B01084FA001084D9B010852
:10A06800569B010813960108659B0108719B01081E
:10A07800B6A101087F9B01088C9B01089F9B0108E2
:10A08800AD9B0108B79B0108C69B0108D49B01083A
:10A09800741D0020E09B0108F19B0108039C010846
:10A0A80010B5214A18B9136802221A8210BD1F4838
:10A0B800146800230380217811F07F0102460DD136
:10A0C800637A990644BF0221017013F0400F0378A8
:10A0D80014BF43F0010323F0010315E0012921D047
:10A0E80002291ED1637913F0800F03F00F034FEAA2
:10A0F800830303F1804303F5B8431B6806D003F0DC
:10A108003003102B07D10123137004E003F44053EC
:10A11800B3F5805FF6E7064B1B681B699847034851
:10A1280010BD184610BD00BF74290020B81D0020BE
:10A138009828002010B5064C18B9236801221A8205
:10A1480010BD044B1B689B68984720680C3010BDF5
:10A15800742900209828002010B5064C18B92368E7
:10A1680001221A8210BD044B1B681B68984720689F
:10A178000A3010BD742900209828002003788B42EB
:10A1880083BF034B03EB410148880020704700BFA1
:10A19800B81D002070B500221346244914180C4439
:10A1A800A47E83EA0423082413F4004F4FEA4303F0
:10A1B80018BF83F4815304F1FF3418BF83F00103FF
:10A1C80014F0FF049BB2EFD10132192AE5D100F156
:10A1D800190200F11A050A440D44967EAA7E02EB84
:10A1E800062292B29A421FD1104B93F83B50E2B22A
:10A1F800AA4216D2431C03EB4203DBB2CA1801334E
:10A208000B44927E9B7E03EB02239BB24FF4AF621A
:10A2180053431B13064A03F5487322F814300134DC
:10A22800E5E7012381F83C3070BD00BFB81D002070
:10A23800BA1D002003788B420BD9074B1A78074BBD
:10A2480089001944086C02B1400800F5777080B2A3
:10A2580070470020704700BF802A0020B81D0020EA
:10A2680007299DBF034B03EB8101B1F87000002063
:10A27800704700BFB81D0020034B03EB4101B1F844
:10A288009000C008704700BFB81D002070B5334C5F
:10A29800054606F0B5FFD4F8B030C4F8B000C31ACC
:10A2A800B3F5FA5FC4F8B43082BF002384F8B8303D
:10A2B80084F8B93094F8B8302BB9A12D02BF274AD9
:10A2C800012182F8B91094F8B910244A29B1D1189B
:10A2D800EDB201338D7682F8B83094F8B85094F81E
:10A2E800BA30AB4239D11D4B93F8BB30052B02D0A5
:10A2F800062B03D02CE00020FFF74CFFE37E1E2B3B
:10A3080026D100200246C1B26B1E994219DA2144B7
:10A318008B7E0821DBB283EA0206F60744BF83F08E
:10A328001803C3F3460301F1FF3154BF5B0843F040
:10A33800800311F0FF01C2F34702ECD101301A4645
:10A34800E1E723449B7E9A4202D10320FFF722FFD4
:10A35800002384F8B93084F8B83070BDB81D0020E7
:10A3680010B5044606F04CFF0F4BD3F8BC20C3F8D9
:10A37800BC00821A41F288318A42C3F8C02084BFE7
:10A38800002283F8C42093F8C420074913440F2AF5
:10A39800E4B218BF013283F8C54012BF81F8C42067
:10A3A800012381F8D53010BDB81D002010B5044632
:10A3B80006F026FF0F4BD3F8D820C3F8D800821A2E
:10A3C80041F288318A42C3F8DC2084BF002283F836
:10A3D800E02093F8E02007491344142A18BF0132FB
:10A3E80083F8E14012BF81F8E020012381F8F630BC
:10A3F80010BD00BFB81D00202DE9F843324F3D685D
:10A408002A8A2E7AB2B9042E14D1304C30482378D7
:10A41800012B0BD12F4B19682F4B89B20B445B00D2
:10A4280019681A6030230380227048E010230380E3
:10A43800072644E0AC8AAB69A24294BF04260226F0
:10A44800944228BF14461FFA84F840469847214A88
:10A4580013689BB203F1005303F540535B0004F10A
:10A46800010E1B689BB203F1005303F540534FEAFA
:10A478006E0E5B000021714500F1020009D010F852
:10A48800019C10F802CC4CEA092C23F821C00131B8
:10A49800F1E71268104B92B213445B001A681C6013
:10A4A8002B8AC8EB03032B826B8A9844084BA5F8C8
:10A4B800128030221A80094B4FF440521A803B68B0
:10A4C8001E72BDE8F88300BF74290020A92F002060
:10A4D80092280020505C0040023000209028002084
:10A4E8000E4B0F4A1B689BB203EBC00002443E2987
:10A4F8004FEA420209D94B09C80604BF03F1FF33EA
:10A508009BB29B0243F4004304E04B08C90748BFD1
:10A5180001339B0211681360704700BF505C004014
:10A528000630002010B5454B1A68107810F07F00EF
:10A5380004D1537A23F02003537210BD02287AD134
:10A548005388002B78D11379002B75D1537923F0D8
:10A558008000840004F1804101F5B84113F0800FB8
:10A56800096814BF01F0300101F44051032862D892
:10A57800002960D0927A002A5DD004F1804404F565
:10A58800B8441906226825D502F03002102A4CD1A9
:10A5980003F07F039B0003F1804303F5B8431A6877
:10A5A800510641BF196840F60F720A4042F4004252
:10A5B80044BF42F0C0021A601A6822F4E04222F056
:10A5C800400292B282F0300242F4004242F080022D
:10A5D8001A602AE002F44052B2F5805F25D128B90A
:10A5E800174B93F82C10FFF77BFF11E09B0003F14A
:10A5F800804303F5B8431A68520441BF196840F60E
:10A608000F720A4042F4404244BF42F080021A608E
:10A61800236823F4804323F070039BB283F44053F0
:10A6280043F4004343F080032360064B1B685B69D7
:10A638009847002010BD022010BD00BF74290020DB
:10A64800A80000209828002000230360436083604E
:10A658008381036143618361C361036243628362EF
:10A6680070478A68036810B50C6A14430A69144372
:10A678004A6914438A691443CA6914434A6A1443E9
:10A688008A6A23F4FF4323F07003224313430360D1
:10A698008B8943600B6883604B68C36010BD026898
:10A6A8004FF6FE731340036000230360436083602A
:10A6B800C360294B984201D1284A27E0284B984289
:10A6C80001D1264A2AE0274B984201D1234A2DE09E
:10A6D800254B984201D1214A30E0244B984201D1C0
:10A6E8001E4A33E0224B984204D11C4A536843F473
:10A6F80070032EE01F4B984204D1184A536843F068
:10A70800706326E01C4B984204D11C4A536843F0FE
:10A718000F031EE01A4B984204D1184A536843F0BD
:10A72800F00316E0174B984204D1144A536843F4D7
:10A7380070630EE0144B984204D1104A536843F4F6
:10A74800704306E0114B984204D10C4A536843F415
:10A7580070235360704700BF0800024000000240A9
:10A768001C000240300002404400024058000240F1
:10A778006C000240800002400804024000040240CD
:10A788001C040240300402404404024058040240C1
:10A79800084BDA68D10709D4DA68D20608D4DB682E
:10A7A80013F0040F14BF03200420704701207047E2
:10A7B8000220704700200240036A23F0010303626D
:10A7C800036A70B5446882690D6822F4803222F009
:10A7D800730215438A8923F0020313438A881343BB
:10A7E800134A90420FD002F5006290420BD002F556
:10A7F8004062904207D002F58062904203D002F591
:10A80800806290420DD1CA89CE8823F00803134391
:10A818000A8A24F4407414434A8A23F00403334315
:10A8280014438A68446085614263036270BD00BF57
:10A83800002C0140994A536803F00C03042B2DE9BE
:10A84800F04105D0082B06D095490160B3B916E050
:10A85800934B036012E053685468C3F38343991C15
:10A86800E30349BFD36A8F4B8D4C03F00F0344BFFA
:10A878000133B4FBF3F34B43036000E0002351685A
:10A88800894FC1F303117D5C0168EDB221FA05F42B
:10A8980044605668C6F30226BE5D24FA06FEC0F878
:10A8A80008E05668C6F3C226BE5DF6B2F440C4603E
:10A8B800D2F82C80C8F3041808F00F0C07EB4C0CE6
:10A8C80018F0100FBCF810C01FFA8CFC07D0BCF1B0
:10A8D800000F04D0B3FBFCFCC0F810C000E001611D
:10A8E800D2F82CC0CCF3442C0CF00F0807EB480727
:10A8F8001CF0100F3F8ABFB204D01FB1B3FBF7F7AB
:10A90800476100E04161176BFF065ABF644F8761DA
:10A918008161176BBF065ABF614FC761C161176B71
:10A928007F065ABF5E4F07620162176BFF0506D5A7
:10A93800994204D1AE4202D14F00476200E044621E
:10A94800176BFF0406D5994204D1AE4202D14F00DD
:10A95800876200E08462176BBF0506D5994204D16F
:10A96800AE4202D14F00C76200E0C462176B7F0598
:10A9780006D5994204D1AE4202D14F00476400E0A7
:10A988004464176B3F0506D5994204D1AE4202D103
:10A998004F00876400E08464176BBF0406D59942B2
:10A9A80004D1AE4202D14B00C36400E08464156B4D
:10A9B8003A4BAD0701D1046315E01C6B04F00304A6
:10A9C800012C01D101630EE01C6B04F00304022C7E
:10A9D80002D14FF4004305E01B6B03F00303032B84
:10A9E80001D12F4B0363146B2C4B14F4403F02D15D
:10A9F800C0F834E018E01C6B04F44034B4F5803F30
:10AA080001D1416310E01C6B04F44034B4F5003FFD
:10AA180002D14FF4004306E01B6B03F44033B3F557
:10AA2800403F01D11E4B4363146B1C4B14F4402F61
:10AA380002D1C0F838E018E01C6B04F44024B4F5E7
:10AA4800802F01D1816310E01C6B04F44024B4F51D
:10AA5800002F02D14FF4004306E01B6B03F44023A0
:10AA6800B3F5402F01D10E4B8363146B0B4B14F4D9
:10AA7800401F02D1C0F83CE020E01C6B04F44014F5
:10AA8800B4F5801F01D1C16318E01C6B04F44014B5
:10AA9800B4F5001F0AD14FF400430EE00010024045
:10AAA80000127A0000093D00380000201B6B03F4F7
:10AAB8004013B3F5401F01D1134BC363126B134B03
:10AAC80012F4400F03D1C0F840E0BDE8F0811A6BE2
:10AAD80002F44002B2F5800F02D10164BDE8F081B2
:10AAE8001A6B02F44002B2F5000F02D14FF4004392
:10AAF80006E01B6B03F44003B3F5400F01D1024B92
:10AB08000364BDE8F08100BF00127A000010024023
:10AB1800F0B500230E681C460125A54005EA060E7F
:10AB2800AE452BD10F797A1E012A15D885680322E4
:10AB38009A4025EA020282604D7982689D40154359
:10AB48008560828892B222EA0E0282808A7985889C
:10AB5800A2402A4392B28280032205689A40D243D7
:10AB68001540056005689F402F430760C768174078
:10AB7800CA7902FA03F547EA0502C2600134102CCB
:10AB880003F10203C8D1F0BD38B52DED048B4A4C52
:10AB98000368C4F8F8308388A4F8FC30023A0D46FC
:10ABA800062A05D8DFE802F00A101822292F3500F6
:10ABB800B4F8F8300B80B4F8FA3013E0B4F8FA308F
:10ABC8000B80B4F8F83005E0B4F8F8305B420B803D
:10ABD800B4F8FA305B4205E0B4F8FA305B420B8017
:10ABE800B4F8F8306B80B4F8FC301DE0B4F8F830F5
:10ABF8005B420B80B4F8FA3012E0B4F8FA300B80FC
:10AC0800B4F8F8300CE0B4F8F8300B80B4F8FA3047
:10AC180005E0B4F8FA305B420B80B4F8F8305B42D8
:10AC28006B80B4F8FC305B42AB80244B93F8303037
:10AC3800002B3ED1B5F9003094ED430AD4ED407AAB
:10AC480009EE103AB5F9023008EE103AB8EEC88AA3
:10AC5800B5F90430B8EEC99A28EE000A08EE903A21
:10AC6800A7EE890AF8EEE88AD4ED467AA7EEA80A94
:10AC78000AF0E2FF94ED440AD4ED417A288028EEE8
:10AC8800000AA7EE890AD4ED477AA7EEA80A0AF0C7
:10AC9800D3FF94ED450AD4ED427A688028EE000A85
:10ACA800A7EE890AD4ED487AA7EEA80A0AF0C4FFED
:10ACB800A880BDEC048B38BDB81D002038000020EA
:10ACC800094B1A68137844F6FB7103EB431300FB36
:10ACD80003135078C0EB0030B3FBF0F39078B3FB6C
:10ACE800F0F080B2704700BF781A002008B50A4813
:10ACF80090F8253100EB43030A22B3F8341189B2E6
:10AD0800A0F83C1100F5A07006F073FB80B2FFF7C5
:10AD1800D7FF024B188008BDB81D00207C1A002000
:10AD2800F0B50124B0FBF4F58D4201D34C43F9E7AB
:10AD38000026D4B1B0FBF4F504FB1500B4FBF1F424
:10AD48001EB9002D01DC002CF3D1092D03F1010EF1
:10AD5800EFB204DD002A14BF3725572500E030255F
:10AD68003D441D7001367346E3E71C70F0BDF0B535
:10AD78000124B0FBF4F58D4201D34C43F9E70026DA
:10AD8800D4B1B0FBF4F504FB1500B4FBF1F41EB923
:10AD9800002D01DC002CF3D1092D03F1010EEFB2D7
:10ADA80004DD002A14BF3725572500E030253D442F
:10ADB8001D7001367346E3E71C70F0BD03685A1C2A
:10ADC8000260197070472DE9F843089E002B07466A
:10ADD8008846144614BF4FF030094FF02009334617
:10ADE80013F8012B0AB9254603E0002CFBDD013CD2
:10ADF800F6E7002D04DD38464946C047013DF8E72F
:10AE080024EAE4743546A01B284415F8011B11B147
:10AE18003846C047F7E7BDE8F883024B186806F0E4
:10AE2800E5BA00BF6010002090ED017A07EE901A95
:10AE3800B5EE407AF1EE10FA01BFF8EEE77A9FED31
:10AE48000E7A67EE877AB7EE007A04BFC7EE277AE4
:10AE5800C0ED017A90ED017AD0ED007A30EE877A74
:10AE680030EE670AC0EE870AE0EE807AB0EE670A35
:10AE7800C0ED007A704700BFDB0FC94010B50278FB
:10AE8800202A034600F10100F9D0092AF7D02D2A1B
:10AE980003D10346BFEE000A04E02B2A08BF03468D
:10AEA800B7EE000ADFED387A1A46134612F8010B9E
:10AEB800A0F13001CCB2092C0AD807EE101AB8EE6E
:10AEC800C77AF2EE046AA7EEA67AF0EE477AECE7C4
:10AED8002E2816D1F2EE046A1146B0EE666A0B46C9
:10AEE80011F8012B303AD0B209280AD807EE102AF7
:10AEF800B8EEC77A87EE267A66EE866A77EE877AA4
:10AF0800EDE71A7802F0DF02452A35D15A782D2A62
:10AF180002D10233012004E02B2A14BF013302338B
:10AF28000020013B002213F8011F3039CCB2092C54
:10AF380003D80A2404FB0212F5E7B2F59A7F28BF6A
:10AF48004FF49A721346B7EE007A072B05D9DFED56
:10AF58000F6A083B27EE267AF7E702F007032BB1C2
:10AF6800F2EE046A27EE267A013BF8E7F0EE476A2C
:10AF780020B1C7EE877A03E0F7EE006A67EEA67A9B
:10AF880020EE270A10BD00BF0000000020BCBE4C08
:10AF980030B52DED028B87B0B0EE408A0C2200212F
:10AFA800054603A80AF039FCB5EEC08ADFED2A7A17
:10AFB800F1EE10FACCBF38EE278A38EE678ADFED5B
:10AFC800277A28EE278A6946FDEEC87A17EE904A56
:10AFD80084EAE470A0EBE47004F0E8FF002CACBF56
:10AFE80020232D2368468DF80C300AF05AFC0128DE
:10AFF80007D130238DF80D308DF80E308DF80F30D5
:10B008000CE0022805D130238DF80D308DF80E3074
:10B0180004E0032804BF30238DF80D30694603A8E7
:10B028000AF022FC03A80AF03CFC0338C4B222460A
:10B0380003A928460AF062FC00232B552846084934
:10B048000AF012FC03AB284619190AF00DFC284631
:10B0580007B0BDEC028B30BD6F12033A00007A4492
:10B0680012A0010870B5064615460846B6FBF2F46C
:10B0780014B12046FFF7F6FF05FB1464024B1B5D75
:10B0880000F8013B70BD00BF14A001082DE9F04F86
:10B09800814689B08A4616461C4600253178002923
:10B0A80000F0DD80252902D00136484675E0727827
:10B0B800302A08BFB278A2F1300319BFB71C4FF08D
:10B0C800000BF71C4FF0010B092B4FF0000819D8A3
:10B0D800A2F13003D9B2092905D80A2202FB08389F
:10B0E80017F8012BF4E7A2F16103052B02D8A2F1AE
:10B0F800570305E0A2F14103052B03D8A2F137035A
:10B108000A2BEADD6C2A31D13A78642A07F1010664
:10B1180000F083800BD8252A3DD003D8002A00F000
:10B128009E80BBE7582A0CD0632A19D0B6E7732A49
:10B1380022D002D86E2A37D0B0E7752A5CD0782A98
:10B14800ACD1271D2068A2F1580462424FF01001CB
:10B15800624155E02CD9582A32D0632A2AD13E467A
:10B1680048462178271DD04701350FE0642A64D06E
:10B178000ED9732A14D13E46236800934846514697
:10B1880042460023FFF71FFE271D05443C4685E77E
:10B19800252ADFD13E4648462521D04701357DE79F
:10B1A8000AD86E2A06D13E46236804341D6075E726
:10B1B800002A54D03E4671E7752A26D0782AF9D15C
:10B1C800A2F1580304F1040C5A422068CDF80CC0CF
:10B1D8004FF010015A4105ABFFF7A2FDDDF80CC096
:10B1E8003E46644605AB00934846514642465B4698
:10B1F800FFF7E9FD054451E72068271D0A210022D1
:10B2080005ABFFF7B4FD3C46ECE704F1040CCDF8C0
:10B218000CC020680A210022DDE72068002804F11C
:10B22800040708DA2D238DF8143040420DF1150378
:10B238000A210022E5E705ABFAE72068002804F1B7
:10B24800040C0ADA2D238DF8143040420DF1150351
:10B25800CDF80CC00A210022BEE705ABF8E7284666
:10B2680009B0BDE8F08F0FB413B50B4904AB0868FB
:10B278000A4953F8042B09680193FFF707FF0446AE
:10B28800074B186806F0A6F80028F9D0204602B047
:10B29800BDE8104004B070477C0100207801002010
:10B2A8006010002080EAE073A3EBE0738B4206DBBA
:10B2B800002801DD401A704702D00844704700207A
:10B2C8007047B0EEE06AF0EEC05AB4EEE56AF1EE0F
:10B2D80010FAD4BFF0EE656AF0EE466AF5EE406A01
:10B2E800F1EE10FA0BD0B4EEE56AF1EE10FA54BFA5
:10B2F800F0EE657AF0EE467AC7EEA66A01E0DFED79
:10B30800206ADFED207A9FED207A9FED205AA6EE85
:10B31800A77ADFED1F7AE7EE267A9FED1E7AA7EE71
:10B32800A67ADFED1D7AE7EE267AF4EEC65AB1EE7C
:10B33800677ADFED1A7AA6EEA75AF7EE007AE5EEFD
:10B34800267AF1EE10FAC7EE277AC8BF9FED147A75
:10B35800F5EEC00AC8BF77EE677AF1EE10FA48BF7B
:10B368009FED107AB5EEC00A48BF77EE677AF1EE26
:10B3780010FA48BFF1EE677AB0EE670A704700BF6F
:10B388000000000039094E3DE3B59EBE69A2163E95
:10B3980088FA16BE45FE7FBFA7DFA8B499FB243FF5
:10B3A800DB0FC93FDB0F4940FDEEC07A17EE903A3C
:10B3B8002033402B43D8DFED237AB4EEE70AF1EED1
:10B3C80010FA04DDDFED207A30EE670AF3E7DFEDEF
:10B3D8001F7AB4EEE70AF1EE10FA04D5DFED1A7A17
:10B3E80030EE270AF3E7DFED1A7AB4EEE70AF1EE5A
:10B3F80010FA04DD30EE670A37EEC00A0AE09FED66
:10B40800157AB4EEC70AF1EE10FA44BF30EE270AF7
:10B4180037EE400A60EE007ADFED0F6A9FED0F7A93
:10B42800A7EEA67ADFED0E6AE7EE876A9FED0D7A42
:10B43800A7EEA67A20EE276AA6EE070A70479FEDC8
:10B44800060A7047DB0F4940DB0FC940DB0F49C0D4
:10B45800DB0FC93FDB0FC9BF0000000092E741B90D
:10B468009730083C15A82ABEDFED027A30EE270A8D
:10B478009AE700BFDB0FC93F064B1A8822EA000093
:10B48800904210B518801C4602D0012005F038FF04
:10B49800208810BD541B0020064B1A881043904288
:10B4A80010B518801C4602D0012005F029FF20881D
:10B4B80010BD00BF541B0020024A936823EA000015
:10B4C800906070477012002008B5104B1A7800235E
:10B4D800D9B2914207D20E4951F8231009680020C9
:10B4E80008600133F4E7322005F0A6FE094B1B681B
:10B4F8005A0309D5084B9B685B0305D440F2DC501E
:10B50800BDE8084005F098BE08BD00BF482B0020E4
:10B51800182B0020741A0020701200202DE9F34126
:10B5280007F052F9454A6F23137040F6040353801D
:10B53800BE231371EF2382F80038002382F8013804
:10B5480019461646F25C0133514040F60402934214
:10B55800F8D13A4B83F80118394B1A69120604D509
:10B56800384A5A6002F188325A6004270020013FA5
:10B5780017F0FF074FD0324B334C3422DA6004F116
:10B588007848A8F57C38C8F30A0343B1002356F875
:10B598000880019304F0DAFC0428E8D116E004F0EE
:10B5A800D5FC0428E3D1264D2B6943F002032B6117
:10B5B8006C612B6943F040032B6104F0C7FC2B69D5
:10B5C800042823F002032B61E0D0D0E71C4D2B693F
:10B5D80043F001032B611FFA88F3238004F0B6FCC3
:10B5E80004280FD1A31C0193019B4FEA1848A3F824
:10B5F800008004F0ABFC2B69042823F001032B61C5
:10B6080005D0B4E72B6923F001032B61AFE70F4B9B
:10B6180004349C42B3D10A4A1369042843F08003D6
:10B62800136102D104F06CFD10B9052005F080FE0D
:10B6380007F0B4F802B0BDE8F08100BF7012002036
:10B64800002002402301674500F0030804F80308BE
:10B6580010B50E4C2068FDF7E7FD2068047A00223B
:10B6680002FB02F3193B634303F6C4135343192146
:10B6780093FBF1F3064921F812300132072AEFD182
:10B688000449BDE81040FDF785BD00BFE411002066
:10B6980030100020B01300202DE9F04104F030FDF7
:10B6A80010B9042005F044FEAE4CAF4D07F08CF8FD
:10B6B800AE4940F6040220460AF0A4F894F8D037C0
:10B6C800022B84BF002384F8D03794F8D0274FF496
:10B6D800D27101FB02F3E018234400F539702860A9
:10B6E80093F8440303F55073022801FB024284BF18
:10B6F8000020187192F844339D4A13700C2202FB03
:10B7080003439C4A03F2D2731360A36846F209020A
:10B718001A401AB9934A43F400539360A368D807B0
:10B7280003D54FF40050FFF7C7FEA368590409D5A5
:10B738000820FFF7C1FE4FF40050FFF7BDFE0120BF
:10B74800FFF7BAFEA3681A0706D54FF40050FFF7B3
:10B75800B3FE0120FFF7B0FEA3689B0402D540208A
:10B76800FFF7AAFE012284F8152294F8DE217D4B0A
:10B778002AB193F8E22112B1002283F8E2217E4B2C
:10B788007E4E1E604FF0000C674604EB0C03B3F8C6
:10B79800F6E14FEA5E0101F077314FEA9E0303F0CC
:10B7A8003333C1EB0E00C11A4FEADE0303F0113345
:10B7B800CB1A03EB23131EF0010803F00F324FF0EE
:10B7C800FF0392FBF3F3C3EB032318BF0137A2EB8C
:10B7D800030318BFFFB2012B0ADD022B40F0BF8024
:10B7E800B8F1000F00F0BB801EF0BC0F00F0B7806E
:10B7F8000CF1080CBCF1200FC7D1013F012F00F25A
:10B80800AE80FFF725FF302200215D485D4F0AF02A
:10B8180004F85D4BD5F800801F605C4B002108F1EF
:10B828008500C3F80080FDF73FFD594B80F001000B
:10B838001870584B07F128021A60574B07F1D402C9
:10B848001A6098F8000003F09DF82868534B00F53B
:10B85800CB721A60FCF714F8514B94F8D601DFED5F
:10B86800516A07F196021A6064214F4BC82211FBF6
:10B8780000225A6000229A60DA601A615A619A615D
:10B88800DA6183F8202083F82120484B07F12E0243
:10B898001A602B68464A93ED1B7A03F22511116052
:10B8A800444A03F295111160434A07F108011160F7
:10B8B800424A1760424A07F1A201116067EE266A00
:10B8C800404A07F1AC01B6EE007A116087EE267A9D
:10B8D8003D490E60B4F86411101D07EE901AB4F8D3
:10B8E8006611F8EE677AC2ED027A07EE901A93F8BD
:10B8F8006810117193F88410517194F8E111117462
:10B90800F8EE677AB3F82211C2ED037A07EE901ABF
:10B918002E49F8EEE77A0860536182ED077A9FEDC9
:10B928002C7AC7EE277A03F17001916129492A4AD6
:10B938000B602A499FED2A7A67EE877AC2ED007A72
:10B9480003F174020A60274903F21D130B60264BAA
:10B958001F60264BBDE8F0411A6006F01FBF04F0D7
:10B96800C9FA4EE770120020B811002000F0030851
:10B97800B82A0020E41100201C2F0020F813002012
:10B98800600F0020B0130020940F0020980F0020B3
:10B99800030000208827002060060020A40F002054
:10B9A800442E0020DB0F49404C2F0020F0270020B8
:10B9B800B41D002090090020EC2B0020F02B002063
:10B9C800A4080020801F00206809002068280020A3
:10B9D8000000614400080020A0080020F4070020AF
:10B9E8004C3D0F449008002098080020F4060020E1
:10B9F80008B5FFF793FDFFF74FFE0120BDE80840AB
:10BA080005F07EBC2DE9F74FA74C05F0F9FB266839
:10BA18006568A768861BF643451BC71BED43FF43B4
:10BA2800F60F8046ED0FFF0F2EB93FB9002D00F03D
:10BA38008682B9462CE04FF0000929E0B14627E09C
:10BA480003EB8A0BBBF802301A050ED413F4805F9F
:10BA58001DBF964A9BF801101268954A954B14BF72
:10BA680052F82120126843F82A20BBF80230D80582
:10BA780016D499050AD5904B1B7813F0040F0CBF08
:10BA88008E4A8F4A8B4B126843F82A2009F1010924
:10BA9800207B8C495FFA89FA82450B68D0D326E06F
:10BAA800894A5046594603F087FB884B1B885A063B
:10BAB80003D550465946864A16E0580703D55046DE
:10BAC8005946844A10E0190703D550465946824A18
:10BAD8000AE09A0703D550465946804A04E0DB0736
:10BAE800D4D57F4A5046594603F066FBCEE7DFF8C7
:10BAF80008E20093BEF906307822A3F57A7353431F
:10BB08004FF47A7293FBF2F303F22B1301930022A2
:10BB1800F3465FFA82FE864517D2009B03EB820E3E
:10BB2800BEF802E01EF4806F0DD0DFF88891019B0B
:10BB380039F822E040F2671A9E449EFBFAFC0AFBA1
:10BB48001CEE29F822E00132E3E74DB308F5C333D0
:10BB5800A0336360637B544A13BB9373614B1B68C8
:10BB680013F0020F0AD0DFF894E19EF800E0BEF16E
:10BB7800000F03D04FF0010E82F80EE0DA0506D56B
:10BB8800594BDB781BB1A37B43F00203A3734A4BE9
:10BB98001B7813F0050F02BFA37B43F00403A373C4
:10BBA80094F80EE0BEF1000F03D13F4B5B7B002BF6
:10BBB8004FD094F80DC01CF0010FACF10C031DD14F
:10BBC800BCF1030F07D8DFF8E8903C4A1EF0040FD9
:10BBD80008BF4A4600E0364AACF1040CBCF1070F36
:10BBE80005D8DFF81CC11EF0010F18BF6246DBB292
:10BBF800032B0ED81EF0020F3C4B06E0DBB2032BE2
:10BC080006D82F4B2A4A1EF0020F18BF1A4600E02A
:10BC1800274A4FF0000C5FFA8CF383420DD20B6871
:10BC280003EB8C035B881B0642BF224BD2F80090C3
:10BC380043F82C900CF1010CEDE785B1BEF1000F33
:10BC480008D0637B184A0133DBB2142B06D10023DA
:10BC580004E025B1637B002BF3D100E05373002E81
:10BC680052D0234AB2F90250B2F90020002DB8BFD1
:10BC78006D42002A4FF03203B8BF524295FBF3F5EC
:10BC880092FBF3F2EDB2D3B2AB4238BF2B46194A5E
:10BC980013B192FBF3F300E0134643442360E37BC4
:10BCA800014A7BBB01232EE0A01F0020AC1D002011
:10BCB800E8920108DA0D0020A62F002088820108EA
:10BCC80078820108B01D002074800108541B0020F0
:10BCD8007A80010880800108868001088C8001082C
:10BCE80092800108741A00204C2F002090820108CD
:10BCF80068120020400D0300202F0020DC1A0020CD
:10BD0800988201080023D3738E4D8F4B2D78E27BE8
:10BD1800ADB9002F00F00E818C4B267B1A788C4B26
:10BD28008C4D93F800C08C4BD3F800E00B6802F000
:10BD380004020021D2B203EB86060F46B5E01AB919
:10BD4800864A1A61002508E0854AFAE70A68AB00C6
:10BD5800D6187688760604D40135EBB28342F5D33B
:10BD6800D7E7804EB6F90060192E25DD12F803E0FA
:10BD780094F814C026690EF00F09E1450CDCDFF8D1
:10BD8800C8C19CF815C0BCEB1E1FDEBFDFF8D8E1A8
:10BD9800D6F800C043F80EC012F803E094F816C0B5
:10BDA8000EF00F09E14533DBDFF89CC19CF815C0A4
:10BDB800BCEB1E1F2CDC26E0193629DA12F803E04A
:10BDC80094F814C026690EF00F09E1450CDCDFF881
:10BDD80078C19CF817C0BCEB1E1FA2BFDFF888E132
:10BDE800D6F800C043F80EC012F803E094F816C065
:10BDF8000EF00F09E1450BDBDFF84CC19CF817C0CA
:10BE0800BCEB1E1F04DBD6F800E0574E43F806E0F3
:10BE1800544EB6F90260192E1BDD12F803C094F8CF
:10BE280014E026690CF00F09F1450CDCDFF81891D5
:10BE380099F81590B9EB1C1FDEBFDFF82CC1D6F8B6
:10BE4800009043F80C90D25C02F00F0CF4451EDD14
:10BE580082E7193680DA12F803C094F816E02669EA
:10BE68000CF00F09F1450CDBDFF8DC9099F8159020
:10BE7800B9EB1C1FDEBFDFF8F0C0D6F8009043F81E
:10BE88000C90D25C02F00F0CF445FFF665AF94F805
:10BE980017E0BEEB121FA2BF334A36689E505BE71D
:10BEA8005888000504D404330435B342F8D122E09D
:10BEB8004AB101EB0C0A06209AFBF0F900FB19A025
:10BEC80001280DDC01E057B9012793F801900EEB2A
:10BED80089003EF829A090F80290C07803E0174640
:10BEE800002081468246013125F802AC85F8009091
:10BEF8006870C9B2D7E7164A1378013B13F0FF03FD
:10BF080008BF06231370114B1B785B0741BFBBF9B1
:10BF18000630A3F57A7303EBC3034FF47A7243BF79
:10BF280093FBF2F30133DBB20123104A92FBF3F3E4
:10BF38004344A36003B0BDE8F04FF8F747BF03B030
:10BF4800BDE8F08F880E0020A01F0020A62F00203B
:10BF58006A000020DC0D0020AC1D0020948201083E
:10BF6800E892010868120020DA0D0020400D030055
:10BF78002DE9F04F2DED0A8B85B08346029390F89A
:10BF88005030019100925BB1322BA8BF322307EEEB
:10BF9800903AB8EEE7BADFEDD77A87EE8BBA01E0D0
:10BFA8009FEDD5BAD54BDFEDD6BA1B88D54C002B03
:10BFB80008BF012307EE903AB8EEE79A238869EEA6
:10BFC8002BBA98073BEE2BBA8BEE8BBA27D5CE4A05
:10BFD800B2F90030B2F9022083EAE37182EAE27032
:10BFE800A1EBE371A0EBE27088420546B8BF0D46AD
:10BFF800B5F5E17F16DA8842DFEDC4AA05DD002A2F
:10C00800D8BF524207EE902A04E0002BD8BF5B420B
:10C0180007EE903AF8EEE77AC7EEAAAA04E0DFED59
:10C02800BCAA01E0F7EE00AADFEDB99AB94AD946F1
:10C038004FF0000AB0EE69AAB748268830F81A50BF
:10C04800B1482BB207EE903AF8EEE77AB5EE047AEB
:10C0580067EE877A30F91A309FEDB07AFDEEE77A0D
:10C0680006EE903AF8EEE77AB1075FFA8AF74FEAF8
:10C078004A0867EE877AF8EEE66A79D0A84830F978
:10C088001A3007EE103AB8EEC77AB0EE006AA6EE9C
:10C09800867A009BC3F1000EBDEEC77A17EE100A30
:10C0A800704503DB8342A8BF03469E469D48029B1A
:10C0B80038F900009FED9C5AC0EB0E0E33F91A00B8
:10C0C8009BF81C30704407EE100A0AEE103A9BF8F1
:10C0D8000830B8EEC76A07EE103AB8EE477AB8EEFD
:10C0E8004AAA26EE077AF1EE045A27EE057A6AEE96
:10C0F800255ABDEEC77A17EE100AB1EE657ABDEE85
:10C10800C7AA1AEE103A984208DBBDEEE5AA1AEE65
:10C11800103A8342A8BF03460AEE103A834800EB60
:10C128008A0090ED007AA6EE2B7ABBEE0E6AB4EE8A
:10C13800C67AF1EE10FAB8EECAAA09D4B3EE0E6ABE
:10C14800B4EE467AF1EE10FAC8BFB0EE467A01E0D6
:10C15800B0EE467A80ED007A9BF8123009EE903AFC
:10C16800F8EE699A27EE297ADFED719A67EE299A37
:10C17800F30751D42DB2002DB8BF6D42B5F5206F2D
:10C1880002DD0020106026E09FED6A6A99F8013010
:10C1980026EE867A06EE103AB8EE466A87EE066A0A
:10C1A80092ED007A36EE676AA6EE2B7A9FED626A08
:10C1B800B4EEC67AF1EE10FA09D49FED606AB4EED7
:10C1C800467AF1EE10FAC8BFB0EE467A01E0B0EE5A
:10C1D800467A82ED007A99F80B3092ED007A08EEF3
:10C1E800103AB8EE488AB00728EE077A9FED548ACD
:10C1F80027EE088A14D576EECA6AB0EE4A7AAAEE15
:10C20800A67A38EE698AF0EE476AB0EE697AAAEE45
:10C21800887AB0EE478A03E0B0EE698AF0EE4A6A9F
:10C2280048489FED496A1AF80030039207EE103A21
:10C23800B8EEC77A4FEA8A0627EE677A051D3544B5
:10C24800E7EE066A95ED007AC5ED007A37EEC77A13
:10C2580000F10C0587EE2B7A354414301AF80030BB
:10C26800D5ED007A37EE677A08EE903AEBEE077A6A
:10C27800F8EEE88AC5ED007A67EEA87ADFED338A32
:10C28800334D67EEA88A36EE880AB0EE66CA30EEFD
:10C29800680A09F0D1FC25F808002088039A10F4F0
:10C2A800006F07D02B480078410703D53846FBF7C5
:10C2B8006FFB039A284B294FFDEECC6AFDEEC87A36
:10C2C800F1EE688A16EE901A17EE900AFDEEE88AEB
:10C2D800F150F05118EE901A214803903150043271
:10C2E80009F101099846BAF1000F3DD14FF0010A52
:10C2F800A2E600BF83F9223EAF4C593C70110020E2
:10C30800BD378635541B0020681200200000E14329
:10C3180000000000B81F00209C110020CDCC4C402C
:10C328009E2F0020D41100206F12033CC41F002050
:10C338000AD7A33D0000A043000040C300004043CB
:10C348000AD7233CCC1F0020A69B443BF7CC92384D
:10C3580044270020A62F00204C2700205827002023
:10C368006427002000803B45BDEEC99A5FED037A43
:10C378009BF85320914E9249DFF8649219EE103AD7
:10C3880023F0030309EE103A019BB8EEC99A9B7992
:10C3980089EE279AB5EE000A002A6DD0B6F9042076
:10C3A8009BF80300002AB8BF52425A43854B92FBC0
:10C3B800F3F364336422434393FBF2F308EE903AB9
:10C3C800B1F9043007EE903AF8EEE77AF8EEE88A29
:10C3D80027EE800A09F030FC07EE900AF8EEE77ABB
:10C3E800B6F9043067EEA88ADFED777AC8EEA78A37
:10C3F80080EAE072A2EBE072B2F5207F07EE903A95
:10C40800F8EEE77A77EEE88A05DC83EAE372A2EBD6
:10C41800E372642A03DD0023C9F80830A3E003EBC4
:10C4280083031A019BF8033092FBF3F31B1A07EE00
:10C43800903AF8EEE77AD9F8083067EE897AFDEE97
:10C44800E77A17EE902A1A441346B2F57A5F5F4AE4
:10C45800A8BF4FF47A539342B8BF1346C9F80830BF
:10C468007D2293FBF2F39BF80D2053439B1107EEBB
:10C47800903AB8EEE78A76E0B6F904A000925B003D
:10C48800283303FB0AFAB1F9043007EE903AF8EEC4
:10C49800E77A4FEA6A1A27EE800A09F0CDFBBAF16B
:10C4A800000FC0EB0A0007EE900AB8BFCAF1000AF5
:10C4B800BAF1320FB8EEE77A03DD009AC9F808201E
:10C4C8001BE09BF80D3007EE903AF8EE677AD9F842
:10C4D800083067EE277A67EE897AFDEEE77A17EE7D
:10C4E800902A13443A4A9342A8BF1346394A9342C2
:10C4F800ACBFC9F80830C9F80820D9F808305B1370
:10C50800B3F5807FA8BF4FF480736FF0FF029342AA
:10C51800B8BF134607EE903AB8EEE78AFDEEC77A41
:10C528009BF8032017EE903A53439B1107EE903A7D
:10C53800294B1B78032BF8EEE78A14D9BBF84E2059
:10C54800B2F5FA7F0FD2FDEEE87A534217EE901A51
:10C55800994204DB914217EE903AA8BF134607EEC2
:10C56800903AF8EEE78A78EE887AFDEEE77ACDED34
:10C57800007ABDF80030AB801BB200EE103AB8EE7E
:10C58800C00A09F059FB2388A8801A0506D5134B61
:10C598001B785B0702D50220FBF7FAF9FDEEE88A63
:10C5A800BDEEC88A039AC8ED028A002387ED028A85
:10C5B800936005B0BDEC0A8BBDE8F08F68120020CF
:10C5C8009C1100200CFEFFFF0000A04280C1FFFF6D
:10C5D800FEFFFF0F020000F0482B0020A62F0020CE
:10C5E800142700202DE9F04F87B000260593BE4B95
:10C5F8000491B3F90270B3F900300292002FB8BF6A
:10C608007F42002BB8BF5B429F42B8BF1F46B7F5B9
:10C61800FA7F8046A8BF4FF4FA770090B346019698
:10C62800B2463446B14B198811F0030246D0AE4BDE
:10C63800AF4D33F8143035F914504FF0020E13FB98
:10C648000E53029DC5F1000C63454FEA440003DB1D
:10C658009D42A8BF1D46AC46A64BC55E059B33F957
:10C668001430C5EB0C0C0CEB030598F8083064206B
:10C678006B4393FBF0F398F81C006FF0040A0AFB75
:10C6880000FA534504DB00EB800A9A45A8BF9A4696
:10C69800994850F824302B4442F21075AB42A8BF99
:10C6A8002B46964DAB42B8BF2B4640F8243098F83D
:10C6B800120043431B13012A019338D08A4B904838
:10C6C80033F914B0009B50F824E093F801C08D4B67
:10C6D80033F9145085EAE573A3EBE573B3F5206FDE
:10C6E8004FEA840616DC0BEB8B031A0192FBFCF372
:10C6F800042295FBF2F55D1BAE44BEF57A5FA8BF38
:10C708004FF47A5E804B9E45ACBF40F824E040F879
:10C71800243002E0002340F8243083597D2693FB1F
:10C72800F6F6009BDB7A7343402693FBF6F6880700
:10C7380011D50198C7F5FA7307FB0BF907FB06F546
:10C748004FF4FA7103FB0A9903FB005599FBF1F2C8
:10C7580095FBF1F505E0C9074DBF019D35465A46E1
:10C768005246630069490393664B605C33F814E0F2
:10C7780020310FFA8EF34FF0040C93FBFCF909FB00
:10C7880000F06FF04F0990FBF9F9914431F914204A
:10C7980021F814E098F850109B1A93FBFCF379B138
:10C7A80007EE903A5A485B4BB8EEE70AD3ED000A19
:10C7B80000EBC400FEF738FBFDEEC07A17EE903AA6
:10C7C800554A564912F804C0039803EB430309EB92
:10C7D80005020CFB03F34FF0200C93FBFCF3D21A79
:10C7E8004252424A1288120508D54D4A127850071B
:10C7F80004D520460393FBF7CBF8039B494A4A49E3
:10C808004A4841F824905B4242F82430009B40F8A3
:10C818002450013300930D4681460CB9012401E7E9
:10C82800314B3748B3F90410049B86689B790F3362
:10C838005B004B435B113349002B4FF00404B1F903
:10C84800041091FBF4F1A3EB0101B8BF5B42322B5A
:10C8580098F80D400BDC364B04FB0164A342A8BFDB
:10C868002346344CA342ACBF8360846001E00023BC
:10C878008360314B98F803401B784C43032B4FEAF5
:10C88800A4140CD9B8F84E30B3F5FA7F07D2594240
:10C898008C4203DB9C42A8BF1C4600E00C4686681D
:10C8A80046F34F36B6F5807F6FF0FF03A8BF4FF40D
:10C8B80080769E42B8BF1E46184BA11999800B4B33
:10C8C8001B88190508D5164B1B785B0704D5022071
:10C8D8000092FBF75DF8009AAC600023C9F8086085
:10C8E800936007B0BDE8F08F68120020541B002049
:10C8F8009E2F0020D4110020E41F0020F0D8FFFF55
:10C90800142700209C11002080C1FFFFCC1F0020AD
:10C918002C27002010270020E01F0020442700209B
:10C92800A62F0020642700204C270020582700202D
:10C93800FEFFFF0F020000F0482B00202DE9F04F0A
:10C9480087B080460493AC4B03911C88029204F094
:10C958000204A4B294B1A94BB3F90240B3F9003070
:10C96800002CB8BF6442002BB8BF5B429C42B8BFE2
:10C978001C46B4F5007FA8BF4FF40074C3460025D9
:10C988009E4B33F815E09E4B33F815300193BDF9F3
:10C9980004009C4B80EAE077A7EBE0770FFA8EFC67
:10C9A8000421B7F5206F90FBF1F189B24FEA450AEF
:10C9B8004FEA4C0C0AB24FEA850953F825600FDCA0
:10C9C800C2EB0C021644B6F57A5FA8BF4FF47A564C
:10C9D8008D4A9642ACBF43F8256043F8252002E013
:10C9E800002243F8252053F80970834A9BF80B303E
:10C9F8001288FF115F439BF80130960703FB0CF385
:10CA08004FEAA7174FEAA31344D0804A32F90A2005
:10CA180002261EFB062E029A5242964503DB029A14
:10CA28007245A8BF72467A4EDFF818E23AF90660F6
:10CA3800961B049A32F91520164459F80E2042F232
:10CA4800107C32446245A8BF6246DFF8FCC16245EB
:10CA5800B8BF624649F80E2098F808E00EFB06F6C3
:10CA680098F81CE00EEB8E0EF611CEF1000C664520
:10CA780003DB7645A8BF7646B44698F81260724341
:10CA88001213BF1ACCEB03036743634302EB672718
:10CA98000CEB63235F4A565D243211FB06F6A3EBC9
:10CAA800A6163AF9023098F85010C01A042390FBE1
:10CAB800F3F0BDF804302AF8023079B107EE900A95
:10CAC800554B5648D3ED000AB8EEE70A00EBC5000F
:10CAD800FEF7AAF9FDEEC07A17EE900A504B514ABC
:10CAE8005B5D00EB400058434311F119C91A2AF85D
:10CAF80002104149088810F4006F8A460AD04A4952
:10CB08000978490706D5284605920193FAF740FFA8
:10CB1800059A019B4548464949F80060454E49F841
:10CB280001705B4249F806300BF1010B0746894654
:10CB38000DB9012524E7314B98F80D00B3F904101D
:10CB4800039B9B790F335B004B435B112C49002BF4
:10CB5800B1F904104FF0040591FBF5F52949A3EB51
:10CB68000505B8BF5B42322B8C680BDC324B00FBEF
:10CB780005408342A8BF034630488342ACBF8B6060
:10CB8800886001E000238B6098F803305D432C4BEC
:10CB98001B78032B4FEAA5150CD9B8F84E30B3F51E
:10CBA800FA7F07D25842854203DB9D42A8BF1D4643
:10CBB80000E005468C6844F34F34B4F5807F6FF08D
:10CBC800FF03A8BF4FF480749C42B8BF1C462B19C2
:10CBD8009380BAF800301A0506D5134B1B785B070B
:10CBE80002D50220FAF7D4FE0023BD60C9F8084038
:10CBF800B36007B0BDE8F08F541B00206812002016
:10CC08009C1100201427002080C1FFFF9E2F0020C8
:10CC1800D4110020CC1F0020102700202C27002032
:10CC2800E01F002044270020A62F00204C270020CA
:10CC38005827002064270020FEFFFF0F020000F0A5
:10CC4800482B0020E41F0020F0D8FFFF2DE9F04F0B
:10CC58002DED028B85B000260293A74B0192B3F904
:10CC68000270B3F900300090002FB8BF7F42002B4C
:10CC7800B8BF5B429F42B8BF1F46B7F5FA7F8346ED
:10CC8800A8BF4FF4FA77B046B146B24634469B4B3C
:10CC98001B8813F003004BD0022C49D0964A9849C0
:10CCA80032F8142031F914104FF0020E12FB0E1155
:10CCB800019A524291424FEA440503DB019A8A42A3
:10CCC800A8BF0A468F4935F9019002999BF81C5074
:10CCD80031F91410C9EB020202EB01099BF80810A4
:10CCE80001FB09F2642192FBF1F16FF0040202FBEF
:10CCF80005FA514505DB05EB85029142A8BF1146AF
:10CD08008A46814D814A55F8241042F2107E4944E2
:10CD18007145A8BF714691429BF81290B8BF114661
:10CD280009FB01F9012845F824104FEA293942D0B6
:10CD3800774D714935F91450009A764831F91480C5
:10CD480092F801E050F8242085EAE576A6EBE5762E
:10CD5800B6F5206F4FEA840120DC022C18D008EBCE
:10CD68008800000190FBFEFE042095FBF0F5C5EB62
:10CD78000E0E02EB0E0CBCF57A5F6648664DA8BF36
:10CD88004FF47A5CAC45ACBF41F800C00D5007E0E9
:10CD980088EAE876A6EBE876642EE0DD00254550C3
:10CDA8005C48009A09587D2691FBF6F6D17A7143C2
:10CDB800402691FBF6F69D0712D5022C10D0C7F538
:10CDC800FA7307FB06F507FB08F103FB0A114FF49A
:10CDD800FA7003FB095391FBF0F193FBF0F508E0BF
:10CDE800D80704D5022C02D04D46514601E03546FD
:10CDF8004146474B33F91400042390FBF3F34748AB
:10CE0800205C022C03FB00F36FF04F0093FBF0F360
:10CE18000B444FEA440C08EE103A0ED1404B4148FF
:10CE2800D3ED000ACDF80CC0B8EEC80A1E21FDF7F4
:10CE3800FBFFDDF80CC0BDEEC08A354B3A493CF823
:10CE480003003CF901302CF801009BF850100FFA50
:10CE580080FEC3EB0E034FF0040E93FBFEF399B173
:10CE680007EE903A31482E4BCDF80CC0B8EEE70AE1
:10CE7800D3ED000A00EBC400FDF7D6FFFDEEC07A43
:10CE8800DDF80CC017EE903A29492A4811F804E059
:10CE980018EE102A03EB430351190EFB03F34FF06E
:10CEA800200E93FBFEF3C91A2CF8001013490988C9
:10CEB800090508D5204909784A0704D5E0B2039343
:10CEC800FAF766FD039B1D4918EE102A41F8242045
:10CED8001B4941F824501B495B4241F82430009B10
:10CEE80001340133032C00937FF4D1AE05B0BDECBF
:10CEF800028BBDE8F08F00BF68120020541B002091
:10CF08009E2F0020D4110020E41F0020F0D8FFFF3E
:10CF18009C1100201427002080C1FFFFCC1F002097
:10CF28001027002008270020F41F00202C270020AD
:10CF3800E01F002044270020A62F00204C270020B7
:10CF480058270020642700206C4B6D4A2DE9F04FCC
:10CF58005E8914684FEA062AB4EB0A0A9C884FEAED
:10CF680004481C894FF000054FF0000B65EB0B0BD4
:10CF7800A4FB0A6704FB0B77F40944EA476418EB3F
:10CF880004065C884FF000094FEAE7154FEAC438F9
:10CF9800DC8849EB050787B0CDE90467A4FB0A677D
:10CFA80004FB0B77340A44EA076418EB04064FEADB
:10CFB80027259C894FF0000949EB0507CDE9006753
:10CFC800AAFB046704FB0B77F40D44EA472414F525
:10CFD800FA664FEAE75545F10007B6F5FA6F77F1BB
:10CFE8000003CDE90267964667DAA4FB046704FBF1
:10CFF80005F34FF0050C07EB4307DDE90489A6FBB1
:10D008000C230CFB07335F104FEA3206B8EB060817
:10D018004FEA920669EB070946EA83769F10DDE935
:10D028000023921B63EB0703DDE90267CDE90023C8
:10D03800344A4FF0FF33964277EB0303CDE9048976
:10D0480028DA40F6AC52A4184FF000035D4104FB07
:10D0580005F3A4FB044505EB43056FF006026642A1
:10D0680002FB0566A4FB0223334418EB020649EBD6
:10D078000307CDE904670B26A4FB062306FB05334B
:10D08800DDE900455B104FEA3202A41A65EB03059F
:10D09800CDE900450AFB0BF3DDE90245AAFB0AAB23
:10D0A8000BEB430B4FEADA7242EA4B02A41A4FEA3F
:10D0B800EB7365EB0305CDE90245DEF80440009B00
:10D0C800019DA4FB032304FB05334FEA52584FEAA2
:10D0D800635948EAC328DDE90423B8EB020269EB87
:10D0E80003039946D30B43EA494300B1036009B1EE
:10D0F800029B0B6007B0BDE8F08F00BFFE02002066
:10D10800FC1F002024FAFFFF054B1A7A02F0FF01EA
:10D1180022B10122027000221A7270470170704712
:10D12800FC1F002037B5104B04465D6818780621AF
:10D138006A46A847A8B19DF800209DF8013043EA47
:10D14800022323809DF802209DF8033043EA02233E
:10D1580063809DF804209DF8053043EA0223A380EC
:10D16800012003B030BD00BFEC02002013B5104B06
:10D1780004465B683B2006216A469847A8B19DF89B
:10D1880000209DF8013043EA022323809DF8022005
:10D198009DF8033043EA022363809DF804209DF83C
:10D1A800053043EA0223A380012002B010BD00BF6E
:10D1B800EC020020094B0A491B681B6923F01F0079
:10D1C80010B50122445803F01F0302FA03F31C426E
:10D1D8001EBF4350034B1A7210BD00BFF802002057
:10D1E80014040140FC1F0020772048210122F8F791
:10D1F8005DB8772058210122F8F758B803460A4647
:10D2080068201946F8F752B81FB5044602210C20C9
:10D2180001220DF10703F7F7CDFF08B900203BE025
:10D228009DF80730DB07F9D50321062202AB0C2055
:10D23800F7F7C0FF0C20092101220DF10703F7F7CA
:10D24800B9FF0028EAD09DF8073013F00C0FE5D19C
:10D258009DF809209DF8083043EA0223C3EB833385
:10D268009B009DF80B2023809DF80A3043EA022397
:10D27800C3EB83339B009DF80D2063809DF80C3031
:10D2880043EA0223C3EB83339B00A3800C200A21CB
:10D298000122F8F70BF8012004B010BD07B50021F2
:10D2A80001AB03227720F7F785FF9DF805309DF83D
:10D2B80004001B0243EA00439DF80600184303B02C
:10D2C8005DF804FB08B5FFF7E9FF014B586008BD9E
:10D2D800FC1F002008B5FFF7E1FF014B186008BDEF
:10D2E800FC1F002030B505460C4613462946224649
:10D2F8006820BDE83040F7F75DBF07B50A21002276
:10D308000C20F7F7D3FF142003F096FF0A210F2211
:10D318000C20F7F7CBFF0A2003F08EFF01AB10219A
:10D3280003220C20F7F746FF0A2003F085FF0A21A5
:10D3380000220C20F7F7BAFF0A2003F07DFF0DF159
:10D348000303022101220C20F7F734FF0DF1030338
:10D35800092101220C20F7F72DFF0A2101220C20B8
:10D36800F7F7A4FF03B05DF804FB70B54FF09044E5
:10D3780010250E46258504F039FC304604F036FCAD
:10D38800A561012070BD38B54FF0904314461022B6
:10D398001A8540F080000D4604F028FC174B2946FA
:10D3A8009B894FF47A7319B3144A1289950706D4E6
:10D3B800013B9BB24FF6FF729342F5D10CE0104A45
:10D3C800FF2010700D480089C0070BD4013B9BB2A9
:10D3D8004FF6FF708342F5D10A4A138801339BB296
:10D3E800138005E012780CB1227001340139DAE7B4
:10D3F8004FF0904310229A61012038BD003001405F
:10D408000C300140202E0020F0B5394D6B7A85B0E4
:10D41800002B6AD1374C2368002B66D01A68364E29
:10D4280012B171690A4372619A88ADF8002002222C
:10D4380098688DF80320694600228DF80220F7F7D6
:10D44800A3FDB369226843F00103B361137D167B22
:10D4580003F0030103F0FC0303F1804303F5803379
:10D4680089009F680F20884027EA00009860986824
:10D4780006FA01F1014399609368188A9388184065
:10D488002CD11E4B527D596859B303F051FF2268C5
:10D498001369012623F01F0103F01F0306FA03F0A6
:10D4A800174BC8501369029308230DEB030000279C
:10D4B8008DF80D308DF80C708DF80E6004F008FCB6
:10D4C80023688DF806705B7D8DF8043001A803236E
:10D4D8008DF805308DF8076004F0B0FB01236B72FE
:10D4E80003E0084959601A70D1E705B0F0BD00BFE4
:10D4F800FC1F0020F802002000100240FC2A002037
:10D5080014040140BDD1000870B50446FFF77CFF44
:10D51800FFF77AFFB4F5807F0ED0BB2C0ED8612CB4
:10D528000ED8292C0ED8132C0ED8092C0ED8002C66
:10D5380014BF062500250AE0002508E0012506E0BD
:10D54800022504E0032502E0042500E005251A4C25
:10D558008021A3686B209847642003F06DFEA368C0
:10D56800072168209847642003F066FEA36800211D
:10D578006B209847642003F05FFEA36801216B20AD
:10D588009847A36818211B209847A36810211C20DE
:10D598009847A36829461A209847084AA36811782B
:10D5A80019209847A368122137209847A368382084
:10D5B8000121BDE870401847EC0200200E0300204E
:10D5C80008B5FFF721FF024B4FF480521A8008BDBF
:10D5D800040000202DE9F0410369C76805460E469E
:10D5E8001F40002F35D0B7FA87F24FF00043D340E1
:10D5F800DB432B611F40A2F11B03042BF1D8DFE8AA
:10D6080003F0221F1C190300746A24B1013C002393
:10D61800A4B2736201E0EC6AA4B2D6F82080B8F133
:10D62800000FDED0D8F80030404621469847D8F899
:10D638000480F4E73068696B07E07068A96B04E060
:10D64800B068E96B01E0F068296C036889B2984713
:10D65800C7E7BDE8F08101480149BBE70040014048
:10D66800C42B002001480249B4E700BF0004004071
:10D678009C2B00204FF080400049ABE7742B002022
:10D6880001480249A6E700BF002C01404C2B0020AE
:10D69800014802499EE700BF002C01404C2B0020A6
:10D6A800224B10B5224C5A43224BB3FBF2F20388AB
:10D6B8000139013AA04289B292B29BB20ED004F568
:10D6C8000064A0420AD0B0F1804F07D0A4F5983486
:10D6D800A04203D004F58064A04202D123F0700375
:10D6E8009BB2154CA04206D004F58064A0421CBF32
:10D6F80023F440739BB203800D4BC16298420285AC
:10D708000FD003F5006398420BD003F540639842AD
:10D7180007D003F58063984203D003F580639842ED
:10D7280001D1002303860123436110BD40420F004D
:10D73800002C014000A24A04001000400B4B800A54
:10D7480098420DD004D8B0F5801F0BD10120704746
:10D75800074B984208D00533984203D103207047FD
:10D7680002207047FE20704700207047010010001B
:10D778004B001000F8B50468064620460F461546CB
:10D78800FFF7DCFF03284BD8B27A910847B9022388
:10D798008B40D4F80CE0DB439BB203EA0E03E36052
:10D7A8000A23204A03FB001342F82370043342F88B
:10D7B800235015463FB1B17AE268890802238B40AD
:10D7C8009BB21343E360282202FB00522032EFF39E
:10D7D8001286502383F3128803B203EB8303DB0022
:10D7E80003F10C011C3329442B4451F8047F17B171
:10D7F80017600A6804329942F7D100231360F3B224
:10D8080083F31188282303FB0050036A1BB1E368E4
:10D8180043F0010303E0E2684FF6FE731340E36050
:10D82800F8BD00BF4C2B0020014800F08BB800BFAA
:10D8380008200020014800F085B800BF5C200020C7
:10D84800014800F07FB800BFB0200020026BC1681B
:10D85800034610B5406942B11A6C8C1A013A005D52
:10D8680008BF0A46C0B21A6410BD1A6A805C013249
:10D878008A4228BF0022C0B21A6210BD436B13B19E
:10D8880090F844007047836A406A1B1A584258410E
:10D898007047426A816A03698A4238BFD218521AAD
:10D8A800416B21B149680A44591E8A4203D2013B9F
:10D8B800981AC0B2704700207047036B13B15B68B9
:10D8C800016C01E0C369016A8B423CBFC2689B18C6
:10D8D800581AC0B27047836A8169426B1944D16093
:10D8E800416A99429DBF0169CB1A5360CB1A96BF12
:10D8F8000023536083624FF0000380F844301368BC
:10D9080088BF816243F0010313607047436A8269EC
:10D91800D154436A02690133934228BF002343620A
:10D92800436B1BB11B68DB0705D4D4E7026D136892
:10D9380043F08003136070474171F7F7E5B88160E1
:10D94800F7F7E2B8026D036B70B50446D5699BB969
:10D95800A90611D5C36A1BB1908C80B298470BE019
:10D96800E169928C40694E1CD2B2E6614254E16989
:10D97800E268914228BFE361616BA1B92A0612D51A
:10D98800636AA26A9A42236D09D0501CA669A062F4
:10D99800B25C1A852369984205D3A16203E01A682C
:10D9A80022F080021A602B0742BF236D08221A62F8
:10D9B80070BD0D4B0D484FF400525A600C4A116867
:10D9C8004FF6FE730B401360426B11684FF6FE73FF
:10D9D8000B401360426A836A9A4200D07BE70123B6
:10D9E80080F84430704700BF00000240B02000209B
:10D9F800440002402DE9F0471E46A24B8CB09842E5
:10DA0800894690469DF850507ED19F4B9F4A1A6098
:10DA18009F4A5A6102F580729A614FF48072DA6007
:10DA28001A619C4A1A63143A5A63A2F54842203A8A
:10DA3800DA6404329A64C3F808801865964B9A69C8
:10DA480042F480429A615A6942F001025A61022303
:10DA58008DF80830032315F0010A8DF809304FF0CE
:10DA680000038DF80A3014BF022301232C078DF818
:10DA78000B3017D5894C102701978AF001038DF8D0
:10DA88000A30236A23F470232362236A43F4E023D1
:10DA98002362204601A9FDF73BF8BAF1000F23D114
:10DAA800A76121E0B0070ED50CA9102341F82C3D41
:10DAB8007A48036A23F470230362036A43F4E02379
:10DAC8000362FDF725F8F1070ED50CA9202341F8CC
:10DAD8002C3D7248036A23F470030362036A43F41B
:10DAE800E0030362FDF714F80E238DF800300022DE
:10DAF800012368468DF801308DF802208DF8033037
:10DB0800614C04F09BF80CE1654B984276D1654B6B
:10DB18005E4A1A604FF48072DA601A61624A5A618A
:10DB280002F580729A615C4AC3F808801865D36967
:10DB380043F40033D36102238DF80830032315F032
:10DB4800010A8DF809304FF000038DF80A3014BF30
:10DB5800022301232A078DF80B3019D54FF0904482
:10DB68004FF4804701978AF001038DF80A30636A01
:10DB780023F070636362636A43F0E0636362204684
:10DB880001A9FCF7C5FFBAF1000F27D1A76125E06D
:10DB9800B30710D50CA94FF4804341F82C3D4FF042
:10DBA8009040436A23F070634362436A43F0E06342
:10DBB8004362FCF7ADFFF70710D50CA94FF40043FB
:10DBC80041F82C3D4FF09040436A23F07043436284
:10DBD800436A43F0E0434362FCF79AFF26238DF83B
:10DBE80000300022012368468DF801308DF80220AC
:10DBF8008DF803302B4C04F021F892E02B4B98421F
:10DC080040F010812A4B214A1A604FF48072DA6082
:10DC18001A61284A5A6102F580729A611E4AC3F84D
:10DC280008801865D36943F48023D36102238DF8F3
:10DC38000830032315F0010A8DF809304FF000036E
:10DC48008DF80A3014BF022301232C078DF80B30FE
:10DC580034D5194C4FF4806701978AF001038DF889
:10DC68000A30636A23F470636362636A43F4E063AF
:10DC78006362204601A9FCF74BFFBAF1000F41D1BE
:10DC8800A7613FE000380140B020002098800108DB
:10DC980004210020580002400010024000080048FB
:10DCA800004400405C20002004230020004800407D
:10DCB800082000200425002000040048B0070FD5E4
:10DCC8000CA94FF4806341F82C3D5848436A23F46B
:10DCD80070634362436A43F4E0634362FCF718FFEE
:10DCE800F1070FD50CA94FF4006341F82C3D4F48BC
:10DCF800436A23F470434362436A43F4E043436254
:10DD0800FCF706FF27238DF8003000220123684620
:10DD18008DF801308DF802208DF8033003F08EFF66
:10DD2800434CC4F82C900027012384F84430276220
:10DD3800E761A76267626671C4F80880A57120462A
:10DD4800F6F7E2FEF20734D5236B002B2AD001A8A0
:10DD5800FCF77AFCE36C01934FF480530A93802319
:10DD68000693E368ADF8103020230993206B6369AC
:10DD780002930B970597079708970397FCF78FFC73
:10DD880001A9206BFCF76DFC236B216D1A6842F02A
:10DD980001021A608A6842F040028A605B689BB29E
:10DDA800236406E0236D20221A621A6842F02002DA
:10DDB8001A60B3072FD5636B43B301A8FCF744FC83
:10DDC800A36C01934FF480530A938023069323692D
:10DDD800ADF8103000251023606B03930B95059563
:10DDE800079508950995FCF75AFC606B01A9FCF7A3
:10DDF80038FC636B1A6842F002021A60226D5D609B
:10DE08005D60936843F08003936004E0226D1368BB
:10DE180043F080031360226D136843F0010313601D
:10DE2800204600E000200CB0BDE8F0870004004860
:10DE3800082000202DE9F04F2DED028B85B081469A
:10DE480003938A4B02921B889D0737D5109B8848FD
:10DE5800DC89B0F900301B1B03F2F31540F2E632FF
:10DE6800954203D8002BB8BF5B4201E04FF4FA7328
:10DE7800B0F90220121B02F2F31440F2E630844299
:10DE880003D8002AB8BF524201E04FF4FA72934215
:10DE9800B8BF1346C3F5FA73052293FBF2F30A22BF
:10DEA800643B534399F81C20D2105343642293FBDC
:10DEB800F2F3134423EAE373DBB200E06423009334
:10DEC800CB1C0193C8460025019B6A4813F8011F23
:10DED8000193022D4FEA450A06D1B0F9040001F179
:10DEE8001B044443631131E030F81530624830F9BF
:10DEF8001500022413FB04001AB2029B5B429842ED
:10DF080003DB029B8342A8BF03465C4830F90A4002
:10DF1800039830F915001B1B1844544B1E88F4074E
:10DF280010D41B3151430B11B1070FD599F812408A
:10DF38009DF9001044434C43642294FBF2F203EB36
:10DF4800221303E099F8083043431B114C4A042478
:10DF580032F90A2092FBF4F41C1B4A4B98F8012072
:10DF6800EF5C62437A436421022D92FBF1F24FEA9F
:10DF7800E21208EE102A09D1B8EEC80A181D1E21AF
:10DF8800D3ED030AFCF750FFBDEEC08A3D4A3E4B75
:10DF980098F80B601B8802F1100E03FB04F05EF882
:10DFA8002510C01206FB0016B6F5001F3749A8BF9A
:10DFB8004FF4001602F11C008E42B8BF0E4650F80E
:10DFC800251040F82540611A1B094FF6FF70B0FB79
:10DFD800F3F34B4399F850104EF825604FEA850B40
:10DFE80076139B1179B107EE903A02F12800B8EE4A
:10DFF800E70A00EBC500D2ED030AFCF715FFFDEEBA
:10E00800C07A17EE903A98F81510214A03EB4303AB
:10E018004B435F43642397FBF3F718EE103A3F1224
:10E0280033443B4422F80A30104B1B881A0506D5A6
:10E03800184B1B785B0702D5E8B2F9F7A9FC164B19
:10E0480018EE102A01354BF8032003F10C0218339F
:10E05800032D4BF802604BF8037008F101087FF4B8
:10E0680033AF05B0BDEC028BBDE8F08F541B002028
:10E07800202F0020681200209E2F0020D41100209D
:10E088009C11002004270020E01100200000E0FF80
:10E0980044270020A62F00204C2700202DE9F04F10
:10E0A8002DED0A8B97B011F0FD0806460191A94C99
:10E0B80006D0A94B1B689A0700F1B08000F041BC5C
:10E0C800236FA648DFF8949298470028F1D0A44F10
:10E0D80094F8802048464946FCF756FD3B8804F1F1
:10E0E800D002002B70D0D4F884301B7808EE103A98
:10E0F80004F1880A04F19405B7F800B039F918005A
:10E10800BBF57A7F02BF0023CAF800302B61DAF82A
:10E1180000300344CAF800302B6907EE900A013337
:10E12800012B4FEA4801F8EEE77A2B6106D100236C
:10E13800C5ED017AC5ED007AAB601BE0D5ED006A4C
:10E1480007EE103A37EEE66AB8EEC77A86EE077A37
:10E1580036EE877AD5ED026A85ED017A77EEC77AD1
:10E1680085ED007AE6EE276AF0EE667AC5ED036A79
:10E17800C5ED026A0023BBF1010F29F801305352A3
:10E188002DD12B690392012BC3BF03F1FF3300EE9E
:10E19800103AD5ED037A9FED730A0291C4BFB8EE29
:10E1A800C00A87EE800A07F091FF0299039A18EED9
:10E1B800103A5BB1F8EEC87AB4EEE70AF1EE10FA5D
:10E1C80004DD4FF47A733B8000231CE0DAF800305A
:10E1D8004FF47A7003F5FA7393FBF0F3535208F196
:10E1E8000108B8F1030F0AF1040A05F1140583D1F7
:10E1F800BBF1010F04D15846029203F051F8029A7C
:10E208003B88013BDFE739F8131032F81300091A8D
:10E2180029F813100133032BF5D14AE7019B002B92
:10E2280000F08F8394F8D6704A4D6FB1012F40F0FB
:10E23800808305F59070D5ED466A95ED477A05F52A
:10E2480096730021804613E102F0DAFFD5F8E0303A
:10E258009FED457AC5F8D800C31A07EE903AF8EE54
:10E26800677A424BC5F8E00067EE877A5B68C5EDD0
:10E27800377A05F1E400984705F1E408002800F032
:10E28800F1803B4B40461A784146FCF77DFCB5F8D7
:10E29800EA30002B42D0D5F8EC103B46B4F8EA201F
:10E2A80038F913702B4DB2F5C87F324A04BF0020ED
:10E2B80042F823004FEA830E52F80E00384442F821
:10E2C8000E00002028F8130021F813000133032B57
:10E2D800E4D1B5F8EA30012B1BD1D5F8F0304FF472
:10E2E800C87703F1C80292FBF7F20A80D5F8F42048
:10E2F800C83292FBF7F24A801F4AD5F8F8301288E4
:10E30800C83393FBF7F39B1A8B8030807080FDF73E
:10E318006FFBB4F8EA30013BA4F8EA30174B1B68EE
:10E328005B0740F18B80B4F8FC200A4B322A27D1D6
:10E33800D3F8EC201188A3F8FE1051889288A3F82E
:10E3480002213288A3F804217288A3F80011A3F8E7
:10E35800062117E0042700208C1A00209C110020B9
:10E36800A22F002000000000BD378635D82A0020E3
:10E37800A82F0020F427002004000020741A002091
:10E38800002A3BD0D4F8EC000023B4F8FC2038F97C
:10E3980013E0C54D322AC54A04BF002142F82310B4
:10E3A8009F00D1597144D151002228F8132020F838
:10E3B80013200133032B1146E7D1B5F8FC30012BAC
:10E3C80017D10C2085F8142185F8153102F068FF63
:10E3D800D5F8EC30B5F8FE201A80B5F800215A803F
:10E3E800B5F802219A80B5F804313380B5F80631C2
:10E3F8007380B4F8FC30013BA4F8FC3094F8163173
:10E40800A94ADBB1D2F8EC00D2F80831002182F831
:10E418001611322593FBF5F30380D2F80C3193FBE8
:10E42800F5F34380D2F81031A14A93FBF5F3128833
:10E438009B1A838031807180FDF7DAFAD4F8EC20DA
:10E44800B4F8E43011885B1AA4F8E4305188B4F8C1
:10E45800E6305B1AA4F8E6309288B4F8E8309B1AE4
:10E46800A4F8E83094F8D630013384F8D630D9E6E9
:10E478008D4D904F05F1E40232F8112027F8112054
:10E4880012B207EE902A8C4AF8EEE77A32F9112098
:10E4980067EEA67A0131E0EC017A07EE902AF8EEF1
:10E4A800E77A032967EE877AE3EC017AE0D105F58C
:10E4B800967005F59C71024603F0A3F905F5967070
:10E4C80005F5A27104AA03F09CF904A895ED370A92
:10E4D800DFF8D4A1014603F0ADF9DDED054ADDED25
:10E4E800047A9DED065A95ED574AD5ED563A95EDC5
:10E4F800543AB6EE007A64EE874A67EE875A64EEBD
:10E50800A47A25EE075AE5EEA57A07A80146B7EEE4
:10E51800008AE5EE057A0AAA0DAFF0EE482AE7EE82
:10E52800C72A0AF5B67965EE846AD5ED557AE2EE22
:10E53800A36A25EE236AE4EE836A23EEE57AB1EE58
:10E54800452AE2EE276AA2EEA76AA4EEA77A67EE4A
:10E55800E57AF1EE641AE2EE837AA1EE846AA2EE1D
:10E56800847AE1EEA37AA5EE836AA5EE037AE2EE59
:10E57800047A85ED556AC5ED547AB1EE466AC5ED63
:10E58800566A85ED577AF1EE666AB1EE477A8DEDF7
:10E59800097A8DED076ACDED086A03F032F995ED39
:10E5A800540A464810A903F045F907A8434913AA95
:10E5B80003F008F913A810A93A4603F022F90AA8AB
:10E5C800394613AA03F0FEF83A463C4813A903F06B
:10E5D80018F93B4BD5ED587A9DED0F7A1A78B4EEC1
:10E5E800E77AF1EE10FACCBF42F0080222F00802F6
:10E5F8001A70D4F864311B78F0EE489A0AF5BE75A3
:10E608003BB3DAED5A8A4846B0EE680A10A903F01F
:10E6180011F99AED5E8A0AF59070B0EE480A13A9CE
:10E6280003F008F94A4610A813A903F0EAF82846A7
:10E63800B0EE680A10A903F0FDF8384613A9B0EE49
:10E64800480A03F0F7F810A813A92A4603F0D9F8E6
:10E6580007E098E8070089E8070097E8070085E8D9
:10E668000700D4ED497AD4ED486A94ED4A7A0E4D04
:10E6780067EEA77A0023E6EEA67AE7EE077A9FED23
:10E68800117AF4EEC77AF1EE10FA06DC9FED0E7AF5
:10E69800F4EEC77AF1EE10FA1AD5C4F84431C4F88A
:10E6A8004831C4F84C3126E0042700200C2800200B
:10E6B80004000020521200209C110020BC80010898
:10E6C800901A0020B81E8D3F3D0A673F6F12833AAB
:10E6D80005F5B67005F5BE7105F5A27203F072F87E
:10E6E800D5ED377A1FED070A05F5A27080EE270AE7
:10E6F800014603F09FF8B4F88831984D01339BB276
:10E70800B3F57A7FA4F888312ED195ED550AD5ED69
:10E71800546A95ED567AD5ED577A20EE000AA6EEA2
:10E72800A60AA7EE070AA7EEA70A07F0CFFC89EE0C
:10E73800800A0023A5F88831D5ED556A95ED567AFB
:10E74800D5ED577A95ED546A60EE266A20EE077A81
:10E7580060EE277A26EE000AC5ED556A85ED540A63
:10E7680085ED567AC5ED577AD4ED558A94ED57AABA
:10E7780094ED54BAD4ED56AA9FED799A68EECA7A08
:10E78800B7EE007AEBEE2A7A77EEA77AF4EEE97A1A
:10E79800F1EE10FA0EDCFFEE006AF4EEE67AF1EE26
:10E7A80010FA24D4F4EE477AF1EE10FAC8BFF0EE6E
:10E7B800477A01E0F0EE477A17EE900A04F0C0F9C4
:10E7C80041EC100B07F07EFA51EC100B04F00CFA38
:10E7D80008EE100AB5EEC08AF1EE10FA09DD78EEFF
:10E7E800497AF5EEC07AF1EE10FA10DC23E09FEDDD
:10E7F8005D8AF1EE487A77EEC97AF5EEC07AF1EEE5
:10E8080010FAB5EEC08A13DDF1EE10FA06DD38EE27
:10E81800499ADFED557AB4EEE79A03E09FED527A14
:10E82800F4EEC77AF1EE10FA4CBF0123002312E090
:10E83800F1EE10FA06DD38EE499ADFED4C7AB4EEC7
:10E84800E79A03E09FED497AF4EEC77AF1EE10FA01
:10E85800CCBF0123002353B1B0EE4A0AF0EE4B0AB5
:10E86800FCF72FFD9FED42CA70EE008A41E02AEEC8
:10E878008A0A6AEEAABAABEE280AB0EE6B7A30EED4
:10E88800000AA8EEA87AB5EE400AF0EE007AF0EE9B
:10E89800690AF1EE10FAE7EE670AB0EE679A04D15A
:10E8A800F5EE400AF1EE10FA04D0FCF70AFDB0EEDE
:10E8B80040CA01E09FED2ECA28EEAA0AEAEE0ABA7B
:10E8C800ABEE0A0AF0EE690A30EE000AEBEEC90A6E
:10E8D800B5EE400AF1EE10FA04D1F5EE400AF1EE79
:10E8E80010FA04D0FCF7EDFCF0EE408A01E0DFED11
:10E8F800208A9FED209A204D2CEE090A07F09CF9FA
:10E9080028EE090A288007F097F9DFED1C7A1C4ADF
:10E91800688068EEE78AFDEEE88ACDED018ABDF8E9
:10E92800043013F4004F18BF03F5B47313800023A9
:10E9380000E00123002284F8D620002B7FF472AC7B
:10E9480006E00023A4F8E430A4F8E630A4F8E830A0
:10E9580017B0BDEC0A8BBDE8F08F00BF042700207C
:10E96800DB0FC93FDB0FC9BF35FA0E3C35FA0EBCC9
:10E97800000000004D3D0F44D4110020E12E6542F7
:10E988006012002001380A4B042804D8DFE800F0A0
:10E998000507090B0D00074A08E0074A06E0074A81
:10E9A80004E0074A02E0074A00E0074A1A60704795
:10E9B8000001002055CC00083DDE0008E5210108D3
:10E9C80045C90008EDC5000879BF0008704708B5BB
:10E9D8000B4B002093F82C10FBF782FD094B1B68AA
:10E9E800187A082801BF084B4FF480521A80102269
:10E9F80008BF5A80A0F109035842584108BD00BF1A
:10EA0800A80000207429002090280020024B4FF411
:10EA180080221A60704700BF140401407047704795
:10EA28007047FEE7FEE7FEE7704730B50024E3B223
:10EA380093420DD2030F092B94BF3033373301F8BB
:10EA4800143001EB4403002500015D700134EEE74A
:10EA580030BD30B5002202F1805303F5B8539B0056
:10EA680042F400441D6840F60F7144F080042940C8
:10EA780001322143042A1960EDD1024B40F0800095
:10EA8800186030BD4C5C00402DE9F347884D894C37
:10EA98002B68894E9BB2A380A28831880A409705CB
:10EAA80007D54FF6FF53854A2B6013780133DBB245
:10EAB8001370A3880B40180440F100830023ADF8BD
:10EAC80002302B687B4F9AB21804A28040F1F6827C
:10EAD800BB8803F00F03BB71002B40F0C182784A5A
:10EAE80013689BB23B803B8803F030037B803B88F4
:10EAF80003F440533B8011684BF6BF730B4083F41B
:10EB0800005383F0200343F4004343F08003136071
:10EB1800BB88D90621D4116848F60F730B406949A0
:10EB280013600B681A7A022A884601D0042A02D197
:10EB3800FBF762FC5AE2062A40F06B825A78052AF3
:10EB480008D11A78520605D1D878FFF782FFBB683A
:10EB58001B6A9847E3689B685AE213689BB2ADF852
:10EB68000230BDF802301F0540F1D0811168554FC1
:10EB780040F68F730B40544913600A68534B92B2A6
:10EB880013445B0088461A683B68187A092817D02E
:10EB980092B2520002F1804202F5C0421178197017
:10EBA800517859709188C8B2090A41EA0021598000
:10EBB8001189C8B2090A41EA002199809289DA804C
:10EBC80001221A72DA8893F80190002A40F0DC805A
:10EBD8001A7812F07F024AD1B9F1090F0FD1DA7809
:10EBE800012A00F2B8809978002940F0B480998809
:10EBF800002940F0B0809A72A3685B68A9E0B9F177
:10EC0800050F10D193F90320002A01DA0823B9E08F
:10EC18009A78002AFAD19A88002AF7D19B7A002B91
:10EC280000F0A280F2E7B9F1030F0ED1DA78012AD9
:10EC380040F091809A88002A40F08D805A7A42F0FC
:10EC480020025A72A368DB6983E0B9F1010F40F032
:10EC58008280DA78012A7ED19A88002A7BD15B7A71
:10EC6800980678D5FBF75EFC00287DD073E0012A72
:10EC78002ED1B9F10B0F6ED1E26858799269D97823
:10EC880090473B689A7A002A65D0002863D11A79A0
:10EC9800002A60D19B78002B5DD1064B9B68DB680E
:10ECA8009847084B1B685A79DA72DA781A735BE06E
:10ECB800445C004090280020DC290020AA2F002076
:10ECC800005C004074290020505C004004300020A3
:10ECD800022A40D1B9F1010FC4D0B9F1030F3AD1DA
:10ECE800587920F0800E4FEA8E0202F1804101F53A
:10ECF800B84110F0800F096814BF01F0300101F429
:10ED08004051BEF1030F26D8B3F802E0BEF1000F60
:10ED180021D101B39B7AF3B102F1804202F5B842E6
:10ED2800010613684BBF23F4E04323F4804323F028
:10ED3800400323F070034BBF9BB29BB283F01003D8
:10ED480083F4805343F4004343F080031360A368C3
:10ED58009B69984708E0E36848465B699847032839
:10ED68000FD000287FF452AFD8F80020A14B92B200
:10ED780013445B001A6800221A603023638006235C
:10ED880000E009233A6847E1B9F1060F12D11A7871
:10ED9800520678D19B78012B02D1E368DB6967E0E2
:10EDA800022B02D1E3681B6A62E0032B6BD1E36894
:10EDB8005B6A5DE0B9F1000F38D15988002962D14A
:10EDC8005A6822F47F42B2F5003F5CD11A7812F0FB
:10EDD8007F0204D19B88002B00F0D58153E0012AE3
:10EDE80008D1E26858799269904700284BD13B686E
:10EDF8009B7A17E0022A46D15A7902F00F010BB22A
:10EE08009B0003F1804303F5B84312F0800F1B68A1
:10EE180014BF03F0300303F44053032933D812F02E
:10EE2800700F30D1002B40F0AE812CE0B9F1080F03
:10EE380004D11B785B0600F0A88124E0B9F10A0F21
:10EE480021D11A7802F07F02012A1CD19A7AD2B114
:10EE58005988C1B95A6822F47F42B2F5803F12D16D
:10EE6800E268587992699047002800F090810AE09A
:10EE78004BB13A684FF00008A2F8128093614046FF
:10EE8800984740460BE0E3683A681B695078984712
:10EE9800032804D1584B1B6809221A72BDE03A684E
:10EEA800138A4FF6FF718B4201D10923B4E002287F
:10EEB80000D00BB90823AFE092F9001000291FDA3F
:10EEC800D18801910198834202D9019B138210E0F5
:10EED8008B420ED2E16891F82C00834201D20021C6
:10EEE80005E093FBF0F100FB113313B90121434B0B
:10EEF8001970E36893F82C309382FBF77DFA8CE065
:10EF0800032313724FF44053238086E0BDF8023088
:10EF18001BB2002BBFF6D5AD116840F68F730B40BE
:10EF28001360354A17683B7A022B904671D0042B40
:10EF38006FD0032B01D0052B66D1BB693A8A8BB9F8
:10EF4800398A00293BD04FF4405323802C4B1A6850
:10EF5800284B92B213445B001A6800221A603023CF
:10EF680063802CE0002AEBD0B7F81490914528BFB5
:10EF780091461FFA89FA504698473B8ACAEB030321
:10EF88003B827B8A53447B821D4B1A681D4B92B28D
:10EF980013445B0009F101021B689BB203F10053A3
:10EFA80003F5405352105B004FF0000E9645C7D052
:10EFB80053F82E1020F81E100EF1010EF6E7BB8A4A
:10EFC8008B42D8F8003001D8032201E011B10522A4
:10EFD8001A720BE006221A72094B1A68054B92B294
:10EFE80013445B001A68196030236380D8F8003036
:10EFF8001B7A0FE00230002074290020A92F00207E
:10F00800505C004004300020072B02D1E368DB6825
:10F0180098470823D8F800201372FFF7D8FC5E4BF6
:10F028001A684BF6BF7313402288D704228848BF5A
:10F0380083F480539004628848BF83F40053D10658
:10F04800628848BF83F01003920648BF83F020030C
:10F0580043F4004343F080034F4A9BB213602DE012
:10F068009A0002F1804202F5B842116889B2ADF8FF
:10F078000210BDF8021009B2002909DA106840F63A
:10F088008F7101401160013B444A52F82330984780
:10F09800BDF802301F067FF514ADA1798B0003F18E
:10F0A800804303F5B84348F60F72186802401A60A7
:10F0B8003A4B03EB81039B69984702E5A2883388A2
:10F0C8001340590505D54FF6FF332B60344B5B6869
:10F0D8009847A28831880A40920444BF4DF6FF73CE
:10F0E8002B60A3882F4A0B40DB0452D54EF6FF73E2
:10F0F8002B6000231374137C052B41D8DFE803F041
:10F10800030D1418222D6369264D1BB900F0DCFF8E
:10F11800062300E005232B743BE000F0D5FF042311
:10F1280023740123636134E002236374032328E01A
:10F13800637C013BDBB26374637C53BB194B0422D1
:10F148001A7426E0184A13689BB243F01003136040
:10F15800052323740A2363741BE0637C114A013B73
:10F16800DBB26374637C03F0FF0093B90E490C684B
:10F178004FF6EF7323400B6006231374506108E0C9
:10F188000623237405E0094B73E6094B71E6094B26
:10F198006FE602B0BDE8F087005C0040C880010857
:10F1A800A800002090280020405C0040A9A000088A
:10F1B80061A100083DA1000810B54B88DC0641BFDD
:10F1C8002F4B14791B6853F8244044BF2D4B43F848
:10F1D80020404B889B0641BF294B54791B6853F844
:10F1E800244044BF274B43F820404B881C070ED5CA
:10F1F800254B0C781B78B3EB141FA1BF204BD47898
:10F208001B6853F82440A4BF1E4B43F820404B888A
:10F218009B070ED51D4B0C781B78B3EB141FDFBF73
:10F22800174B54781B6853F82440DCBF154B43F840
:10F2380020404B88DC070FD5154C0B78247803F059
:10F248000F03A342DFBF0E4B14781B6853F824400A
:10F25800DCBF0C4B43F820404B885B070FD50B787D
:10F268000C49097803F00F038B42A1BF044B927835
:10F278001B6853F82220A4BF024B43F8202010BD7E
:10F28800AC1D0020DA0D0020B71F0020B51F00209C
:10F29800B41F0020B61F0020254A2648264900230F
:10F2A800F0B5156803700B701C461A462E1976883F
:10F2B8004EB92F5D3FB9037000230A704B70077871
:10F2C8001C461A460CE0360548BF013204F1040416
:10F2D80003F1010348BFD2B2802CDBB2E6D1EAE7E2
:10F2E800E0B2B8420CD215F8240006099E4200F09C
:10F2F8000F00A8BF731C9042A8BF421C0134EFE75F
:10F308008A704B70C2F3470102F001020A444C1E96
:10F318000A490B480A70C3F3470203F00103134478
:10F3280004700849501E084A08701370F0BD00BFE9
:10F33800B01D0020AC1F0020A8280020B61F002008
:10F34800B41F0020B71F0020B51F00202DE9F04F83
:10F35800C24BDA682DED028B1A61C14A1168D96077
:10F36800C0490B6843F020030B60BF4B1978012993
:10F3780090460CBF002201221A70BC4B1A789107E4
:10F3880089B040F13D83BA490978042940F23883AD
:10F39800B849097801F0040101F0FF0011B922F021
:10F3A80001021A701B78DB0702D408B1F8F7CAFA11
:10F3B800B149CA78531C052293FBF2F202EB820290
:10F3C8009A1AAE4BCA701B78039392000023AC4C78
:10F3D800DFF8CCC2DFF8D8925CF8231091FBF9F57E
:10F3E80004F1080004F1100640F82350A54844F839
:10F3F800231000FB051142F2107091FBF0F080B26F
:10F4080026F813004FF0140E04F1140604F13C0A18
:10F418000EFB036E5AF823605EF802704EF8021075
:10F42800F61B314444344AF82310052691FBF6F1C3
:10F4380009FB051144F82310039C012C4FEA830BA8
:10F44800E24605D10238B0F5797F98BF4BF80C1029
:10F458000BB90123BBE7884CD8F80030226D9FED2B
:10F468008A7A8A4E8A4D9B1A07EE903AF8EE677AA6
:10F47800D8F800302365C7EE877A7C4B1B78B7EE47
:10F48800008AF4EEC87AF1EE10FA58BFF0EE487A26
:10F4980013F00103C4ED157A12D005AA00927D4B32
:10F4A80006AA01920CCB9AE80300F8F749F96421FF
:10F4B800059A069BB2FBF1F293FBF1F3328000E070
:10F4C80033802B8094F858306B48002B3BD0D0ED1C
:10F4D800157AC26DDAF80030C8EE276A9B1A026EF8
:10F4E800022507EE103AB8EEC77ADAF8043027EEAC
:10F4F800267A9B1AFDEEC77AB0F9662017EE901AA5
:10F5080007EE903A644BB8EEE77AD3ED007A67EEEF
:10F51800277A67EEA67AFDEEE77A17EE903A02FAB6
:10F5280083F3B0F9642093FBF5F302FA81F29BB2FE
:10F5380092FBF5F292B2A0F86A30A0F86820A0F821
:10F548006630A0F86420012384F85830534BDAF869
:10F5580004101B88DAF80000474D514E216603F06D
:10F568003003E065002B00F04B8205F17403009333
:10F5780005F178030193EA6E2B6FF8F7E1F87268EA
:10F588002B6F9B1A07EE903A434B326893ED007A43
:10F59800EB6EF8EEE77A9B1AEB67384B67EE877AE3
:10F5A8001B78FDEEE77A012BC5ED207A03D0022BFC
:10F5B80000F0DF8024E2D5ED287A3A4BD5ED215AC8
:10F5C80095ED255A95ED156A95ED264AD5ED274A0C
:10F5D80035491D68B1EE677ABDEEC77AFDEEE77A68
:10F5E80017EE10EA17EE90CA0020304A91ED007A23
:10F5F80052F8207007EE907AF8EEE77AA2F1140339
:10F6080067EEA57A33F81060FDEEE77A283217EE38
:10F61800903A9B1B9BB222F810301BB207EE903A2F
:10F62800F8EEE77A3B4467EE857A4400FDEEE77A28
:10F63800CDED037A07EE903AF8EEE77ABDF80C8044
:10F6480067EE847AA7EE867AFDEEC77A17EE902ADF
:10F65800724531DB6245A8BF62462EE004080020EF
:10F66800481200208C1A0020EA110020901A00206D
:10F67800961A0020A62F0020A8280020A00F0020FE
:10F68800AC280020806967FF00007A440A1B00202C
:10F698000C1B0020EC1100206C000020541B0020E3
:10F6A800981A0020A40F0020D40F0020242900203D
:10F6B80080969800DB0FC940724607EE902AF8EE54
:10F6C800E77A5FED046AC1ED007AFDEEE77A31363C
:10F6D80017EE903A43449AB2AB78D1ED027A07EE2E
:10F6E800103AB8EE477A4B684F6027EE267AFB1A35
:10F6F80088EE077AB6B2622E06EE903AF8EEE66A1F
:10F7080037EE067AC6EE866A86EE077A76EEE76AFE
:10F71800E7EE267AC1ED047AC1ED027A0FD964EEDC
:10F72800A77ABA4EFDEEE77A17EE903AB3F5FA6F7C
:10F73800A8BF4FF4FA63B342B8BF334600E00023D2
:10F7480013441BB240F6B8329342A8BF1346B04ADE
:10F758009342B8BF1346AF4AA352AF4A142303FBE0
:10F76800002351F8142B1A60002840F04981012029
:10F778003BE7AA4BD5F874801F68D4F878903E8987
:10F78800DFEDA78A4FEA58039E4228BF1E46B5F808
:10F79800A8301AB29642C3BFD5ED157A9FEDA17A6B
:10F7A80067EE877AB6B2C1BFFDEEE77A17EE906AC8
:10F7B800F618B6B2C8BFA5F8A860D4F8AC50C5EB27
:10F7C80009052846F8F700F80028D8BF404241F25A
:10F7D80093129042CCBF0020012088B307EE905AC4
:10F7E800B8EEE70A20EE280AFBF7DEFD07EE908A5E
:10F7F800F8EE677A40F6B83320EE270AFDEEC07AB5
:10F80800CDED037ABDF80C20A4F8B02012B29A42CC
:10F81800A8BF1A467E4B9A42ACBF09EB02034B4481
:10F8280048F6A042934203DDA3F50C43A03B04E055
:10F83800002BBCBF03F50C43A033C4F8B43001E07F
:10F84800C4F8B490D4F8B450C5F50C53283307EE77
:10F85800903AF8EEE77A67EEA88AB0EE680AFBF706
:10F8680003FE8DED070AB0EE680AFBF79DFDD4EDA7
:10F87800317AD4ED2E4AD4ED155A94ED2F4A94EDF1
:10F88800305A65498DED060AB1EE677ABDEEC77A42
:10F89800FDEEE77A0DF1180E17EE10AA17EE90BAE2
:10F8A8000020614AFEEC016A32F91030DFF88C91D1
:10F8B80007EE903A07EE106AF8EEE77AB8EEC77AE4
:10F8C8003C32D6EE877A4FEA400CFDEEE77ACDED72
:10F8D800037ABDF90C30B3F57A7FA8BF4FF47A7379
:10F8E8004B45B8BF4B461FFA83F922F810900FFA20
:10F8F80089F207EE902AF8EEE77A27EEA47ABDEEB1
:10F90800C77A8DED037A27EE847AD1ED007ABDF8B7
:10F918000C90E7EE257AFDEEE77A17EE902A52452D
:10F9280003DB5A45A8BF5A4600E0524607EE902A24
:10F93800F8EEE77A9FED3D6AC1ED007ABA7891ED6D
:10F94800027A06EE902AF8EE666A4A684B6066EE1E
:10F95800866A9A1AC8EE266A143106EE102AB8EE9C
:10F96800C66A76EEA56A86EE256AC5EEA66A36EE02
:10F97800476AA6EE867A01ED017A01ED037A25EE53
:10F98800077ABDEEC77A17EE103ABDEEE77A4B4418
:10F9980017EE102A13441BB240F6B8329342A8BFA0
:10F9A80013461B4A9342B8BF13461A4A2CF8023032
:10F9B8001F4A142303FB0023C3ED007A08B9012072
:10F9C8006FE73B7923B1642395FBF3F5194B1D8051
:10F9D8003B8898450DD9D4F8AC30A06FC01AF7F71A
:10F9E800F3FE80EAE072A2EBE07242F210739A42F0
:10F9F80006DD114B01221A700E4BB4F8C8201A808C
:10FA080009B0BDEC028BBDE8F08F00BF30F8FFFFF6
:10FA180048F4FFFF28100020FC0F0020A40F00204E
:10FA2800D30237390000C84210290020DB0FC94033
:10FA3800D40F00209C0F0020A00F002018FCFFFF0F
:10FA480020B9034B1B6808221A8270470148704787
:10FA5800742900207000002020B9034B1B6808227D
:10FA68001A827047014870477429002070000020EE
:10FA780021B901288CBF022000207047022070475E
:10FA880010B5094B1A68D378042B0BD8074C518A48
:10FA9800DB00234418B99B895B1A138210BD9B684D
:10FAA800581810BD002010BD7429002070000020D7
:10FAB800054B1968054B4A8A18B99B8D9B1A0B820E
:10FAC8007047986A1044704774290020700000201D
:10FAD800054B1968054B4A8A18B99B8E9B1A0B82ED
:10FAE8007047186B1044704774290020700000207C
:10FAF800074B1B681B7803F07F03212B06D100F00E
:10FB0800DF00022814BF022000207047022070473F
:10FB180074290020212810B508D1114B1B681B78C7
:10FB280003F07F03212B10D0022010BD2028FBD129
:10FB38000B4B0C4A1B6810701B7803F07F03212BBA
:10FB4800094B18BF00230BB9EEE7084B044A1268AB
:10FB580000249361548220469847204610BD00BF78
:10FB680074290020AB2F002049FA000861FA000828
:10FB78007047034B1A78202A04BF00221A70704776
:10FB8800AB2F0020014B04221A607047882F0020F9
:10FB9800034B9B7B13B1034B05221A60704700BFD0
:10FBA80074290020882F00200D4B0E491A680E4B2F
:10FBB80092B213445B000D4A1B68C3F3090310B5E6
:10FBC8001362136A9BB201335B1000229A4206D07B
:10FBD800074851F8044B20F812400132F6E710BDEF
:10FBE800505C0040206200401E3000207429002034
:10FBF80098290020014B00225A667047742900207A
:10FC08002DE9F843664B674E1B68DFF8B881664AF2
:10FC180000254FF0C0099D7283F80990DD723560A8
:10FC2800D8F8003023F4EC4323F0700343F4007356
:10FC38009BB2C8F80030D8F8003023F4E04323F032
:10FC480040039BB248F2800483F010032343C8F8B2
:10FC58000030336812FA83F35B0040271A681F608C
:10FC680033689BB203F1005303F540535B00284609
:10FC78001A6880221A60D8F8003023F4F8731B053C
:10FC88001B0D2343C8F80030484B93F86410FAF76B
:10FC980027FCD8F80030464A464923F4804323F02D
:10FCA80070039BB283F440532343C8F800301368B1
:10FCB80023F4EC4323F070039BB21360336811FA0A
:10FCC80083F35B0003201968C3F8009013683A496E
:10FCD80023F4E04323F040039BB283F02003234343
:10FCE8001360136823F4804323F0700323439BB20B
:10FCF8001360536823F4EC4323F0700343F4C063A8
:10FD08009BB25360336811FA83F35B0019684FF4B0
:10FD180080711960536823F4804323F070032343F0
:10FD28009BB25360536823F4E04323F040039BB233
:10FD380083F0200323435360D8F80C301F4A23F480
:10FD4800EC4323F070039BB2C8F80C30336812FA06
:10FD580083F35B0039461A684FF488721A60FAF721
:10FD6800BFFBD8F80C3023F4804323F070039BB218
:10FD780083F440532343C8F80C30D8F80C3023F4EC
:10FD8800E04323F040031C43A4B2C8F80C402846C3
:10FD9800FEF75FFE0A4B01221A60BDE8F88300BF38
:10FDA80074290020505C00400430002070000020BE
:10FDB800045C004008300020103000201C30002077
:10FDC800882F0020005C0040134A144B50681B68C1
:10FDD800181810B5146808D011490822FEF725FE36
:10FDE800204610490422FEF720FE0F48026800232F
:10FDF80093720E4A012111600D4913604FF4E054CB
:10FE08000B6014600B604FF43641A0F86810116065
:10FE1800084A136010BD00BFB0F7FF1FACF7FF1F03
:10FE2800DA000020EA00002074290020405C00402D
:10FE3800445C0040882F002010B50446B0F900004B
:10FE480000F041FDB4F9020000F03DFDB4F90400F2
:10FE5800BDE8104000F037BD10B50446006800F05A
:10FE680032FD606800F02FFDA068BDE8104000F08A
:10FE78002ABD2DE9F74F0120F9F784F9002488B34A
:10FE8800012C2FD8194E4FF04C0909FB04FA06EB48
:10FE98000A0808F1B407BD7815B10134E4B2EEE7F9
:10FEA80090F9003090F804E01846114B03228DE8D1
:10FEB800240001212A4653F82E30F8F787FF83469D
:10FEC80060B106F16C00504429464A4605F0A5FC8D
:10FED80001231C44C8F86CB0BB70E4B20120F9F7E8
:10FEE80035F9CCE703B0BDE8F08F00BF74290020D6
:10FEF800048101080021222210B5114805F08DFC6B
:10FF0800104B0022194610480424105C83F8F401B1
:10FF18000132052083F8F941042A4FF0000483F8E0
:10FF2800F80183F8FB4183F8FA0103F10803EAD1E9
:10FF38000123A1F8F631522381F8F23110BD00BF38
:10FF480062140020701200204BA0010810B5FAF7C7
:10FF58001FFC4FF43024012806D11CB1FAF718FC15
:10FF6800013CF8E7052010BD002C08BF052010BD96
:10FF780070B50646441E14F8011F89B1094D28467C
:10FF880005F081FC0028F6D005F1080398423FBF30
:10FF9800054B401BC018A31B38BF80F88831EAE71F
:10FFA80070BD00BF4FA0010870120020031EB8BF2B
:10FFB8002D2210B5B8BF58420C46B8BF01F8012B26
:10FFC8000A22FBF74FF800230370204610BD07B53F
:10FFD8001C4B03F58472C3F804211B4A92F8902144
:10FFE8005AB1012A14D1032183F80A11072183F891
:08FFF8000C2183F80B110C220F
:020000040801F1
:1000000008E0022183F80A11032183F80C2183F808
:100010000B11072283F808210E4B0F4AC3F88420E6
:100020004020F9F7B3F870B10122002390F90000E5
:1000300040218DE80C00094A4FF4E133F8F7CAFE7D
:10004000003018BF012003B05DF804FB74290020C4
:1000500070120020700000203DA2000869A3000873
:100060000120002100F0B0BDF0B5184A92F80D3122
:10007000D2F810711546032B11D807EBC3025E1C92
:10008000941CF6B209D013469288D10705D51042C8
:1000900003D008E00131042908D13346EBE785F8A5
:1000A0000D310020F0BD93F802E00021074C0C2236
:1000B00004F58A7C02FB01F31CF803209645E9D184
:1000C000234484F80D61D3F81801F0BD7429002091
:1000D0000A4B10B519684FF6FB720A401A60084ABD
:1000E000927B1C46074B0AB1052200E001221A60F0
:1000F00000F0AAFA4FF43643236010BD405C004084
:1001000074290020882F00200F4B1A786F2A17D1EE
:10011000598840F60402914212D11A79BE2A0FD1B1
:1001200093F80028EF2A4FF000000BD113F8012BB1
:100130005040064A9342F9D1B0FA80F04009704726
:1001400000207047704700BF00F0030804F8030860
:100150002DE9F04F2DED028BDA4C002140F6040220
:1001600085B0204605F05DFBD74B04F539721A6067
:10017000D64A00231370D64A04F2D27111606F225E
:1001800022700322627140F20112A2604FF41672D3
:10019000A4F86421FA22A4F866214FF4FA7220210F
:1001A000A4F86C21012284F85E2184F8681184F897
:1001B00069216E2184F86A2184F87C2184F88421E5
:1001C000052284F87A1184F823220A2140F2DC52B5
:1001D00084F87B11A4F896212B2140F24C4284F83C
:1001E0007D11A4F89821212140F26C7284F87E11CF
:1001F000A4F89A21232140F2753284F87F11A4F8E3
:100200009C214FF4C87140F64302A4F89E21A4F843
:10021000801125462246032BCCBF0121002103F18A
:10022000010382F8A01114BF1E210521122B82F8B0
:10023000A11102F10202EED140F27E424FF4FA63C4
:10024000A4F8402140F23A72A4F8C631A4F8CA31A9
:10025000A4F8CE31A4F8D231A4F84221052340F20B
:100260007E5284F8E031A4F84821C82340F2EA52D3
:1002700001274FF47A7B32214FF01E0840F2DC5CFC
:100280004FF0190AA4F8E431A4F84A214FF4C873D6
:1002900040F2B45284F8938184F8DF7184F8E1A1CC
:1002A00084F8E27184F8E37184F8E671A4F8E83127
:1002B00084F8EC71A4F846C1CDF80CC0A4F84C2128
:1002C000A4F84E11A4F85031A4F85211029184F808
:1002D000EF71A4F8C4B1A4F8C8B1A4F8CCB1A4F8E3
:1002E000D0B1A4F844B1FFF709FE774A0299136828
:1002F000019200264FF05F0E267383F803E04FF063
:100300000F0E83F805E04FF0220E83F806E04FF061
:100310000E0E83F810E04FF0350E83F81AE04FF020
:10032000210E83F811E04FF0530E83F81BE04FF0DD
:100330005A0E83F808E04FF0780E83F80AE04FF089
:100340002D0E4FF02809142083F80B8083F80C80C1
:1003500083F807A04FF00A084FF0640A83F814E00E
:100360004FF4FA7E1F7058759875597319719F77FD
:1003700083F8019083F8029083F817809E731E76AD
:10038000DE735E7683F8128083F81CA083F80990F0
:10039000A3F84EE0DFF854E1C3F838E0C3F83CE0DE
:1003A000DFF84CE1C3F828E0DFF848E1C3F834E0B7
:1003B000DFF844E1C3F848E0DFED467A9FED468A76
:1003C000C3ED0B7A4FF04B0E83F84CE04FF4E17E17
:1003D000C3ED0C7AA3F85CE0B7EE087AF1EE047A8C
:1003E0004FF0100E83F85EE083F8509083ED087AAA
:1003F00083ED097A83ED108AC3ED117A83F8536097
:1004000083F8548083F8558083F8568083F857A08A
:1004100083F858A083F859A083F85A60DDF80CC01F
:1004200084F8D4174FF0460E042184F8D3E784F8FB
:10043000DA07A4F8DCC784F8D2A784F8D56784F873
:10044000D96784F8D66784F8D76784F8D86783F8C3
:100450006810152183F87410204999672049D967DD
:100460002049C3F8801083F88470A3F86460A3F86F
:100470006660A3F86260C3ED1B7A83F8709083F81E
:1004800071901948FFF778FD019A13684FF448718D
:1004900083F82071A3F8221183F81D6183F81E618F
:1004A00083F81F9183F82461194684F8D68184F873
:1004B000D781A4F8D8B184F8DA61A4F8DCA1174692
:1004C0001CE000BF70120020B8110020B82A0020E4
:1004D000E4110020CDCCCC3E000000009A99193FD9
:1004E000F6287C3F3D0A773F64A001088FC2F53CA7
:1004F000000060406666663F000040400E2202FB3E
:1005000006326FF0170082F82501032082F82601D9
:100510006FF02F0082F82701072082F828016FF082
:10052000230082F82901052082F82A0101365A2089
:1005300081F82C0181F82D016422FF20082E81F81A
:100540002B2181F82E0101F10E01D7D1002183F872
:100550009511C821A3F89611142183F89811A3F8D6
:100560009C211E214FF4967283F89911A3F89E21C5
:100570000121282283F89A11A3F8A0212D4B18EE0F
:10058000102A45F8102F9D42F9D12B480021402216
:1005900005F047F90023294D294C59591A190433FC
:1005A0000868C2F8A402382BF5D104F509700021BF
:1005B000802205F036F905F13801702204F5097042
:1005C00005F024F9FEF76CFE3E6800230125314654
:1005D00004F591604FF4D27284F8F83784F8F65736
:1005E00084F8F75705F012F904F22C6031464FF405
:1005F000D27205F00BF9134B1B681A68C4F8DE279A
:100600005A68C4F8E2279A68C4F8E6271A68C4F85A
:10061000EA275A68C4F8EE279A68C4F8F22702233A
:1006200084F8E85484F88C3605B0BDEC028BBDE844
:10063000F08F00BF3013002014150020C481010882
:1006400070120020E41100201549D1F8883043F4DD
:100650007003C1F88830134B1A6842F001021A6027
:100660005868114A02405A601A6822F0847222F4D3
:1006700080321A601A6822F480221A605A6822F4C2
:10068000FE025A60DA6A22F00F02DA62186B074A39
:1006900002401A6300229A604FF000638B6070473B
:1006A00000ED00E0001002400CC07FF8CCFC00FF21
:1006B0000B4B1B6898420CDD0A4B93F8F83753B983
:1006C000094B1B681B6943B18342CCBF0120022048
:1006D000704700207047022070470120704700BF1C
:1006E000102E002070120020702C002038B5094B0D
:1006F00093F8F85765B9084C2068F8F758FB074B92
:1007000025601B78022B03D1BDE83840FFF7B5BB4D
:1007100038BD00BF70120020702C00206D2C00200E
:10072000044B93F8F8371BB9034B186800F056BE1A
:100730000020704770120020702C002038B505464C
:100740000446204614F8011B21B1034B186800F041
:1007500051FEF6E7401B38BD702C00200FB407B5E2
:1007600004AB064953F8042B01930020FAF792FCDE
:1007700003B05DF804EB04B0704700BF290901081D
:10078000024B0146186800F035BE00BF702C0020F7
:10079000F8B5011F06460023083051F8042F02F176
:1007A00020043F2C3AD802F108040F2C06D802325C
:1007B000032A04D9002B08BF012300E00223814251
:1007C000EBD1012B30680ED0022B1AD0736803F0E6
:1007D00003039B0000F0030043EA0010B36803F03A
:1007E0000303184317E000F00F0040F04000FFF74C
:1007F000C7FFB068736800F00F0040EA0310C0B292
:1008000009E000F03F0040F08000FFF7B9FF3079C9
:10081000FFF7B6FF307ABDE8F840B1E706F10C0704
:1008200034463A46002552F8043D03F18001FF2981
:100830004FEA850510D903F50041B1F5803F02D29A
:1008400045F0010508E003F50003B3F1807F34BFF4
:1008500045F0020545F00305B242E4D165F03F00E2
:10086000C0B2FFF78DFF05F00303022B207807D0FD
:10087000032B0CD0012B13D1FFF782FF60780FE020
:10088000FFF77EFF6078FFF77BFFA07808E0FFF7B7
:1008900077FF6078FFF774FFA078FFF771FFE078CB
:1008A0000434FFF76DFFBC424FEAA505DBD1F8BD6C
:1008B00010B504467F2C06D964F07F00C0B2FFF764
:1008C0005FFFE409F6E7E0B2BDE8104058E74300F7
:1008D00083EAE070ECE70FB437B506AC482054F873
:1008E000045BFFF74DFF2020FFF74AFF2A4623460F
:1008F0000B4901940020FAF7CDFB04460A20FFF7CC
:100900003FFF084BC4F1FF241A6804F57F04FD344F
:1009100014441C6003B0BDE8304004B0704700BF11
:1009200029090108102E0020084629E707B5064BC3
:100930000093064B01930649064A074B0748FAF70E
:1009400096FC03B05DF804FB439301081B93010878
:1009500093A00108A0A00108379301086DA0010829
:1009600008B5037833B90C4B0C481978BDE808403A
:10097000FAF77DBC04F0F0FF02280CD8064B187083
:10098000074B0C2202FB0030064B02301860FAF7CE
:1009900063FE0548E5E708BDB82A0020A7A00108C6
:1009A000401A0020E41100201396010808B50378CE
:1009B0003BB90B4B0B4893F8D017BDE80840FAF74A
:1009C00056BC04F0C9FF022808D8054B83F8D007AD
:1009D000FAF7A8FDFAF764FE0348E8E708BD00BF90
:1009E00070120020ABA001081396010838B50378F7
:1009F00003BB214B1B6801330F2B07D81F490C2267
:100A000002FB03121C4695682DBB00E01C46013416
:100A10000F2C01DD002400E005D818490C2202FB50
:100A200004129568BDB99C42F1D11548BDE8384023
:100A3000FAF71DBC04F090FF0F28044605D80F4AB2
:100A40000C2303FB00239D682DB921460D48BDE80A
:100A50003840FAF70CBC084B1C6000F011FC214632
:100A60002A460948FAF703FC0C235C43034B185D44
:100A7000BDE8384000F018BCF80000209C82010856
:100A8000B8A00108CEA00108E6A0010873B503785C
:100A900013B9F7F7C1FE3DE01F4901AA04F0BDFFFD
:100AA000002401462646254699B134B1012C08D1CF
:100AB000084604F051FF064603E0084604F04CFFE8
:100AC00005461549002001AA04F0A7FF013401469C
:100AD000EAE70B2D02D911480C220BE0022C10D1B1
:100AE000A6F57A73B3F57A7F07D90D484FF47A717A
:100AF0004FF4FA62F7F70DFE0CE00A4B03EB4503E7
:100B00005E80084B084803EB45032946B3F90220F1
:100B1000FAF7ADFB02B070BD609A01089098010829
:100B2000C39D0108B82A0020FDA0010838B50D4C6E
:100B300023688342054606D1F8F739F9204600219B
:100B40004C2204F06EFEE36CAB4209D12846F8F764
:100B50002EF9054800214C22BDE8384004F061BE62
:100B600038BD00BFE02900202C2A0020034B1A6862
:100B7000D379591C1344D171187A7047341B002063
:100B800010B5FFF7F3FF84B2FFF7F0FF04EB00208E
:100B900080B210BD10B5FFF7F3FF0446FFF7F0FF7A
:100BA00004EB004010BD064B10B504462146186802
:100BB00000F020FC034B1B6898796040987110BDD1
:100BC000381B0020341B002038B5044624200D4675
:100BD000FFF7E9FF4D20FFF7E6FF002C084C14BF9C
:100BE00021203E20FFF7DFFF2368002228469A716C
:100BF000FFF7D9FF236893F84900BDE83840D2E7F2
:100C0000341B002001460020DEE710B50446C0B2C8
:100C1000FFF7C9FF200ABDE81040C4E710B504463D
:100C200080B2FFF7F2FF200CBDE81040EDE737B5CA
:100C300082888368044610060D4641BF2B4991F80F
:100C4000D0174FF4D27000FB0133D10544BF2849BF
:100C5000097802F03F0244BF01EB410103EB81033D
:100C6000042A12D006D8012A0DD0022A32D193F9D3
:100C7000001030E0102A0AD0202A0AD0082A29D1F0
:100C8000B3F9001027E0197825E0198823E01968E6
:100C900021E093ED000A6846FAF77EF9014615480F
:100CA000FAF7E5FA05B3D4ED037A6846B8EEE70A39
:100CB000FAF772F901461048FAF7D9FA94ED040AE6
:100CC0006846B8EEC00AFAF767F901460A48FAF72B
:100CD000CEFA09E000210948FAF7C9FA25B1084817
:100CE000E1682269FAF7C3FA03B030BD7012002040
:100CF000B82A00206B9901086499010810A1010825
:100D00000CA10108024B0146D86900F073BB00BF7B
:100D1000B82A002010B5441E14F8011F21B1034B5E
:100D2000D86900F067FBF7E710BD00BFB82A0020C4
:100D3000F7B52B492B4B08782B4D1C682B4B05EB3B
:100D400080001A882A4BD0F8C0101B7829480091DF
:100D50004FF47A71B4FBF1F1FAF789FA2648482189
:100D6000FAF785FA254B1F680026F3B205EB8302DC
:100D7000D2F8D010E9B101249C403C4217D02207A0
:100D800015D01F4AD25C0B2000FB0323164A1D48D6
:100D900002EB8303D3F8F020FAF769FA022C06D1AC
:100DA000194B93F8281011B11848FAF760FA013678
:100DB000DBE71748FFF7AEFF164B17481A68174BCB
:100DC0009A420CBF164B174B1A88174B198892B2D0
:100DD00040F6040303B0BDE8F040FAF748BA00BF9C
:100DE000DC1A0020481200209C8201087C1A002096
:100DF000FC00002013A1010856A101088C1A002054
:100E00000401002066A10108B82A00206EA1010893
:100E1000B6A101087411002072A10108005400401D
:100E2000781100207A110020701100202DE9F04186
:100E30000024804625460F4EA7594146384604F007
:100E400073FD58B139460C48FAF711FA30190021F0
:100E5000FFF7EDFE0948FFF75DFF0135143440F65A
:100E600034539C42E7D11DB90548BDE8F04151E734
:100E7000BDE8F0813C840108E2990108B6A10108AF
:100E8000E79801082DE9F04F2DED028B83B0054660
:100E900004F00BFD064620B1012818D12B782A2B2F
:100EA00015D15C48FFF736FF00245B4D5B48615964
:100EB000FAF7DDF928193146FFF7B9FE5848FFF770
:100EC00029FF143440F634539C42EED19CE028466E
:100ED0003D2104F0DCFC002800F08F800346994699
:100EE00013F8012D202AFAD0441C204604F034FDCA
:100EF00080462046F9F7C6FFC5EB0909B0EE408AE7
:100F00000026DFF834A1142202FB06F40AF5D07B98
:100F100054F80B70384604F0C8FC03461A462846BD
:100F20003946019304F0CAFC019B00285BD15FFAAB
:100F300089F29A4257D10AEB0402D2ED6B7AF8EEAD
:100F4000E77A0BEB0405B4EEE78AF1EE10FA48DB22
:100F5000D2ED6C7AF8EEE77AB4EEE78AF1EE10FAA9
:100F60003FD8B2F8A431D2F8A82113F0200F08BF5F
:100F700008EE108A1C0641BF2A4991F8D0174FF499
:100F8000D27404FB0122D90544BF2749097803F034
:100F90003F0344BF01EB410102EB8102042B18EE39
:100FA000100A0BD004D8013B012B0ED810700CE0B6
:100FB000102B05D0202B06D0082B06D1108004E082
:100FC00082ED008A01E082ED008A39461748FAF77F
:100FD0004EF92846002103B0BDEC028BBDE8F04F6E
:100FE00025E6134803E00136A92E8AD1114803B043
:100FF000BDEC028BBDE8F04F8CE6284603B0BDEC9B
:10100000028BBDE8F04F11E703B0BDEC028BBDE8E9
:10101000F08F00BFA4A101083C840108E2990108F7
:10102000B6A1010870120020B82A0020B9A1010859
:10103000C4A10108E79801089C82010870B5054623
:10104000284604F032FC064658B9194B19485A791B
:10105000194B03EB8203BDE87040D3F8D01EFAF7BA
:1010600006B928461549324604F028FC60B91448F0
:10107000144CFFF74FFE54F8041F19B11248FAF749
:10108000F6F8F8E7114805E00024114B53F8241056
:1010900019B91048BDE870403CE62846324604F0D5
:1010A0000DFC01340028F0D1014B0B4D5C71C7E7FA
:1010B00070120020E4A101089C82010882990108B5
:1010C000F0A101086C9101087E990108B6A1010800
:1010D00070910108E79801081396010808B50748C0
:1010E000FFF718FE064BD869F7F756FE00F0ECFA4A
:1010F000FAF7EEF9034B044ADA6008BD03A20108CF
:10110000B82A002000ED00E00400FA0508B5054803
:10111000FFF700FEFFF71CF8FAF704FABDE80840F5
:10112000DCE700BF0FA2010808B50448FFF7F2FD95
:10113000FAF7F8F9BDE80840D0E700BF25A201089A
:10114000044A536823B192F90020824200D1184723
:10115000704700BFFC2A0020034B4FF4005208B137
:101160009A6170471A85704700040048034B4FF49A
:10117000005208B11A8570479A6170470004004810
:101180000A4B1B6813F4805F094BB3F9063005D096
:10119000C089421A934207DD084400E0008A834276
:1011A000B4BF00200120704701207047741A00204E
:1011B000202F00201FB5094B1B681B030AD58DF893
:1011C000040001230D2001A98DED030A8DF80530DF
:1011D000F6F760FE05B05DF804FB00BF741A00204E
:1011E0001FB5084B1B681B0309D58DF8040002913D
:1011F00000230D2001A98DF80530F6F74BFE05B050
:101200005DF804FB741A002010B50A4A0A4B1168F5
:101210009B6800BF12689142F7D1084A94684FF466
:101220007A7000FB04F2D31AB3FBF4F300FB013035
:1012300010BD00BF4812002010E000E0FC2A002092
:1012400038B5044654B1FFF7DFFF0546FFF7DCFF72
:10125000401BB0F57A7FF9D3013CF3E738BD024A71
:10126000136801331360704748120020172067E7A6
:10127000282065E7014B1B68184700BF8C2F002012
:1012800010B50020FFF7F6FF054B00241C7001F09D
:10129000B5FA044B1C731C619C829C6110BD00BF9D
:1012A000702F0020FC2A002010B5E0B1124B1B6803
:1012B00013F0020304D0114B1B78012B13D9002328
:1012C0000C225A430E4C1119125D824203D0013395
:1012D000102BF5D110BD0B4B986938B14A78407886
:1012E000824203D310BDBDE81040C9E700229961D6
:1012F0009A821A6110BD00BF741A0020FC00002001
:101300009C820108FC2A002010B540001428A8BFC8
:1013100014200023074A022199540B4499181424DD
:10132000834201F8014CF5DBFF21D1540F20BDE8C9
:101330001040B9E7E42A00202DE9F84380460B2548
:10134000013D3FD0224B4FF480421A854FF40042BA
:101350009A6108F1010632274FF005091C4CA38A57
:101360009BB283F48043A382A38A9BB283F400439D
:10137000A3820120FFF77EFF3846FFF761FFA38AB3
:101380009BB283F48043A382A38A9BB283F400437D
:101390000020A382FFF76EFF3846FFF751FFB9F137
:1013A000000F08D0B9F10109D8D14FF4FA70FFF756
:1013B00047FFFA27D2E7013ED0D14FF47A70FFF70A
:1013C0003FFFBDE7034B044ADA60BDE8F88300BF86
:1013D0000008004800ED00E00400FA0503685B69BE
:1013E000184703681B6918470368DB6818470368D8
:1013F0005B68184703681B6818472DE9F84FB0F978
:101400000230934218BF00232DED048B18BF0370E8
:10141000057804460E469146002D40F0978007EE71
:10142000902ADFED7D8AF8EEE77AB6EE009A67EE55
:10143000A88ADFED7A7A68EEA78AA04668EE898AE4
:101440002746B0EE680AF9F7B3FFB0EE408AB0EE77
:10145000680AFAF70DF888EE000A40F2DC5363657B
:101460001023A4F852301823A4F85030DFED6C6A32
:1014700060EE266AB7EE006AB0EE667AA0EE007AF9
:10148000D0EE006A37EE067A76EE866AC6EE077A06
:1014900084ED046A27EE807AB0EE498A27EE007A5E
:1014A00077EE075A84ED017AC4ED025A70EE005AC5
:1014B00084ED037AB8EE007AA5EE807A27EE877A7B
:1014C00067EEA67A84ED057AC4ED067ADFED557AEB
:1014D00098ED047A27EE277AF0EE678AB5EEC07AA7
:1014E000F1EE10FA4CBF77EE487A77EE087A0135C4
:1014F00017EE900A01F0E8FBD8ED017A67EEA87AC2
:10150000C7E90E01F5EEC07AF1EE10FA4CBF77EEA6
:10151000C87A77EE887A08F1040817EE900A01F08D
:10152000D3FB032DC7E9080107F10807CED1A6F2C6
:10153000DC531B042367E3676367C4F88030A36749
:10154000C4F884300123A4F802902370D4F8549096
:10155000B4F95280636A276A206FE26FD4F840C002
:10156000D4F88010C4F88020C9EB060606FA08F605
:101570004FEAE67B734307FB0B332667A7FB06673F
:101580001F44636C656F60674FEAE27B53430CFB5B
:101590000B3EACFB02237344B61A67EB0307E36A06
:1015A000A26AC4F884104FEAE07B434302FB0B3E7F
:1015B000A2FB00237344B6185F41E36CA06CB4F93E
:1015C0005020A5674FEAE17B4B4300FB0B33A0FBA8
:1015D00001011944636B361A206B4FEAE57B05FB6A
:1015E00003F300FB0B3367EB0107A0FB0501194474
:1015F0008019794101F036F908F1FF320123934057
:10160000E067C01841EBE371424601F02BF9BDECF5
:10161000048B4844BDE8F88F6F12833ADB0F4940D2
:10162000F404B53F0000804B2DE9F8430024234B20
:1016300093F84C60E0B2B0420CD203EB8003204A36
:10164000DB6932F810101BB10B2801D8DB68984712
:101650000134ECE71B4B1B685B032CD500242346AD
:10166000E2B2B24227D2DFF8549009F11C074FEAE8
:10167000840857F8242055689D4214D02846FCF76A
:1016800061F8EFF31283502282F3128828216A6AEC
:1016900001FB0090013242676A6942F001026A610F
:1016A000DBB283F3118857F808301B6800221A60F8
:1016B00001342B46D4E7BDE8F88300BFFC2A0020A4
:1016C000BC110020741A002008B50E4B1B6813F4DF
:1016D000805F0D4B14BFD3F8F020D3F8F42093F8BB
:1016E0004C1092880023D8B2884204D2074820F8D0
:1016F00013200133F7E7FFF797FF3220BDE80840DA
:101700009EE500BF741A0020FC2A0020BC110020B6
:101710000A4B1A680A4B30B502F48052D3F8F040F5
:10172000D3F8F45000230AB1A18800E0A988054845
:1017300020F8131001330C2BF5D130BD741A0020A2
:10174000FC2A0020BA2A002070B5124D0024214640
:1017500005F1F900702285F8F84004F062F821469E
:10176000D5F86C310B4A0B4493F9020080B102F1B9
:10177000F9041E680E5108199C8884809B79837136
:1017800092F8F83007310133702982F8F830E7D148
:1017900070BD00BFFC2A0020094B1A680E2303FB12
:1017A0000020437AFF2B07D0064A12789A4203D9C9
:1017B000054A32F8130000E0808800B2704700BF8D
:1017C000B41D00207C2A0020202F0020D0ED024AEA
:1017D00091ED016A90ED015A91ED027AD0ED005A37
:1017E000D1ED007A66EE646AE5EE076A27EE657A67
:1017F000C2ED006AA4EEA77A67EEC57A82ED017A9F
:10180000E5EE867AC2ED027A7047D0ED017A91ED6D
:10181000017AD1ED026A91ED006A37EE877AD0ED58
:10182000027A77EEA67AD0ED006A82ED017A76EE42
:10183000866AC2ED027AC2ED006A704790ED017AC5
:10184000D0ED027AD0ED006A20EE077A60EE277ABA
:1018500026EE800A81ED017A81ED000AC1ED027A5F
:10186000704700BF2DE9F04FAB490B7813F0010F23
:1018700087B003F0040200F07981002A40F08381F0
:10188000A648066816F0806640F07D81980700F152
:101890006D8143F004030B70A14BA24F1A88A24B39
:1018A0001A803B681B0340F11E81A04B80201E70F4
:1018B000FEF7DAFB08B1FFF739F99D4C2578012DC9
:1018C00040F011819B4B93F8F61721B193F8F7275D
:1018D0000AB1914203D3012283F8F62711E096461C
:1018E0000846BEF1000F06D090FBFEFC0EFB1C0C60
:1018F0007046E646F5E791FBF0F183F8F61792FBA8
:10190000F0F283F8F72793F8F8271AB1894A0021F3
:1019100082F8F81793F8F897B9F1000F2ED18020CC
:10192000F7F734FC804648B38021F7F709FC98F8B4
:101930000620814B607053F8223098F90000B3F50F
:10194000613F0CBF0222002202218DE806004A46B8
:101950008021F7F73FFA794B60601B684FF4FA7209
:1019600003EB4303B3FBF2F31BB1402BA8BF4023AF
:1019700000E00123DFF8B881237208B90023B1E049
:1019800008F10C000021142203F04BFF08F12C0396
:10199000C8F8203008F1A003C8F8243008F58A738D
:1019A000C8F82830664B634A1B88A8F8883192F83B
:1019B0009231396892F8F68792F884A1002B614B36
:1019C00018685379A3F1190EC1F3C03C18BF4FF04A
:1019D000010CDEF1000747EB0E07012B14BF3B465D
:1019E0000123049392F8F737574F05979845574BC3
:1019F000D7F800E01B78039301F40069C0F3800B73
:101A0000C1F34001C0F3C0002CBF4FF000084FF0FD
:101A100001086A1ED2B2531E132B3DD8DFE803F033
:101A20000C0C0C0C0C0C0C0C0AADAF292B3F371214
:101A30001212393F049BA3E0039B9342B4BF0023DF
:101A4000012328E09EF80030022B0BD10EEB82031D
:101A500053ED027AF5EE407AF1EE10FA14BF01234D
:101A6000002318E00EEB02035B79003318BF01235B
:101A700011E00B4684E0B9F1000F04D00AF1FF3702
:101A80007B427B4100E04B4603F0010378E0634674
:101A900076E0434674E013B1012393401E43142DB6
:101AA00002D80135EDB2B4E7059BC4F88C61186823
:101AB00019218530F7F7FCFB0023C4F89431A4F812
:101AC0009831A4F89A31C4F8A431C4F8A831204B55
:101AD000D4F8A0211B68C4F8AC3184F89001C4F894
:101AE0009C21022323701A4B124A1B6892F8E021B2
:101AF0004FF47A7101FB0233164A1360094B1B68DD
:101B00001A062DD5144B1B789B0729D5134B1B7830
:101B1000042B25D9062024E0A62F00207C110020CC
:101B200060120020741A00209E0F0020812A0020DD
:101B30006C2C00207012002004810108E0110020AC
:101B4000F41E00208C1A0020B8110020482B002021
:101B500048120020580F0020901A0020961A0020EA
:101B6000052007B0BDE8F04FFFF79EBB5AB9012032
:101B700007B0BDE8F04FFFF7C7BB034600E05B4688
:101B8000002B89D18DE707B0BDE8F08F10B5154A5D
:101B90001378590725D523F004031370124B1B68E3
:101BA0001B0319D5114C2378A3F10802012A0BD885
:101BB000FF200021F6F76EF90D4B1B68C4F8AC311D
:101BC000FEF7AEFD0A2306E0012B05D90A2B03D050
:101BD000FEF78CFD012323700420BDE81040FFF7C1
:101BE00063BB10BDA62F0020741A00206C2C0020AF
:101BF0004812002040F2E9330F4A1289920704D4B8
